:100000000C94BD300C94EE300C94EE300C94EE3029
:100010000C94EE300C94BBEE0C94EE300C94EE305D
:100020000C944CF20C94EE300C94359C0C94EE3005
:100030000C94EE300D94844D0C94EE300C94EE3014
:100040000C94EE300C94F0B00C94EE300C94EE3036
:100050000C94EE300C94EE300D94053B0D94D28848
:100060000C94EE300C941EAD0C94EE300C94EE30EB
:100070000C94EE300C94EE300C94EE300C94EE3088
:100080000C94EE300C94EE300C94EE300C94EE3078
:100090000C94DAAC0C94EE300C94EE300C94EE3000
:1000A0000C94EE300C94EE300C94EE300C94EE3058
:1000B0000C94EE300C94EE300C94EE300C94EE3048
:1000C0000C94EE300C94EE300C94EE300C944AC448
:1000D0000C94EE300C94EE300C94EE300C94EE3028
:1000E0000C94EE30D79ADB9AE19AEA9A039B209B14
:1000F0005D9B949B64D97AD98DD99AD9A4D9D2D948
:10010000F3D9F9D907DA0ADA0CDA16DA27DA38DAA3
:10011000F201DA015C01C0016001B8018001C8018F
:10012000CA01B801B801B801B801B801B801EA01C3
:10013000B801B801B801B801B801B801B801B801F7
:10014000B8014E017E01BE018201AE019601560149
:10015000FC01C201D0010E027A019A015801CC01C2
:100160003801A4013E0146018C01F801B2019C0155
:100170007801040290013E01A801E801E601F001C6
:10018000E401EE015A01A201D2017001EC0110025A
:10019000860194017401C401DC01D201B601F401AD
:1001A000B401084AD73B3BCE016E84BCBFFDC12FD2
:1001B0003D6C74319ABD56833DDA3D00C77F11BE58
:1001C000D9E4BB4C3E916BAAAABE000000803F055B
:1001D000A84CCDB2D44EB93836A9020C50B991868C
:1001E00088083CA6AAAA2ABE000000803F076342F6
:1001F00036B79BD8A71A39685618AEBAAB558C1DBE
:100200003CB7CC5763BD6DEDFD753EF6177231BF3F
:10021000000000803F08000000BE922449123EAB5F
:10022000AAAA2ABECDCCCC4C3E00000080BEABAA10
:10023000AAAA3E00000000BF000000803F000000AE
:100240000000084178D3BB4387D1133D190E3CC34E
:10025000BD4282AD2B3E68EC8276BED98FE1A93ECD
:100260004C80EFFFBE01C4FF7F3F00000000000094
:100270000D94F9830D9450000D94368A0D943D84AD
:100280000D9427010D942A250D94CD4C0D940A84CC
:100290000D9490020D94F2340D94AC1F0D94EE2940
:1002A0000D9424250D94228B0D948E000D943E55B3
:1002B0000D9406840D946F860D94B6260D94FF065A
:1002C0000D9481260D941C890D9496250D94AE01F4
:1002D0000D948B010D94EB510D94374C0D947D8949
:1002E0000D9483860D94D91F0D94B1860D94BE9BF9
:1002F0000D9422840D9485550D94CA1F0D94F654C7
:100300000D9419270D940A550D94E58A0D949D8638
:100310000D9430250D943A070D940E840D94118B95
:100320000D942A840D94CF1F0D94A7860D943855F3
:100330000D949C250D9403840D941C840D94F9A6B2
:100340000D94548A0D9479860D94FF830D9498250D
:100350000D9430840D9427250D94414C0D941C551B
:100360000D941E000D9418840D94E8860D94D48687
:100370000D94FC290D9494250D94C88A0D94045570
:100380000D949F260D9452550D94C0860D94CA006D
:100390000D944A280D94CC280D94F5830D94C51F17
:1003A0000D9460550D94F2860D942D250D94AB8A15
:1003B0000D94464C0D94F5260D94CA860D943B4C35
:1003C0000D944A890D94B8890D9460860D943884F3
:1003D0000D9434840D943D290D948B860D9465867F
:1003E0000D945B860D94EE260D94DE860D946900C7
:1003F0000D9414840D94D41F0D9444550D948E8A3D
:100400000D9499340D94028B0D9426840D94BF4C59
:100410000D9459010D94EB000D949A250D946E5591
:100420000D9493860D94718A6E616E00696E6600FC
:100430004E414E494E495459494E46CDCCCC3D0AC9
:10044000D7233C17B7D13877CC2B329595E6241FAC
:10045000B14F0A000020410000C84200401C462065
:10046000BCBE4CCA1B0E5AAEC59D7400407A10F338
:100470005A00A0724E18090010A5D4E80000E876D2
:1004800048170000E40B54020000CA9A3B00000029
:10049000E1F505000080969800000040420F000042
:1004A00000A08601000000102700000000E8030003
:1004B0000000006400000000000A000000000001CD
:1004C00000000000002C76D888DC674F0823DFC1CD
:1004D000DFAE59E1B1B796E5E3E453C63AE6519988
:1004E0007696E8E6C28426EB898C9B62ED407C6FB1
:1004F000FCEFBC9C9F40F2BAA56FA5F490055A2A68
:10050000F75C936B6CF9676DC11BFCE0E40D47FE73
:10051000F520E6B500D0ED902E0300943577050068
:1005200080841E080000204E0A000000C80C3333EF
:1005300033330F986E12831141EF8D2114893BE6FE
:100540005516CFFEE6DB18D1844B381BF77C1D9087
:100550001DA4BBE424203284725E228100C9F124F0
:10056000ECA1E53D276364696E6F70737578585B25
:1005700000256420627974657320777269747465EC
:100580006E20746F20454550524F4D20617420619C
:100590006464726573732030782530347800443396
:1005A000202D20526561642F57726974652045457E
:1005B00050524F4D0A0020436F756E7420583A20F8
:1005C000005344207072696E74696E67206279749A
:1005D0006520004E6F7420696E206661726D206D1B
:1005E0006F64652E00416374697665204578747286
:1005F000756465723A2000496E76616C69642065A5
:1006000078747275646572005A204F6666736574FB
:1006100000556E6B6E6F776E20636F6D6D616E64EB
:100620003A2022007A5F6D61783A20007A5F6D6926
:100630006E3A2000795F6D61783A2000795F6D69CC
:100640006E3A2000785F6D61783A2000785F6D69BE
:100650006E3A20005265706F7274696E6720656E25
:100660006473746F70207374617475730000534900
:100670004C454E54004E4F524D414C002553204D99
:100680004F44453A2050657263656E7420646F6E06
:10069000653A2025643B207072696E742074696D20
:1006A000652072656D61696E696E6720696E206D87
:1006B000696E733A2025640A00456E642066696C91
:1006C00065206C69737400426567696E2066696CA9
:1006D00065206C6973740025643A2025640A000A59
:1006E00050494E44412074656D7065726174757235
:1006F000653A20252E3166205A2073686966742079
:10070000286D6D293A20252E3366000A53746570D2
:100710003A2025642F360A000A537465703A202562
:10072000642F362028736B6970706564290A5049FC
:100730004E44412074656D70657261747572653ADE
:10074000202564205A20736869667420286D6D29FD
:100750003A300A000A5A45524F3A20252E33660A8B
:100760000073746172742074656D70657261747564
:1007700072653A20252E31660A0025642020252E38
:10078000326600255320583A20252E356620593AE6
:1007900020252E3566205A3A20252E35660A004E31
:1007A0006F7420696E206661726D206D6F64652EB6
:1007B0000025640045303A25642052504D0A5052BD
:1007C0004E303A25642052504D0A00256400417590
:1007D000746F0020452F443D00416476616E63656F
:1007E000204B3D004D3232302053256900255346C1
:1007F000696C616D656E742073657474696E67737E
:100800003A2044697361626C65640A002553466945
:100810006C616D656E742073657474696E67733A8C
:100820000A25532020204D3230302044252E3266B8
:100830000A002553526574726163743A20533D4C2B
:10084000656E67746820286D6D2920463A5370657F
:10085000656420286D6D2F6D29205A3A205A4C6905
:10086000667420286D6D290A25532020204D3230D2
:10087000372053252E32662046252E3266205A25F3
:100880002E32660A25535265636F7665723A20539D
:100890003D4578747261206C656E67746820286DC0
:1008A0006D2920463A537065656420286D6D2F6D63
:1008B000290A25532020204D3230382053252E324E
:1008C000662046252E32660A25534175746F2D52D7
:1008D0006574726163743A20533D3020746F2064F4
:1008E000697361626C652C203120746F20696E74AD
:1008F00065727072657420657874727564652D6FA9
:100900006E6C79206D6F76657320617320726574EB
:100910007261637473206F72207265636F766572A3
:100920006965730A25532020204D32303920532524
:10093000640A002553504944206865617462656407
:100940002073657474696E67733A0A2553202020FA
:100950004D3330342050252E32662049252E326604
:100960002044252E32660A002553504944207365E1
:100970007474696E67733A0A25532020204D333012
:10098000312050252E32662049252E3266204425FE
:100990002E32660A00255353746570732070657299
:1009A00020756E69743A0A255320204D393220583B
:1009B000252E32662059252E3266205A252E326683
:1009C0002045252E32660A25534D6178696D756D77
:1009D00020666565647261746573202D206E6F7288
:1009E0006D616C20286D6D2F73293A0A25532020E4
:1009F0004D3230332058252E32662059252E32664E
:100A0000205A252E32662045252E32660A25534D62
:100A10006178696D756D2066656564726174657372
:100A2000202D20737465616C746820286D6D2F73A0
:100A3000293A0A255320204D3230332058252E32B2
:100A4000662059252E3266205A252E3266204525ED
:100A50002E32660A25534D6178696D756D2061638C
:100A600063656C65726174696F6E202D206E6F72A4
:100A70006D616C20286D6D2F7332293A0A25532041
:100A8000204D3230312058256C752059256C752049
:100A90005A256C752045256C750A25534D6178697A
:100AA0006D756D20616363656C65726174696F6EED
:100AB000202D20737465616C746820286D6D2F7310
:100AC00032293A0A255320204D3230312058256CE6
:100AD000752059256C75205A256C752045256C7537
:100AE0000A2553416363656C65726174696F6E3A80
:100AF00020533D616363656C65726174696F6E2C30
:100B000020543D7265747261637420616363656C27
:100B100065726174696F6E0A255320204D3230343E
:100B20002053252E32662054252E32660A25534145
:100B30006476616E636564207661726961626C657A
:100B4000733A20533D4D696E206665656472617429
:100B50006520286D6D2F73292C20543D4D696E2022
:100B600074726176656C2066656564726174652077
:100B7000286D6D2F73292C20423D6D696E696D754E
:100B80006D207365676D656E742074696D652028CE
:100B90006D73292C20583D6D6178696D756D2058F5
:100BA00059206A65726B20286D6D2F73292C2020C7
:100BB0005A3D6D6178696D756D205A206A65726B5A
:100BC00020286D6D2F73292C2020453D6D6178699B
:100BD0006D756D2045206A65726B20286D6D2F73D1
:100BE000290A255320204D3230352053252E3266D8
:100BF0002054252E32662042252E32662058252E7E
:100C000032662059252E3266205A252E326620451E
:100C1000252E32660A2553486F6D65206F66667310
:100C2000657420286D6D293A0A255320204D3230F5
:100C3000362058252E32662059252E3266205A2518
:100C40002E32660A004D4D55203C3D202746256436
:100C5000202564270A00504944204175746F74753B
:100C60006E652066696E69736865642120507574CD
:100C700020746865206C617374204B702C204B6964
:100C800020616E64204B6420636F6E7374616E74B8
:100C9000732066726F6D2061626F766520696E7475
:100CA0006F20436F6E66696775726174696F6E2E2F
:100CB0006800504944204175746F74756E652066F4
:100CC00061696C6564212074696D656F75740020BD
:100CD000403A00543A00423A005049442041757469
:100CE0006F74756E65206661696C6564212054655A
:100CF0006D706572617475726520746F6F206869BC
:100D0000676800204B643A2000204B693A2000209D
:100D10004B703A200020436C617373696320504923
:100D20004420002054753A2000204B753A200020C2
:100D30006D61783A2000206D696E3A200020643A97
:100D4000200020626961733A200020453A00205A51
:100D50003A0020593A0020453A00205A3A002059DA
:100D60003A00583A00005A30005A310059300059C0
:100D70003100583000583100456E642073746F7034
:100D8000732064696167002E0044656C6574696F47
:100D90006E206661696C65642C2046696C653A203A
:100DA0000046696C652064656C657465643A004E44
:100DB0006F74205344207072696E74696E670050BE
:100DC00072696E742073617665640053442070729A
:100DD000696E7420706175736564000A002F000AE3
:100DE000002F2F20616374696F6E3A63616E6365D3
:100DF0006C0043524153485F43414E43454C0043CE
:100E0000524153485F5245434F5645520043524169
:100E100053485F5245434F5645520022283229001D
:100E20005400496E76616C6964205420636F646578
:100E30002E00556E6B6E6F776E204D20636F64656C
:100E40003A202573200A006E6F2076616C69642059
:100E5000636F6D6D616E64002C20002C20002C20CF
:100E6000006E2F61002C20002C20002C20006E2F03
:100E700061002F00503A005761697420666F72203C
:100E800050494E4441207461726765742074656DE9
:100E900070657261747572653A004C414E4720531B
:100EA000454C20464F52434544002228312900300A
:100EB000303030303030302D303030302D30303038
:100EC000302D303030302D30303030303030303028
:100ED0003030300020555549443A00310020455803
:100EE0005452554445525F434F554E543A00507248
:100EF000757361206933204D4B3300204D414348C9
:100F0000494E455F545950453A00312E3000206219
:100F100061736564206F6E204D61726C696E20464E
:100F200049524D574152455F55524C3A687474705E
:100F3000733A2F2F6769746875622E636F6D2F7017
:100F40007275736133642F50727573612D466972C7
:100F50006D776172652050524F544F434F4C5F562E
:100F6000455253494F4E3A004649524D574152451A
:100F70005F4E414D453A50727573612D4669726DF1
:100F80007761726520004D31313320530020423AA1
:100F90000020453A00543A0020413A0020503A00DF
:100FA0002042403A0020403A00202F003A002054CE
:100FB00000202F0020423A00202F006F6B20543A6F
:100FC000002569206D696E2C2025692073656300FA
:100FD000496E76616C6964204D20636F64653A20C8
:100FE0002573200A00556E6B6E6F776E2047206365
:100FF0006F64653A202573200A004D65736820628E
:101000006564206C6576656C696E67206E6F742010
:101010006163746976652E000A002020000A4D6520
:1010200061737572656420706F696E74733A000A3B
:101030005A20736561726368206865696768743AED
:1010400020002C004E756D20582C593A2000206D40
:101050006963726F6E730045786365737369766553
:1010600020626564206C6576656C696E6720636FCD
:101070007272656374696F6E3A2000473238205788
:10108000300050494E44412070726F6265206361A8
:101090006C6962726174696F6E207374617274003E
:1010A000473238205730004D3234005345545F43A7
:1010B000484F505F005345545F535445505F0053B1
:1010C00045545F574156455F00544D435F004352BE
:1010D0004153485F005072657373206B6E6F6220DE
:1010E000746F2070726568656174206E6F7A7A6CB7
:1010F0006520616E6420636F6E74696E75652E0085
:10110000506C6561736520707265737320746865D7
:10111000206B6E6F6220746F20756E6C6F6164203F
:1011200066696C616D656E740052656D6F766520E1
:101130006F6C642066696C616D656E7420616E64AD
:1011400020707265737320746865206B6E6F622007
:10115000746F207374617274206C6F6164696E6760
:10116000206E65772066696C616D656E742E006116
:101170006E6420707265737320746865206B6E6F87
:101180006200496E736572742066696C616D656E8C
:101190007400436F6C6F72206E6F7420636F727295
:1011A0006563740046696C616D656E74206E6F7462
:1011B000206C6F61646564004368616E67656420DC
:1011C000636F72726563746C793F004C6F61646920
:1011D0006E6720636F6C6F72004368616E67652095
:1011E000737563636573732100506C65617365206B
:1011F0006F70656E2069646C657220616E64207228
:10120000656D6F76652066696C616D656E74206DC5
:10121000616E75616C6C792E005761732066696C24
:10122000616D656E7420756E6C6F6164207375639B
:101230006365737366756C3F00506C656173652000
:10124000757067726164652E004E657720666972FD
:101250006D776172652076657273696F6E20617655
:1012600061696C61626C653A0057616974696E67A7
:1012700020666F722050494E44412070726F626543
:1012800020636F6F6C696E670043726173682064DE
:10129000657465637465642E20526573756D652091
:1012A0007072696E743F0043726173682064657484
:1012B00065637465642E00457874727564657200A8
:1012C00043686F6F73652065787472756465723AF0
:1012D0000043686F6F73652066696C616D656E743D
:1012E0003A004D32303020496E76616C6964206579
:1012F0007874727564657220006F70656E00545268
:1013000049474745524544004E6F206D6F76652E24
:10131000005761697420666F7220757365722E2E96
:101320002E00536F6D652070726F626C656D206565
:101330006E636F756E74657265642C205A2D6C65D2
:1013400076656C6C696E6720656E666F7263656446
:10135000202E2E2E00537461626C6520616D6269CF
:10136000656E742074656D70657261747572652048
:1013700032312D323643206973206E6565646564B1
:101380002061207269676964207374616E642069EA
:10139000732072657175697265642E00506C6561A9
:1013A00073652072756E2058595A2063616C6962AA
:1013B000726174696F6E2066697273742E00536C6B
:1013C0006565702E2E2E0073746172740A0061645C
:1013D000635F696E69740A001B5B324A1B5B313BB9
:1013E00031484F726967696E616C20507275736124
:1013F0002069331B5B323B33485072757361205256
:101400006573656172636800466163746F72792009
:101410005245534554004E6F7620313420323031DE
:101420003800436F6D70696C65643A2000286E6FF8
:101430006E652C2064656661756C7420636F6E66E2
:10144000696729004E6F76203134203230313820E0
:1014500031363A33353A35360020332E352E302D9D
:101460005243312D313638380A002055706C6F6187
:101470006420696E2070726F677265737300205A02
:101480003A0020593A0020583A0043524153485FED
:1014900044455445435445445859004352415348E8
:1014A0005F444554454354454459004352415348D1
:1014B0005F444554454354454458004D323900502B
:1014C00072757361206933204D4B332072656164FE
:1014D000792E00426C61636B6F7574206F63637566
:1014E000727265642E205265636F76657220707229
:1014F000696E743F0053656C667465737420776918
:101500006C6C2062652072756E20746F2063616C54
:1015100069627261746520616363757261746520CC
:1015200073656E736F726C657373207265686F6D2F
:10153000696E672E00546865726520697320737444
:10154000696C6C2061206E65656420746F206D612C
:101550006B65205A2063616C6962726174696F6E99
:101560002E20506C6561736520666F6C6C6F772000
:10157000746865206D616E75616C2C2063686170A4
:101580007465722046697273742073746570732C6D
:101590002073656374696F6E2043616C6962726168
:1015A00074696F6E20666C6F772E005072696E746E
:1015B000657220686173206E6F74206265656E20AD
:1015C00063616C69627261746564207965742E2050
:1015D000506C6561736520666F6C6C6F7720746802
:1015E00065206D616E75616C2C2063686170746537
:1015F000722046697273742073746570732C207343
:10160000656374696F6E2043616C696272617469AD
:101610006F6E20666C6F772E004F6C64207365745C
:1016200074696E677320666F756E642E20446566FC
:1016300061756C74205049442C2045737465707337
:10164000206574632E2077696C6C20626520736559
:10165000742E005761726E696E673A20626F74680B
:10166000207072696E746572207479706520616E85
:1016700064206D6F74686572626F61726420747942
:101680007065206368616E6765642E005761726ED5
:10169000696E673A207072696E7465722074797031
:1016A00065206368616E6765642E005761726E69BC
:1016B0006E673A206D6F74686572626F6172642044
:1016C00074797065206368616E6765642E00202000
:1016D000506C616E6E6572427566666572427974B1
:1016E00065733A20002046726565204D656D6F7206
:1016F000793A2000204C61737420557064617465E0
:10170000643A2000506F77657255700045787465B3
:10171000726E616C2053504920666C61736820576B
:101720003235583230434C206E6F742072657370BE
:101730006F6E64696E672E006572726F72207772C9
:101740006974696E6720746F2066696C6500656EE8
:101750006473746F7073206869743A20006F6B0053
:1017600043726173684465746563742044495341EE
:10177000424C454400437261736844657465637408
:1017800020454E41424C45442100207C2041757447
:10179000686F723A200020536F667477617265201B
:1017A000526573657400205761746368646F6720C5
:1017B0005265736574002042726F776E206F757486
:1017C000205265736574002045787465726E616C93
:1017D00020526573657400446F6E6520736176698D
:1017E0006E672066696C652E0058595A2063616CDB
:1017F0006962726174696F6E20616C6C20726967D6
:1018000068742E20536B65772077696C6C20626555
:1018100020636F72726563746564206175746F6DA7
:1018200061746963616C6C792E0058595A20636148
:101830006C6962726174696F6E20616C6C20726990
:101840006768742E20582F59206178657320617263
:101850006520736C696768746C7920736B65776554
:10186000642E20476F6F64206A6F62210058595AB6
:101870002063616C6962726174696F6E206F6B2E98
:1018800020582F592061786573206172652070653A
:101890007270656E646963756C61722E20436F6E41
:1018A00067726174756C6174696F6E732100585949
:1018B0005A2063616C6962726174696F6E2066613F
:1018C000696C65642E2052696768742066726F6E59
:1018D000742063616C6962726174696F6E20706FED
:1018E000696E74206E6F7420726561636861626CEA
:1018F000652E0058595A2063616C6962726174697F
:101900006F6E206661696C65642E2046726F6E741E
:101910002063616C6962726174696F6E20706F69B7
:101920006E7473206E6F7420726561636861626C9F
:10193000652E0058595A2063616C6962726174693E
:101940006F6E206661696C65642E20506C656173F2
:101950006520636F6E73756C7420746865206D61AB
:101960006E75616C2E0058595A2063616C69627201
:101970006174696F6E20636F6D70726F6D697365EE
:10198000642E2052696768742066726F6E742063DB
:10199000616C6962726174696F6E20706F696E74D8
:1019A000206E6F7420726561636861626C652E00E1
:1019B00058595A2063616C6962726174696F6E2054
:1019C000636F6D70726F6D697365642E2046726F00
:1019D0006E742063616C6962726174696F6E2070ED
:1019E0006F696E7473206E6F7420726561636861D5
:1019F000626C652E0058595A2063616C696272618D
:101A000074696F6E206661696C65642E204265643E
:101A10002063616C6962726174696F6E20706F69B6
:101A20006E7420776173206E6F7420666F756E64BC
:101A30002E00506C6561736520706C616365207366
:101A40007465656C207368656574206F6E206865C9
:101A500061746265642E0044697374616E6365200D
:101A60006265747765656E20746970206F66207496
:101A70006865206E6F7A7A6C6520616E6420746888
:101A800065206265642073757266616365206861B4
:101A900073206E6F74206265656E207365742079A3
:101AA00065742E20506C6561736520666F6C6C6F79
:101AB0007720746865206D616E75616C2C20636899
:101AC00061707465722046697273742073746570F6
:101AD000732C2073656374696F6E2046697273742A
:101AE000206C617965722063616C696272617469EE
:101AF0006F6E2E00506C61636520612073686565B0
:101B000074206F6620706170657220756E646572F6
:101B100020746865206E6F7A7A6C652064757269CE
:101B20006E67207468652063616C696272617469B4
:101B30006F6E206F66206669727374203420706F38
:101B4000696E74732E20496620746865206E6F7A02
:101B50007A6C6520636174636865732074686520BE
:101B600070617065722C20706F776572206F666689
:101B700020746865207072696E74657220696D6D7D
:101B80006564696174656C792E00506C656173657C
:101B90002072656D6F766520737465656C2073685F
:101BA0006565742066726F6D206865617462656436
:101BB0002E00497320737465656C207368656574C5
:101BC000206F6E20686561746265643F00206F66F7
:101BD000203400536561726368696E6720626564D2
:101BE0002063616C6962726174696F6E20706F69E5
:101BF0006E7400206F662039004D656173757269DF
:101C00006E67207265666572656E636520686569DA
:101C1000676874206F662063616C696272617469C1
:101C20006F6E20706F696E7400506C656173652013
:101C3000636C65616E20746865206E6F7A7A6C657E
:101C400020666F722063616C6962726174696F6E85
:101C50002E20436C69636B207768656E20646F6E1D
:101C6000652E004175746F20686F6D650078797A14
:101C700063616C5F6D656173737572655F656E74CA
:101C800065720A0078797A63616C5F73706972615A
:101C90006C382063783D25642063793D2564207A83
:101CA000303D256420647A3D256420726164697545
:101CB000733D25642061643D25640A0078797A6368
:101CC000616C5F7365617263685A206E6F2073691F
:101CD000676E616C0A20783D256C6420793D256C27
:101CE00064207A3D256C640A00204F4E2D534947ED
:101CF0004E414C20617420783D256420793D256457
:101D0000207A3D25642061643D25640A0078797A53
:101D100063616C5F7365617263685A20783D256CFE
:101D20006420793D256C64207A3D256C640A000AA4
:101D300000253032780078797A63616C5F73636173
:101D40006E5F706978656C735F333278333220630D
:101D5000783D25642063793D2564206D696E5F7A46
:101D60003D2564206D61785F7A3D25640A00202559
:101D700032642025640A000A002530327800206D84
:101D8000696E3D2564206D61783D25642064696637
:101D90003D25640A006D61785F633D253264206DE6
:101DA00061785F6C3D25640A006D61785F633D2555
:101DB00064206D61785F723D2564206D61785F6D90
:101DC000617463683D25640A0020783D25642079AC
:101DD0003D2564207A3D25640A0020706174746595
:101DE000726E20666F756E642061742025642025F4
:101DF000640A000000F000F801FC03FE07FE07FE85
:101E000007FE07FC03F801F000000073697A656FB4
:101E10006628746F74616C293D25640A0073697AC1
:101E2000656F6628626C6F636B5F6275666665726C
:101E3000293D25640A0078797A63616C5F6D65617C
:101E400073737572655F6C656176650A00706F69A2
:101E50006E743D256420783D256420793D256420FD
:101E60007A3D25640A0058025802584D584DB00476
:101E7000F055F055B00478797A63616C5F66696EED
:101E8000645F6265645F696E64756374696F6E5FD9
:101E900073656E736F725F706F696E745F787920AF
:101EA000783D256C6420793D256C64207A3D256C55
:101EB000640A00203C20005741524E494E473A20C8
:101EC00046726F6E7420706F696E74206E6F74202E
:101ED000726561636861626C652E205920636F6F63
:101EE0007264696E6174653A000000004041000050
:101EF000C04000005C430000C04000005C430000A4
:101F000046430000404100004643497465726174D5
:101F1000696F6E3A200043616C6962726174696F27
:101F20006E206661696C65642120436865636B207F
:101F3000746865206178657320616E642072756EC7
:101F400020616761696E2E00773235783230636CBC
:101F50005F63666D0A00773235783230636C5F6597
:101F60006E7465720A00504154393132355F524502
:101F7000535F593D256868750A0050415439313224
:101F8000355F5245535F583D256868750A002074D7
:101F90006F6F206C6F6E6720657874727573696FF0
:101FA0006E2070726576656E7465640020636F6C78
:101FB0006420657874727573696F6E2070726576CF
:101FC000656E74656400256920686F7572732025DD
:101FD00069206D696E757465730054494D454F55A0
:101FE000543A004D3131300046756C6C2052582007
:101FF000427566666572006673656E736F725F73B5
:10200000746F705F616E645F736176655F70726933
:102010006E740A006673656E736F725F72657374B7
:102020006F72655F7072696E745F616E645F636F1B
:102030006E74696E75650A0044495341424C4544CB
:102040000A00454E41424C4544004653656E736F4D
:10205000722025530A00504154393132355F696E80
:1020600069743A256868750A00504154393132352F
:102070005F696E69743A256868750A005041543981
:102080003132355F696E69743A256868750A0050A7
:10209000415439313235206E6F7420726573706F20
:1020A0006E64696E672028256429210A00446F6EDA
:1020B00065207072696E74696E672066696C650070
:1020C0004E6F204C696E65204E756D62657220778B
:1020D00069746820636865636B73756D2C204C614F
:1020E0007374204C696E653A20004C696E65204E11
:1020F000756D626572206973206E6F74204C617318
:1021000074204C696E65204E756D6265722B312CA2
:10211000204C617374204C696E653A2000667365CB
:102120006E736F725F6175746F6C6F61645F63680B
:1021300065636B5F7374617274202D206175746FB9
:102140006C6F616420454E41424C45440A00667301
:10215000656E736F725F6175746F6C6F61645F63DE
:102160006865636B5F73746F70202D206175746F89
:102170006C6F61642044495341424C45440A00530A
:10218000544F505045442E20005072696E74657251
:102190002073746F707065642064756520746F209F
:1021A0006572726F72732E2046697820746865209C
:1021B0006572726F7220616E6420757365204D398F
:1021C000393920746F20726573746172742E2028FF
:1021D00054656D70657261747572652069732072E3
:1021E000657365742E20536574206974206166746C
:1021F00065722072657374617274696E6729004E2E
:102200006F20436865636B73756D20776974682010
:102210006C696E65206E756D6265722C204C617301
:1022200074204C696E653A2000636865636B737552
:102230006D206D69736D617463682C204C617374DB
:10224000204C696E653A200053657474696E67733B
:102250002053746F7265640053746F7265642073E9
:10226000657474696E6773207265747269657665EA
:10227000640048617264636F6465642044656661EC
:10228000756C742053657474696E6773204C6F614C
:1022900064656400563200000000C8420000C84275
:1022A0000000C84300008C4300004843000048433E
:1022B000000040410000F042E8030000E803000095
:1022C000C80000008813000000409C4400409C446B
:1022D0000000000000000000204E0000000020412F
:1022E00000002041CDCCCC3E00002040000000008A
:1022F0000000000000000000CDCCCC3E3D0A814132
:10230000FF08433EB099AB438F42FC42E65A343F4C
:102310004C62B04500000000004040000034420024
:102320000000000000000000000041000000E03F4D
:102330000000C8420000C842000040410000F042D6
:10234000C0030000C0030000C800000088130000A4
:10235000454550524F4D204572726F7200436F6E6B
:1023600074696E7565207769746820616E6F746832
:10237000657220626F7764656E3F00250020202023
:1023800020202000202020202020004552415349B9
:102390004E4720616C6C2064617461004661637417
:1023A0006F72792052455345540000007F430080EE
:1023B00054430000524300000000000080C09A997E
:1023C000193E00000000000080C09A99193E24F4D4
:1023D000D43050C38E20C2A24017828B7011127A63
:1023E000910D816CD90AA861E108C758660761514F
:1023F00043061E4B5D05C145A7041A411104093D62
:102400009803713931034036DB0265339102D430D1
:102410005402802E1D02632CEE01752AC501B028DE
:10242000A001102781018F2564012B244B01E0229C
:102430003401AC211F018D200D01801FFC00841E82
:10244000ED00971DDF00B81CD200E61BC600201B64
:10245000BC00641AB200B219A8000A19A0006A18D8
:102460009900D117910040178B00B51684003116E2
:102470007E00B31579003A157300C7146F00581425
:102480006A00EE1366008813630025135E00C7120E
:102490005B006C12570015125400C11151007011ED
:1024A0004F0021114B00D61049008D1047004610F7
:1024B000440002104200C00F4000800F3E00420F57
:1024C0003C00060F3B00CB0E3800930E37005C0E2D
:1024D0003500270E3400F30D3200C10D3100900D90
:1024E0003000600D2E00320D2D00050D2C00D90C92
:1024F0002B00AE0C2900850C29005C0C2700350C44
:1025000027000E0C2600E80B2400C40B2400A00BAF
:1025100023007D0B23005A0B2100390B2100180BDF
:102520002000F80A1F00D90A1E00BB0A1E009D0ADF
:102530001D00800A1D00630A1C00470A1B002C0AAC
:102540001B00110A1A00F7091A00DD091900C40955
:102550001900AB091900920917007B0918006309DB
:1025600017004C09160036091600200916000A0942
:102570001500F5081500E0081400CC081400B80890
:102580001400A4081400900813007D0812006B08C2
:1025900013005808120046081200340811002308DE
:1025A00011001208110001081100F0071000E007E7
:1025B0001000D0071000C0071000B0070F00A107DF
:1025C000100091070E0083070F0074070F006507C6
:1025D0000E0057070E0049070E003B070D002E079F
:1025E0000E0020070D0013070D0006070D00F90669
:1025F0000C00ED060D00E0060C00D4060C00C80629
:102600000C00BC060C00B0060C00A4060B009906DA
:102610000C008D060B0082060B0077060B006C0683
:102620000B0061060A0057060B004C060A00420622
:102630000A0038060A002E060A0024060A001A06B6
:102640000A001006090007060A00FD050900F40546
:102650000900EB050900E2050900D9050900D005CC
:102660000900C7050900BE050900B5050800AD054C
:102670000800A50509009C050800940508008C05C4
:102680000800840508007C050800740508006C0536
:102690000700650508005D050700560508004E05A2
:1026A0000700470507004005080038050700310509
:1026B00007002A050700230507001C05060016056C
:1026C00007000F0507000805060002050700FB04C8
:1026D0000600F5040700EE040600E8040600E20424
:1026E0000700DB040600D5040600CF040600C90479
:1026F0000600C3040600BD040600B7040600B104CA
:102700000500AC040600A6040600A00405009B0416
:10271000060095040500900406008A04050085045F
:102720000500800406007A040500750405007004A5
:1027300005006B04050066040500610405005C04E7
:10274000050057040500520405004D040500480427
:102750000500430405003E0404003A040500350466
:102760000500300404002C040500270404002304A1
:1027700005001E0404001A040400160405001104D8
:1027800004000D040400090405000404040000040E
:102790000400FC030400F8030400F4030400F00345
:1027A0000400EC030400E8030400E4030400E00375
:1027B0000400DC030400D8030400D4030400D003A5
:1027C0000400CC030400C8030300C503030024F481
:1027D00004D9201BC40C5C0E9804C4095F02650771
:1027E0007101F405F900FB04B30048048700C1033C
:1027F00069005803550003034500BE023A008402F5
:10280000310053022A002902250004022000E401BD
:102810001C00C8011900AF011700980114008401C1
:102820001300710110006101100051010E004301FD
:102830000D0036010B002B010B0020010B001501D0
:1028400009000C01090003010800FB000800F30067
:102850000800EB000700E4000600DE000600D800D8
:102860000600D2000600CC000500C7000500C2002B
:102870000500BD000400B9000400B5000400B1006B
:102880000400AD000400A9000400A5000300A2009C
:1028900003009F0004009B000300980003009500C4
:1028A000020093000300900003008D0002008B00E3
:1028B00003008800020086000200840003008100FB
:1028C00002007F0002007D0002007B000200790010
:1028D000020077000100760002007400020072001E
:1028E0000100710002006F0002006D0001006C0029
:1028F00002006A0001006900020067000100660032
:102900000100650001006400020062000100610036
:102910000100600001005F0002005D0001005C003A
:1029200001005B0001005A0001005900010058003D
:10293000010057000100560001005500010054003D
:10294000010053000000530001005200010051003B
:102950000100500001004F0001004E0000004E0039
:1029600001004D0001004C0001004B0000004B0035
:1029700001004A0001004900010048000000480031
:10298000010047000100460000004600010045002C
:102990000000450001004400010043000000430026
:1029A000010042000000420001004100000041001F
:1029B0000100400001003F0000003F0001003E0018
:1029C00000003E0001003D0000003D0001003C0011
:1029D00000003C0000003C0001003B0000003B0008
:1029E00001003A0000003A000100390000003900FF
:1029F00001003800000038000000380001003700F6
:102A000000003700010036000000360000003600EC
:102A100001003500000035000000350001003400E1
:102A200000003400000034000100330000003300D7
:102A300000003300010032000000320000003200CC
:102A400001003100000031000000310001003000C1
:102A5000000030000000300001002F0000002F00B7
:102A600000002F0000002F0001002E0000002E00AB
:102A700000002E0001002D0000002D0000002D00A0
:102A800000002D0001002C0000002C0000002C0094
:102A900000002C0001002B0000002B0000002B0088
:102AA00000002B0001002A0000002A0000002A007C
:102AB00000002A0001002900000029000000290070
:102AC0000000290000002900010028000000280063
:102AD0000000280000002800000028000100270056
:102AE000000027000000270000002700000027004A
:102AF000010026000000260000002600000026003D
:102B0000000026000100250000002500000025002F
:102B10000000250000002500000025000100240021
:102B20000000240000002400000024000000240015
:102B30000100230000002300000023000000230008
:102B400000002300000023000000230001002200F9
:102B500000002200000022000000220000002200ED
:102B600000002200010021000000210000002100DF
:102B700000002100000021000000210000002100D1
:102B800001002000000020000000200000002000C4
:102B900000002000000020000000200000002000B5
:102BA00001001F0000001F0000001F0000001F00A8
:102BB00000001F0000001F0000001F0001001E0099
:102BC00000001E0000001E0000001E000000544D0A
:102BD0004320445249564552204F56455254454D84
:102BE000500025632533642F25642563005A25365C
:102BF0002E326620005A2020202D2D2D2000256306
:102C00002533642525002D2D2D00253368686400AB
:102C100025335325337325250020534400202020DD
:102C200000555342002025753E2575002046257528
:102C30000020463020200025632D2D3A2D2D202008
:102C400000256325337568202563256300256325EA
:102C50003032753A2530327525632563007265730D
:102C6000756C742076616C75653A2025640A0020C5
:102C7000693D25326420636E743D2532642076619F
:102C80006C3D2532640A00636C7573746572733A27
:102C90000A0020693D25326420737465703D253239
:102CA000640A00736F727465642073616D706C6583
:102CB000733A0A00555341525432207278204675B7
:102CC0006C6C2121210A003A2000202020202020A5
:102CD0002020202020202020202020202000203AFA
:102CE0002000202020202020202020202020202004
:102CF00020202020202000202020202020202020F4
:102D0000202020200025730050494E444120486572
:102D10006174696E670054656D702E2063616C2E5E
:102D2000202020202020202020200043616C696288
:102D3000726174696F6E20646F6E650043616C69C7
:102D400062726174696E67205A0042656420646F24
:102D50006E65004265642048656174696E6700486D
:102D6000656174696E6720646F6E652E00486561E9
:102D700074696E670043686F6F736520636F6C6F73
:102D8000723A004661696C207374617473004D3748
:102D900030322043004661726D206E756D6265723F
:102DA000004D363030004D3234004D323320257323
:102DB00000052E2E00526573756D696E6720707266
:102DC000696E7400537570706F727400537461741F
:102DD00069737469637320200043616C6962726176
:102DE00074696F6E004175746F4C6F616420666921
:102DF0006C616D656E7400556E6C6F616420666900
:102E00006C616D656E7400456A6563742066696CFB
:102E1000616D656E74004C6F616420746F206E6F1D
:102E20007A7A6C65004C6F61642066696C616D65CF
:102E30006E74004E6F2053442063617264005072C0
:102E4000696E742066726F6D20534400526573750D
:102E50006D65207072696E740050617573652070C5
:102E600072696E7400507265686561740054756EA5
:102E700065004C6976652061646A757374205A0038
:102E8000496E666F2073637265656E0046696E6990
:102E90007368696E67206D6F76656D656E7473001B
:102EA000536F756E642020202020205B6C6F75644A
:102EB0005D00536F756E642020202020205B6D75AF
:102EC00074655D00536F756E64202020205B73690C
:102ED0006C656E745D00536F756E64202020202039
:102EE000205B6F6E63655D00536F756E64202020FC
:102EF0002020205B6C6F75645D00437261736820F5
:102F00006465742E20205B4E2F415D004372617317
:102F100068206465742E2020205B6F6E5D00437214
:102F2000617368206465742E20205B6F66665D00A7
:102F30004D6F6465202020205B537465616C74685C
:102F40005D004D6F646520202020205B4E6F726D08
:102F5000616C5D0046696C2E2073656E736F722024
:102F6000205B6F6E5D0046696C2E2073656E736F1B
:102F700072205B6F66665D004368616E6765206600
:102F8000696C616D656E7400466C6F770053706597
:102F900065640046616E2073706565640042656417
:102FA000004E6F7A7A6C650053657474696E67734E
:102FB000005072696E742061626F727465640059AA
:102FC0006573004E6F0053746F70207072696E7479
:102FD0000046696C6520696E636F6D706C65746521
:102FE0002E20436F6E74696E756520616E7977610E
:102FF000793F004D61696E00473830004D3435002F
:103000004D3435205A004737360057697A6172646B
:103010002073746174653A202564004469736162A9
:103020006C65206661726D206D6F6465004661722B
:103030006D206E756D626572004D3834004D34340C
:1030400000473238205700473939004469736162BC
:103050006C65206661726D206D6F64653F00436131
:103060006C69627261746500506C65617365206C97
:103070006F616420504C412066696C616D656E74AF
:103080002066697273742E00497320504C4120668B
:10309000696C616D656E74206C6F616465643F007E
:1030A00043616E63656C0046696C616D656E7400AA
:1030B00053656C65637420504C412066696C616D8A
:1030C000656E743A0052756E6E696E672057697A44
:1030D0006172642077696C6C2064656C657465202E
:1030E00063757272656E742063616C69627261747B
:1030F000696F6E20726573756C747320616E6420E5
:1031000073746172742066726F6D207468652062DA
:103110006567696E6E696E672E20436F6E74696EA7
:1031200075653F0050726568656174696E67206EF1
:103130006F7A7A6C652E20506C65617365207761BB
:1031400069742E00456A65637400556E6C6F616426
:103150000055736520756E6C6F616420746F20720A
:10316000656D6F76652066696C616D656E74203182
:103170002069662069742070726F7472756465735B
:10318000206F757473696465206F662074686520AC
:1031900072656172204D4D5520747562652E205503
:1031A000736520656A6563742069662069742069A7
:1031B000732068696464656E20696E207475626549
:1031C0002E004C6F6164696E672066696C616D6585
:1031D0006E7400506C6561736520696E73657274FE
:1031E00020504C412066696C616D656E7420746F6F
:1031F000207468652065787472756465722C20741B
:1032000068656E207072657373206B6E6F622074D8
:103210006F206C6F61642069742E00506C6561735F
:103220006520696E7365727420504C412066696C2C
:10323000616D656E7420746F2074686520666972B4
:1032400073742074756265206F66204D4D552C2077
:103250007468656E20707265737320746865206B86
:103260006E6F6220746F206C6F61642069742E0031
:10327000596F752063616E20616C7761797320727C
:103280006573756D65207468652057697A6172642D
:103290002066726F6D2043616C6962726174696F40
:1032A0006E202D3E2057697A6172642E00506C6545
:1032B00061736520636865636B206F757220686158
:1032C0006E64626F6F6B20616E6420666978207433
:1032D00068652070726F626C656D2E205468656E33
:1032E00020726573756D65207468652057697A6111
:1032F0007264206279207265626F6F74696E6720F4
:10330000746865207072696E7465722E00416C6C11
:1033100020697320646F6E652E204861707079207B
:103320007072696E74696E672100506C65617365B7
:1033300020636C65616E20686561746265642061FC
:103340006E64207468656E20707265737320746893
:1033500065206B6E6F622E00446F20796F75207749
:10336000616E7420746F20726570656174206C6189
:103370007374207374657020746F20726561646A61
:103380007573742064697374616E6365206265741B
:103390007765656E206E6F7A7A6C6520616E642049
:1033A000686561746265643F00492077696C6C20D0
:1033B000737461727420746F207072696E74206C03
:1033C000696E6520616E6420796F752077696C6C19
:1033D000206772616475616C6C79206C6F776572BF
:1033E00020746865206E6F7A7A6C6520627920722D
:1033F0006F746174696E6720746865206B6E6F62AC
:103400002C20756E74696C20796F7520726561630C
:1034100068206F7074696D616C2068656967687495
:103420002E20436865636B2074686520706963743F
:103430007572657320696E206F75722068616E64A5
:10344000626F6F6B20696E206368617074657220B3
:1034500043616C6962726174696F6E2E004E6F77A2
:1034600020492077696C6C2063616C6962726174B9
:10347000652064697374616E636520626574776545
:10348000656E20746970206F6620746865206E6FA9
:103490007A7A6C6520616E64206865617462656427
:1034A00020737572666163652E004973206974200C
:1034B000504C412066696C616D656E743F005365C8
:1034C0006C656374206E6F7A7A6C652070726568C3
:1034D0006561742074656D706572617475726520C4
:1034E0007768696368206D61746368657320796FBC
:1034F0007572206D6174657269616C2E004E6F7714
:1035000020492077696C6C20707265686561742051
:103510006E6F7A7A6C6520666F7220504C412E0077
:1035200049732066696C616D656E74206C6F6164AF
:1035300065643F0049732066696C616D656E742037
:1035400031206C6F616465643F004E6F77204920C5
:1035500077696C6C2070726568656174206E6F7A33
:103560007A6C6520666F7220504C412E004920779E
:10357000696C6C2072756E207A2063616C6962726E
:103580006174696F6E206E6F772E004E6F772072B8
:10359000656D6F766520746865207465737420703E
:1035A00072696E742066726F6D20737465656C202D
:1035B00073686565742E00506C6561736520726573
:1035C0006D6F7665207368697070696E67206865D5
:1035D0006C706572732066697273742E004920776F
:1035E000696C6C2072756E2078797A2063616C69E1
:1035F00062726174696F6E206E6F772E204974203D
:1036000077696C6C2074616B6520617070726F7883
:103610002E203132206D696E732E004669727374EC
:103620002C20492077696C6C2072756E2074686557
:103630002073656C667465737420746F20636865AD
:10364000636B206D6F737420636F6D6D6F6E20619F
:103650007373656D626C792070726F626C656D73E7
:103660002E0048692C204920616D20796F757220E9
:103670004F726967696E616C205072757361206961
:1036800033207072696E7465722E20576F756C648A
:1036900020796F75206C696B65206D6520746F20D3
:1036A000677569646520796F75207468726F7567D6
:1036B00068207468652073657475702070726F631C
:1036C0006573733F00452D636F7272656374005AB2
:1036D0002D636F727265637400592D636F7272652A
:1036E000637400582D636F72726563740041757462
:1036F0006F206465706C6574655B4E2F415D0041A1
:1037000075746F206465706C6574655B6F66665D6B
:10371000004175746F206465706C657465205B6F23
:103720006E5D00536F756E642020202020205B6C3E
:103730006F75645D00536F756E642020202020201B
:103740005B6D7574655D00536F756E64202020207D
:103750005B73696C656E745D00536F756E642020D9
:10376000202020205B6F6E63655D00536F756E6473
:103770002020202020205B6C6F75645D00536F72E9
:10378000743A2020202020205B6E6F6E655D005310
:103790006F72743A20205B616C7068616265745D61
:1037A00000536F72743A2020202020205B74696DD2
:1037B000655D005344206361726420205B6E6F720C
:1037C0006D616C5D0053442063617264205B666CC4
:1037D00073684169725D0052506920706F72742085
:1037E000202020205B6F6E5D0052506920706F7248
:1037F00074202020205B6F66665D0054656D702E1E
:103800002063616C2E2020205B6F6E5D0054656D1F
:10381000702E2063616C2E20205B6F66665D004C0D
:10382000696E2E20636F7272656374696F6E0046F5
:10383000616E7320636865636B20205B6F66665DF5
:103840000046616E7320636865636B2020205B6FA8
:103850006E5D00462E206175746F6C6F6164205B35
:103860006F66665D00462E206175746F6C6F6164D3
:1038700020205B6F6E5D00462E206175746F6C6F4B
:103880006164205B4E2F415D0046696C2E2073659C
:103890006E736F72205B4E2F415D004469736162ED
:1038A0006C65207374657070657273004D6F76651A
:1038B00020617869730054656D706572617475720A
:1038C000650054656D702E2063616C69627261746D
:1038D000696F6E0052657365742058595A20636190
:1038E0006C6962722E0053686F772070696E646134
:1038F000207374617465005049442063616C69628F
:10390000726174696F6E00426564206C6576656CE7
:1039100020636F7272656374004D65736820426541
:1039200064204C6576656C696E670043616C696202
:1039300072617465205A0043616C696272617465DA
:103940002058595A0053656C6674657374202020A2
:10395000202020202020004669727374206C617939
:1039600065722063616C2E0057697A617264004C45
:103970006F61642066696C616D656E742035004C02
:103980006F61642066696C616D656E742034004CF3
:103990006F61642066696C616D656E742033004CE4
:1039A0006F61642066696C616D656E742032004CD5
:1039B0006F61642066696C616D656E742031004CC6
:1039C0006F616420616C6C004C6F61642066696C8F
:1039D000616D656E742035004C6F61642066696CA2
:1039E000616D656E742034004C6F61642066696C93
:1039F000616D656E742033004C6F61642066696C84
:103A0000616D656E742032004C6F61642066696C74
:103A1000616D656E74203100456A65637420666966
:103A20006C616D656E74203500456A65637420664F
:103A3000696C616D656E74203400456A656374203D
:103A400066696C616D656E74203300456A656374E8
:103A50002066696C616D656E74203200456A65632D
:103A6000742066696C616D656E74203100506C6500
:103A70006173652070756C6C206F75742066696C5D
:103A8000616D656E7420696D6D6564696174656CE6
:103A90007900556E6C6F6164696E672066696C6150
:103AA0006D656E740057697A61726420656E64207A
:103AB00073746174653A2025640A00000021104285
:103AC0002063308440A550C660E770088129914A80
:103AD000A16BB18CC1ADD1CEE1EFF1311210027307
:103AE000325222B5529442F772D662399318837BD0
:103AF000B35AA3BDD39CC3FFF3DEE3622443342057
:103B0000040114E664C774A44485546AA54BB5281F
:103B1000850995EEE5CFF5ACC58DD55336722611E6
:103B2000163006D776F6669556B4465BB77AA7196F
:103B3000973887DFF7FEE79DD7BCC7C448E55886AE
:103B400068A7784008611802282338CCC9EDD98EBF
:103B5000E9AFF9488969990AA92BB9F55AD44AB746
:103B60007A966A711A500A333A122AFDDBDCCBBF0F
:103B7000FB9EEB799B588B3BBB1AABA66C877CE416
:103B80004CC55C222C033C600C411CAEED8FFDEC5F
:103B9000CDCDDD2AAD0BBD688D499D977EB66ED526
:103BA0005EF44E133E322E511E700E9FFFBEEFDDAF
:103BB000DFFCCF1BBF3AAF599F788F8891A981CA8C
:103BC000B1EBA10CD12DC14EF16FE18010A100C26B
:103BD00030E3200450254046706760B9839893FB1A
:103BE000A3DAB33DC31CD37FE35EF3B1029012F3BB
:103BF00022D2323542145277625672EAB5CBA5A86A
:103C00009589856EF54FE52CD50DC5E234C324A00A
:103C10001481046674476424540544DBA7FAB799F9
:103C200087B8975FE77EF71DC73CD7D326F236915A
:103C300006B01657667676154634564CD96DC90EC1
:103C4000F92FE9C899E9898AB9ABA94458654806AA
:103C5000782768C018E1088238A3287DCB5CDB3F59
:103C6000EB1EFBF98BD89BBBAB9ABB754A545A37FA
:103C70006A167AF10AD01AB32A923A2EFD0FED6C29
:103C8000DD4DCDAABD8BADE89DC98D267C076C644A
:103C90005C454CA23C832CE01CC10C1FEF3EFF5D39
:103CA000CF7CDF9BAFBABFD98FF89F176E367E559A
:103CB0004E745E932EB23ED10EF01E7C3C3E5E2BC7
:103CC0003D3F2F5B5D3B2C2A225C00222066616910
:103CD0006C65643A204275666665722066756C6C28
:103CE00021002200656E717565696E6720220020D3
:103CF000423A0020453A00543A00494E543400728A
:103D000065636F7665725F6D616368696E655F7329
:103D1000746174655F61667465725F706F776572F8
:103D20005F70616E69632C20696E697469616C20D3
:103D3000007265636F7665725F6D616368696E6559
:103D40005F73746174655F61667465725F706F77CD
:103D500065725F70616E69632C20696E6974696158
:103D60006C20004739322045005052555341207590
:103D7000766C6F004734205330004D323620532587
:103D80006C75004D3130362053004D3832004731CC
:103D9000204625640047312045322A6465666175F6
:103DA0006C745F72657472616374696F6E204634FF
:103DB0003830004731205A00204632303030002061
:103DC000590047312058004D383300506F736974E3
:103DD000696F6E20726561642066726F6D20656523
:103DE00070726F6D3A004D3233202573002E676379
:103DF0006F0046656564726174653A00473120451D
:103E00002D64656661756C745F726574726163744C
:103E1000696F6E20463438300047312045352046E2
:103E2000313230004D3833004D3139302053256464
:103E3000004D313039205325640047323820582056
:103E400059004731205A32352046383030006275EB
:103E500073793A2070617573656420666F722069AA
:103E60006E70757400627573793A20706175736550
:103E70006420666F72207573657200627573793A9B
:103E80002070726F63657373696E67002046004728
:103E900031205A0020460047312045004D3833007C
:103EA0006F6B0A0055564C4F202D20656E642025FF
:103EB000640A007374707325640A00776F726C640F
:103EC00020636F6F7264696E617465733A20282590
:103ED0002E33662C20252E33662C20252E33662982
:103EE0000A00706879736963616C20636F6F726434
:103EF000696E617465733A2028252E33662C20255F
:103F00002E33662C20252E3366290A0043757272E3
:103F1000656E7420706F73205A5F415849533A257B
:103F20002E33660A43757272656E7420706F73204B
:103F3000455F415849533A252E33660A004166745D
:103F400065722077616974696E6720666F7220748C
:103F5000656D703A0A43757272656E7420706F7386
:103F600020585F415849533A252E33660A437572EB
:103F700072656E7420706F7320595F415849533ACF
:103F8000252E33660A005265636F766572696E6727
:103F9000207072696E7420202020001B5B323B3140
:103FA00048416D6269656E743A2020256425631B63
:103FB0005B333B314850494E44413A202020202574
:103FC000642563001B5B303B31484E6F7A7A6C6529
:103FD0003A202020256425631B5B313B3148426534
:103FE000643A20202020202025642563001B5B31BB
:103FF0003B31485057523A20202020202025642E63
:1040000025303164561B5B323B31484245443A20EF
:10401000202020202025642E2530316456001B5B93
:10402000303B314842656C74207374617475731B46
:104030005B313B3248582025641B5B323B32485988
:1040400020256400464C4558202D20203234302F46
:1040500035300050502020202D20203235342F3193
:1040600030300048495053202D20203232302F313B
:1040700030300041425320202D20203235352F3161
:1040800030300050455420202D20203233302F383E
:104090003500504C4120202D20203231352F363034
:1040A00000414253202020202D20203235352F3151
:1040B0003030006E6F7A7A6C65202D2020323530DA
:1040C0002F30006661726D2020202D202032353087
:1040D0002F363000466C6173684169722049502068
:1040E000416464723A004D4D55322020202020203A
:1040F000204E2F4100756E6B6E6F776E0025642E1B
:1041000025642E25642D2564002046573A004D4D28
:10411000553220636F6E6E6563746564004E6F7612
:1041200020313420323031380045334476366675DC
:104130006C6C0045494E53795F31306100315F3717
:10414000356D6D5F4D4B33002D2D2D2D2D2D2D2DCE
:104150002D2D2D2D00207265706F20556E6B6E6FAA
:10416000776E0020332E352E302D5243312D3136CF
:104170003838004669726D776172653A0025642EA1
:1041800025642E25642E2564004D373032004D37CE
:104190003031004578747275646572006D6D000091
:1041A00059005800580059005A002563252E313215
:1041B000533A2573252B30362E336600436F6F6CD0
:1041C000646F776E00566F6C746167657300546539
:1041D0006D7065726174757265730042656C7420F0
:1041E00073746174757300457874727564657220B8
:1041F000696E666F0058595A2063616C2E206465A1
:104200007461696C7300446174653A00686F777417
:104210006F2E707275736133642E636F6D00666FFD
:1042200072756D2E707275736133642E636F6D00DD
:10423000707275736133642E636F6D0046696C61D3
:104240006D656E7420657874727564696E6720267A
:10425000207769746820636F727265637420636F7E
:104260006C6F723F00507265686561742074686598
:10427000206E6F7A7A6C6521004552524F523A0097
:104280004175746F6C6F6164696E672066696C61FB
:104290006D656E74206973206163746976652C2086
:1042A0006A75737420707265737320746865206B0F
:1042B0006E6F6220616E6420696E73657274206631
:1042C000696C616D656E742E2E2E00546F74616C76
:1042D000207072696E742074696D6500546F74612A
:1042E0006C2066696C616D656E74005072696E74E5
:1042F0002074696D650046696C616D656E7420752A
:10430000736564005269676874004C65667400598F
:104310002064697374616E63652066726F6D206DD1
:10432000696E0053657665726520736B657700531F
:104330006C6967687420736B6577004D6561737590
:1043400072656420736B6577005B303B305D207075
:104350006F696E74206F66667365740041646A7578
:104360007374696E67205A005265736574005265F4
:1043700061722073696465205B756D5D0046726FC4
:104380006E7420736964655B756D5D005269676862
:104390007420736964655B756D5D004C656674209F
:1043A00073696465205B756D5D0053657420746589
:1043B0006D70657261747572653A001B5B324A25D7
:1043C00053203A1B5B313B394825382E3266206D2D
:1043D0000A2553203A0A25376C6464203A2532684E
:1043E000686468203A253032686864206D001B5B81
:1043F000324A25533A1B5B313B364825382E32660C
:104400006D200A2553203A1B5B333B384825326424
:104410006820253032646D202530326473002536E3
:104420002E32666D6D004E2F41001B5B303B3048D5
:1044300025533A0A25530A25533A0A25533A001BB5
:104440005B303B3135484E2F41001B5B303B3135F3
:104450004825342E326601001B5B303B3048255323
:104460003A0A25530A25533A202025352E32660173
:104470000A25533A202025352E3266010020003EC1
:10448000003E0020003E003E0054656D7065726184
:10449000747572652063616C6962726174696F6EB4
:1044A000206661696C65642E20436F6E74696E7559
:1044B000652077697468207072657373696E672010
:1044C000746865206B6E6F622E0054656D70657246
:1044D00061747572652063616C6962726174696F81
:1044E0006E20646F6E652E20436F6E74696E756505
:1044F0002077697468207072657373696E672074C1
:104500006865206B6E6F622E005A3020284C45443F
:10451000206F6E2920005A3120284C4544206F66B8
:10452000662900502E492E4E2E442E412E207374A3
:104530006174650054656D70657261747572652093
:1045400063616C6962726174696F6E206661696C27
:1045500065640054656D7065726174757265206381
:10456000616C6962726174696F6E2069732066693B
:104570006E697368656420616E6420616374697636
:10458000652E2054656D702E2063616C69627261C6
:1045900074696F6E2063616E206265206469736167
:1045A000626C656420696E206D656E75205365745C
:1045B00074696E67732D3E54656D702E2063616C57
:1045C0002E004578747275646572004D6F766520B3
:1045D0005A004D6F76652059004D6F766520580062
:1045E0001B5B324A4372617368206465746563744F
:1045F000696F6E2063616E1B5B313B3048626520E2
:104600007475726E6564206F6E206F6E6C792069B0
:104610006E1B5B323B30484E6F726D616C206D6F6C
:104620006465001B5B324A5741524E494E473A1B64
:104630005B313B3048437261736820646574656325
:1046400074696F6E1B5B323B304864697361626CE6
:10465000656420696E1B5B333B3048537465616C45
:104660007468206D6F6465004175746F6C6F616470
:10467000696E672066696C616D656E742061766134
:10468000696C61626C65206F6E6C79207768656E0D
:104690002066696C616D656E742073656E736F72F0
:1046A000206973207475726E6564206F6E2E2E2ED5
:1046B000004552524F523A2046696C616D656E74E6
:1046C0002073656E736F72206973206E6F74207231
:1046D0006573706F6E64696E672C20706C656173B2
:1046E0006520636865636B20636F6E6E65637469D4
:1046F0006F6E2E00526573656E6400486561746963
:104700006E672064697361626C65642062792073EE
:1047100061666574792074696D65722E004B494C31
:104720004C45442E20005072696E74657220686199
:104730006C7465642E206B696C6C28292063616C35
:104740006C656421004D31303420496E76616C69AE
:104750006420657874727564657220004D3130355F
:1047600020496E76616C6964206578747275646541
:104770007220004D31303920496E76616C696420B9
:10478000657874727564657220004D323138204945
:104790006E76616C696420657874727564657220E8
:1047A000004D32323120496E76616C696420657843
:1047B000747275646572200025533A20256C640A72
:1047C00025530A002079645F6D696E3D2575207957
:1047D000645F6D61783D25752079645F6176673D22
:1047E00025752073685F6176673D25750A00207323
:1047F000745F73756D3D25752079645F73756D3DCC
:1048000025752065725F73756D3D25752065725F36
:104810006D61783D256868750A00004B494C4C3A3B
:104820002025640A006673656E736F725F6F715F37
:104830006D656173737572655F73746F702C20257D
:104840006868752073616D706C65730A00667365C6
:104850006E736F725F6F715F6D6561737375726593
:104860005F73746172740A004D36303000465345F0
:104870004E534F525F5245434F5645520066736543
:104880006E736F725F757064617465202D204D3694
:1048900030300A006673656E736F725F6572725FA7
:1048A000636E74203D20300A004731204533204696
:1048B00032303000473120452D3320463230300031
:1048C0004D3730310020573A0020453A00543A0025
:1048D0005A206C6976652061646A757374206F75FF
:1048E00074206F662072616E67652E205365747444
:1048F000696E6720746F20302E20436C69636B20D3
:10490000746F20636F6E74696E75652E005A206C2B
:104910006976652061646A757374206F7574206FA1
:10492000662072616E67652E2053657474696E67C8
:1049300020746F20300043757272656E7400557379
:10494000656420647572696E67207072696E7400A8
:104950005049442063616C2E2066696E69736865F6
:1049600064005049442063616C2E202020202020C8
:10497000202020202000506C6561736520776169DC
:1049800074004D313137204669727374206C61793F
:1049900065722063616C2E005072696E74207061C4
:1049A0007573656400496E76616C69642050494492
:1049B0002063616C2E20726573756C74732E204EAB
:1049C0006F742073746F72656420746F2045455056
:1049D000524F4D2E004D353030004731205A313581
:1049E00020463135303000473931004731205835C5
:1049F00030205931393020453020463730303000B2
:104A0000473930004D373032004D373032204300C7
:104A10004D3730322055004D373032004D3730326F
:104A20002043004731205A3135204631353030009F
:104A3000473931004731205835302059313930203D
:104A40004530204637303030004D3833004739305C
:104A5000004D3834004D313034205330004D38345F
:104A6000004D373032204300473120583130205933
:104A7000313830204634303030004731205A313020
:104A80002046313330302E303030004D313430203C
:104A90005330004D31303420533000473120452D04
:104AA000302E30373530302046323130302E3030F5
:104AB000303030004D31303700473120583530200C
:104AC0005935352045332E363237373300473120BC
:104AD00058323030205935352045302E343933386E
:104AE0003600473120583230302059373520453391
:104AF0002E3632373733004731205835302059377A
:104B0000352045302E34393338360047312058357A
:104B100030205939352045332E3632373733004768
:104B2000312058323030205939352045302E343933
:104B30003338360047312058323030205931313542
:104B40002045332E36323737330047312058353041
:104B500020593131352045302E343933383600472D
:104B6000312058353020593133352045332E3632F7
:104B70003737330047312058323030205931333500
:104B80002045302E36363137340047312058323008
:104B90003020593135352045322E36323737330003
:104BA00047312058313030205931353520453200D9
:104BB00047312058373520593135352045322E358B
:104BC000004731204631303830004731205A302EEE
:104BD0003135302046373230302E303030004731DA
:104BE0002058353020593135350047312046343092
:104BF0003030004D323034205331303030004731C6
:104C0000205A352046373230302E30303000473190
:104C100020452D312E353030303020463231303085
:104C20002E3030303030004D3833004739300047B7
:104C30003231004739322045302E3000473120587C
:104C40003130302E30204531322E35204631303053
:104C5000302E30004731205836302E302045392E46
:104C6000302046313030302E300047312058352E3C
:104C7000302045342E302046313030302E30004741
:104C800031205A302E32302046313030302E300034
:104C90004731205835352E302045323520463134C5
:104CA00030302E3000473120592D322E3020463101
:104CB0003030302E3000473120583234302E302002
:104CC0004532352E30202046323230302E300047EB
:104CD00039322045302E30004731205A302E3320D3
:104CE00046313030302E30004731205835352E30A7
:104CF0002045382E302046323030302E30004731BB
:104D00002058352E30204533322E30204631383071
:104D1000302E30004731205835352E302045333283
:104D20002E302046313037332E30004731205A3074
:104D30002E342046313030302E3000473120592D6E
:104D4000332E302046313030302E30004D38330095
:104D50004739322045302E3000473238004D31304F
:104D6000392053323135004D31393020533630003F
:104D70004D31343020533630004D313034205332F1
:104D80003135004D313037006F6B0A00737461723A
:104D9000740A004D4D5532206669726D77617265F7
:104DA0002076657273696F6E20696E76616C6964D6
:104DB0002E2052657175697265642076657273691B
:104DC0006F6E3A206275696C64206E756D626572F3
:104DD000202564206F72206869676865722E0066FE
:104DE0006C0A006E6B0A0046530A0052300A0045F6
:104DF000340A0045330A0045320A0045310A0045AD
:104E0000300A0055300A0043300A004C340A004C86
:104E1000330A004C320A004C310A004C300A00546C
:104E2000340A0054330A0054320A0054310A005440
:104E3000300A004D4D55203D3E2027434D44205221
:104E400045545259203078253258270A004D4D5587
:104E5000203D3E2027434D442041434B20307825C0
:104E60003258270A004D4D55203D3E20274572728D
:104E70006F20356D2054696D656F7574270A004D7C
:104E80004D55203D3E202766697854686550726F05
:104E9000626C656D2121270A004D4D55203D3E2055
:104EA000276F6B270A004D4D55203D3E20276F6B25
:104EB000203A29270A004D4D55203D3E2027776195
:104EC0006974696E6720666F722066696C616D65D2
:104ED0006E742040204D4B332053656E736F7227E4
:104EE0000A004D363030004D363030204155544F99
:104EF000004653454E534F525F5245434F5645521D
:104F000000256868750050300A0045450A004D4D7F
:104F100055203C3D202746696C616D656E74207399
:104F200065656E206174206578747275646572279A
:104F30000A0045450A004D4D55203C3D2027523082
:104F4000270A0045450A004D4D55203C3D20274588
:104F50002564270A0045450A004D4D55203C3D205B
:104F6000275530270A0045450A004D4D55203C3D48
:104F700020274330270A0045450A004D4D55203C67
:104F80003D20274C2564270A0045450A0045450A6F
:104F9000004D4D55203C3D2027542564270A0046EE
:104FA000530A0052300A0045340A0045330A0045CE
:104FB000320A0045310A0045300A0055300A0043E4
:104FC000300A004C340A004C330A004C320A004CC0
:104FD000310A004C300A0054340A0054330A005499
:104FE000320A0054310A0054300A004D4D55202D2C
:104FF00020454E41424C45440025686875005030BC
:105000000A0050300A004D4D552076657273696F65
:105010006E2076616C69640025750053320A0025A4
:1050200075004D4D55206E6F7420726573706F6EF4
:1050300064696E67202D2044495341424C45440029
:1050400053310A004D4D5520737461727473207290
:105050006573706F6E64696E670A004D4D55206E02
:105060006F7420726573706F6E64696E670A0000FA
:1050700000803F555585410000803F0000C8410039
:10508000000040555505420000C03F000048420066
:1050900000204055558542000070C1ABAAA64200D1
:1050A0000060C10000A0410000C0C000002041001D
:1050B000002041ABAA3A41000020C15555D540001F
:1050C0000048C2555505424D373031204530004D1E
:1050D000373031204531004D373031204532004DD9
:1050E000373031204533004D373031204534004DC5
:1050F000373031204534004D373031204533004DB5
:10510000373031204532004D373031204531004DA8
:105110003730312045300046696C616D656E742012
:105120006E72206F7574206F662072616E676521E4
:1051300000506C65617365207570646174652066EC
:1051400069726D7761726520696E20796F75722062
:105150004D4D55322E2057616974696E6720666F18
:10516000722072657365742E004D4D55204F4B2E85
:1051700020526573756D696E672E2E2E004D4D554C
:10518000204F4B2E20526573756D696E6720706FCE
:10519000736974696F6E2E2E2E004D4D55204F4B46
:1051A0002E20526573756D696E672074656D70652C
:1051B0007261747572652E2E2E00466978207468AF
:1051C0006520697373756520616E64207468656E0F
:1051D00020707265737320627574746F6E206F6EC9
:1051E000204D4D5520756E69742E00507265737395
:1051F00020746865206B6E6F6220746F2072657317
:10520000756D65206E6F7A7A6C652074656D70655A
:105210007261747572652E004D4D55206E65656422
:1052200073207573657220617474656E74696F6E36
:105230002E00506C656173652072656D6F76652018
:1052400066696C616D656E7420616E64207468655A
:105250006E20707265737320746865206B6E6F6268
:105260002E00456A656374696E672066696C616DBE
:10527000656E740025632533642F25642563000063
:105280000E1315110E000000041209120400000094
:105290001C1F11111F00000006191803130C000435
:1052A0000E1F041C000000040A0A0A0A11110E0055
:1052B0001F1511151F0000000103161C0800000037
:1052C00000110A04110A040C12120C00000000253F
:1052D00063252D3138532563002563252E31355341
:1052E0003A2573253364002563252E3132533A2540
:1052F000732500457872656D65207370616E206F4F
:105300006620746865205A2076616C75657321008B
:1053100000004041000000400000E4420000004066
:105320000000574300000040000057430000C44203
:105330000000E4420000C442000040410000C442BA
:1053400000004041000042430000E44200004243AC
:105350000000574300004243205B6F66665D0042D9
:105360006564206C6576656C696E67206661696C42
:1053700065642E2053656E736F72206469646E7469
:1053800020747269676765722E2044656272697362
:10539000206F6E206E6F7A7A6C653F20576169745A
:1053A000696E6720666F722072657365742E0010D7
:1053B00000C90210012C014001220170011801B046
:1053C000010E01F00104015002FA00B002F00030B9
:1053D00003E600D003DC009004D2007005C800A0F2
:1053E00006BE000008B400B009AA00D00BA00060FF
:1053F0000E960060118C000015820020197800C004
:105400001D6E00A0226400B0275A00902C500000AE
:10541000314600E0343C0010383200903A280060F9
:105420003C1E00A03D1400803E0A00203F0000709A
:10543000012C0190012701B0012201C0011D01F0E2
:105440000118011002130130020E016002090190DF
:10545000020401C002FF000003FA004003F50080CF
:1054600003F000D003EB002004E6007004E100E04C
:1054700004DC004005D700C005D2004006CD00D0B6
:1054800006C8008007C3003008BE00F008B900C09D
:1054900009B400B00AAF00B00BAA00D00CA5000000
:1054A0000EA000500F9B00C01096005012910000FB
:1054B000148C00C0158700B0178200B0197D00D091
:1054C0001B7800001E730040206E0090226900F0DF
:1054D00024640040275F0090295A00E02B550010FB
:1054E0002E500020304B0010324600E03341009037
:1054F000353C001037370070383200A0392D00B02D
:105500003A2800A03B2300603C1E00103D1900908B
:105510003D1400103E0F00703E0A00C03E05000022
:105520003F000090137D00B0157800F01773006005
:105530001A6E00F01C6900A01F640050225F00205A
:10554000255A00E0275500902A5000202D4B00A03E
:105550002F4600F031410010343C00F0353700A0F8
:1055600037320020392D00603A2800703B2300605C
:105570003C1E00203D1900C03D1400403E0F00A01D
:105580003E0A00F03E0500403F0000703FFBFF90E8
:105590003FF6FFB03FF1FFC03FECFFD03FE7FFE039
:1055A0003FE2FFF03FDDFFF03FD8FF20484F54457A
:1055B0004E4420544845524D414C2052554E41577F
:1055C00041590020484541544245442054484552E1
:1055D0004D414C2052554E41574159005448455277
:1055E0004D414C2052554E415741590042454420AF
:1055F000544845524D414C2052554E415741590057
:1056000020544845524D414C2052554E4157415926
:105610002028205052454845415420484F54454E7B
:1056200044290020544845524D414C2052554E418A
:10563000574159202820505245484541542048455B
:105640004154424544290050524548454154204563
:1056500052524F5200424544205052454845415411
:10566000204552524F52004572723A204D415854D3
:10567000454D50003A204578747275646572207308
:1056800077697463686564206F66662E204D4158A3
:1056900054454D50207472696767657265642021B6
:1056A000004572723A204D415854454D50204245B4
:1056B000440054656D70657261747572652068652B
:1056C00061746564206265642073776974636865DA
:1056D00064206F66662E204D415854454D5020740D
:1056E00072696767657265642021004572723A20AD
:1056F0004D494E54454D50204245440054656D700F
:105700006572617475726520686561746564206294
:105710006564207377697463686564206F66662EBC
:10572000204D494E54454D5020747269676765722B
:1057300065642021004572723A204D494E54454D12
:1057400050003A20457874727564657220737769E9
:105750007463686564206F66662E204D494E54451B
:105760004D5020747269676765726564202100740A
:105770006D63323133305F686F6D655F656E746580
:105780007228617865735F6D61736B3D3078253089
:105790003278290A00746D63323133305F686F6D7F
:1057A000655F6578697420746D63323133305F737F
:1057B000675F686F6D696E675F617865735F6D6164
:1057C000736B3D3078253032780A0043616E6E6F1E
:1057D0007420656E746572207375626469723A2014
:1057E0000053442063617264206F6B006F70656EBC
:1057F000526F6F74206661696C656400766F6C75BA
:105800006D652E696E6974206661696C656400530C
:105810004420696E6974206661696C00536F72740C
:10582000696E672066696C657300536F6D652066ED
:10583000696C65732077696C6C206E6F742062658B
:1058400020736F727465642E204D61782E204E6F28
:105850002E206F662066696C657320696E2031208A
:10586000666F6C64657220666F7220736F72746904
:105870006E67206973203130302E001F1F1F1F1FDD
:105880001F1F1F2E002E004E6F77206672657368F3
:105890002066696C653A20004E6F7720646F696EF0
:1058A000672066696C653A20002220706F730022C1
:1058B00020706172656E743A2200535542524F5502
:1058C00054494E452043414C4C20746172676574C5
:1058D0003A2200747279696E6720746F2063616C7C
:1058E0006C207375622D67636F64652066696C65F3
:1058F00073207769746820746F6F206D616E7920F2
:105900006C6576656C732E204D4158206C6576650C
:105910006C2069733A0057726974696E6720746FFE
:105920002066696C653A200046696C652073656C79
:105930006563746564002053697A653A200046699E
:105940006C65206F70656E65643A200046696C6115
:105950006D656E742073656E736F7200537761703E
:105960007065640046726F6E742F6C656674206695
:10597000616E7300417869730041786973206C65CA
:105980006E677468004C6F6F73652070756C6C6522
:105990007900456E6473746F70206E6F742068694F
:1059A0007400456E6473746F70004D6F746F720095
:1059B000456E6473746F707300576972696E672007
:1059C0006572726F7200426564202F2048656174B1
:1059D0006572004E6F7420636F6E6E6563746564EC
:1059E000004865617465722F546865726D697374DF
:1059F0006F7200506C6561736520636865636B202E
:105A00003A0053656C6674657374206572726F72C8
:105A100020210046696C616D656E742073656E733C
:105A20006F723A005072696E742066616E3A00457A
:105A3000787472756465722066616E3A0053656CA5
:105A40006674657374206661696C6564202000412A
:105A50006C6C20636F72726563742020202020209C
:105A600000436865636B696E672073656E736F7260
:105A7000732000436865636B696E6720626564200C
:105A80002020202000436865636B696E67205A20E0
:105A900061786973202000436865636B696E6720D5
:105AA000592061786973202000436865636B696ED3
:105AB0006720582061786973202000436865636B14
:105AC000696E6720686F74656E64202000436865A6
:105AD000636B696E6720656E6473746F70730045E5
:105AE00072726F72202D20737461746963206D650A
:105AF0006D6F727920686173206265656E206F76C4
:105B000065727772697474656E00436172642072A5
:105B1000656D6F766564004361726420696E7365BC
:105B200072746564002D2D2D2D2D2D2D2D2D2D2DD7
:105B30002D2D2D2D2D2D2D2D2D0043616C69627283
:105B40006174696E6720686F6D6500000000000079
:105B5000110A0450525553413344465700207930BE
:105B60003D25640A002078303D25640A004F4B0A29
:105B7000004552524F522061643D25640A002020A6
:105B8000207A303D25640A00207A303D25640A00E1
:105B90002079303D25640A002078303D25640A00D4
:105BA00078797A63616C5F66696E645F706F696E45
:105BB000745F63656E746572320A00462564202541
:105BC000640A00332E352E302D52433100726300AB
:105BD0006265746100616C7068610064657600786C
:105BE000797A63616C5F73706972616C322063787B
:105BF0003D25642063793D2564207A303D2564206D
:105C0000647A3D2564207261646975733D25642062
:105C100061643D25640A000102102020080810205C
:105C20004010204080020102010804020101020428
:105C300008102040808040201008040201800402E7
:105C4000018040201008040201080402010102043E
:105C50000810204080010204081020408010080431
:105C60000880102040044080102040048000002262
:105C700000250028002B002E003100340002010016
:105C800000050108010B01050505050705080808C1
:105C900008020202020A0A080804040404010101BD
:105CA00001010101010303030303030303040707C5
:105CB000070C0C0C0C0C0C0C0C0202020206060663
:105CC00006060606060B0B0B0B0B0B0B0B07070A46
:105CD0000A0A0A0A0A050505040404080802746D84
:105CE00063323133305F676F746F5F737465702038
:105CF0002564202564202564202564200A002E00C8
:105D00006F70656E206661696C65642C2046696CF5
:105D1000653A20000000A0400000A04000000040C4
:105D200025336420737465703D253264206D736380
:105D30006E743D2534640A0000007F4300805843A0
:105D40009AD95143FFFFFF46696C616D656E7420FF
:105D50006F7574206F662072616E67652025642000
:105D60000A0067636F64655F4D3730312062656795
:105D7000696E0A0057616974696E6720666F7220E8
:105D80006E6F7A7A6C6520616E6420626564206350
:105D90006F6F6C696E670053656C66207465737411
:105DA000204F4B0053656C662074657374207374C8
:105DB0006172742020006C63645F73656C66636855
:105DC00065636B5F617869732025642C2025640A04
:105DD000004D3834004731205A31352046313030BB
:105DE000300047323820570025632041584953205E
:105DF0005347313D25640A0041786973206C656E14
:105E000067746820646966666572656E63653A25C5
:105E10002E33660A004D6561737572656420617882
:105E20006973206C656E6774683A252E33660A00C4
:105E30004D3234004D3233202573006175746F2567
:105E4000692E670022206661696C65643A2042759C
:105E5000666665722066756C6C2100456E717565AD
:105E6000696E6720746F207468652066726F6E7447
:105E70003A2022004572726F723A002200456E711C
:105E80007565696E6720746F207468652066726F2F
:105E90006E743A2022006563686F3A004572723A68
:105EA000205052494E542046414E204552524F52A6
:105EB000005072696E742066616E2073706565644F
:105EC000206973206C6F776572207468656E206539
:105ED00078706563746564004572723A2045585461
:105EE000522E2046414E204552524F520045787462
:105EF00072756465722066616E20737065656420DA
:105F00006973206C6F776572207468656E206578A0
:105F1000706563746564002F2F20616374696F6E10
:105F20003A70617573650000002100240027002A83
:105F3000002D003000330001010000040107010AB8
:105F400001000020002300260029002C002F003231
:105F5000000001000003010601090100000A0B0214
:105F6000090C0D0E080703040100000000000000EA
:105F70000000000000000000000000000000000021
:105F800000000000000000121110000000000000DE
:105F90000000000000000000000000000000000001
:105FA00000000000000000000000000000000000F1
:105FB000002563252E3132533A2573252B30362E9A
:105FC000316600202020202020202020202020209A
:105FD00020202020202020003E003E0020003E0007
:105FE0003E0020004E6F74207370696E6E696E679C
:105FF000005370696E6E696E67004C656674206848
:106000006F74656E642066616E3F0046726F6E74D9
:10601000207072696E742066616E3F0046616E206A
:10602000746573740046696C2E2058643A25336495
:106030002059643A2533640A496E743A2025336442
:106040002020536875743A202533640046696C61DA
:106050006D656E742073656E736F720A6973206468
:10606000697361626C65642E001B5B303B30484E87
:106070006F7A7A6C652046414E3A2025346420526E
:10608000504D0A5072696E742046414E3A202025C8
:1060900034642052504D0A001B5B303B3048546F33
:1060A00074616C206661696C757265731B5B313B52
:1060B0003148506F776572206661696C75726573DF
:1060C0002020252D33641B5B323B314846696C61CF
:1060D0006D2E2072756E6F7574732020252D3364BC
:1060E0001B5B333B31484372617368202058202585
:1060F0002D336420205920252D3364001B5B303B59
:1061000030484C617374207072696E7420666169E6
:106110006C757265731B5B313B3148506F776572EC
:10612000206661696C757265732020252D33641BB0
:106130005B323B314846696C616D2E2072756E6F23
:106140007574732020252D33641B5B333B3148432A
:106150007261736820205820252D33642020592037
:10616000252D336400546F74616C004C617374208E
:106170007072696E74009E01760111241FBECFEF0C
:10618000D1E2DEBFCDBF00E00CBF16E0A0E0B2E080
:10619000E2E7F3E703E00BBF02C007900D92A63BD6
:1061A000B107D9F729E1A6EBB6E001C01D92A73DE2
:1061B000B207E1F710E3CCEBD0E300E006C0219793
:1061C0000109802FFE010F94C4B8CB3BD10780E0BA
:1061D0000807A9F70F94F88E0D94A8B90C94000045
:1061E0002F923F924F925F926F927F928F929F92E7
:1061F000AF92BF92CF92DF92EF92FF920F931F93D5
:10620000CF93DF93CDB7DEB7C757D1090FB6F89458
:10621000DEBF0FBECDBF8091981390919913892B4B
:1062200011F40C94DF6F82E090E09093230280934E
:10623000220288E393E00E949DA78823B1F0809119
:106240002B0D90912C0D6AE270E005960F9427B902
:10625000009711F0DC011C9280912B0D90912C0D78
:1062600005960F944E530C94FD6AC0908715D090FC
:106270008815860103561C4E46E050E06EEC70E136
:10628000C8010F945AAC892B09F0EFC08DE393E05D
:106290000E949DA7882309F49BC088E50F947E9BEC
:1062A000182F89E50F947E9B811112600F948683CD
:1062B0008091B70601E0080F0093B706811105C071
:1062C00084E696E10E9432DD0EC048EC5FEA60E0B1
:1062D00070E084E696E10E94EDDC882331F01092B4
:1062E00064161092B70601E007C0033049F7109218
:1062F00064161092B70600E081E00F9415370F94F2
:106300000B3782E00F94812F10FF15C086E69FE0C7
:106310000F9457B361E0680F86E69FE00F9469B36E
:1063200085E09FE00F9464B3BC016F5F7F4F85E011
:106330009FE00F9483B311FF15C088E69FE00F9490
:1063400057B361E0680F88E69FE00F9469B383E07C
:106350009FE00F9464B3BC016F5F7F4F83E09FE0C9
:106360000F9483B381E00F94153782E00F94812F4F
:1063700087EA92E10F94DC5140E061E081E00F9404
:10638000A96E0F948683002321F061E08DE09EE0EA
:106390001BC0E091FE0CF0E0EE0FFF1FE757FA4E36
:1063A0001182108240E060E089E892E10F94940746
:1063B000182F81E00F94153761E0112319F08FEF4A
:1063C0009DE002C082EF9DE00E9459DB0C94FD6AC3
:1063D0008CE493E00E949DA7882379F080913F0E82
:1063E000882331F060E070E080E89FE30E94CFE610
:1063F00081E080930C020C94FD6A8AE593E00E9490
:106400009DA7882311F40C94FD6A10923F0E81E041
:1064100080930C0280917C0E811104C00E94B2CE48
:106420000C94FD6A813011F00C94FD6AE1EEFDE000
:1064300084918F01882339F00E9462AD0F5F1F4F56
:10644000F8018491F7CF8AE00E9462ADEDE5F7E1B3
:1064500084918F01882311F40C948A690E9462ADA3
:106460000F5F1F4FF8018491F5CF44E050E069ECD5
:1064700070E1C8010F945AAC892B09F00EC1860156
:106480000F551C4E49E050E06FEB70E1C8010F94CE
:106490005AAC892BD9F4F601E655FC4E108115341F
:1064A00031F01855143010F00C94FD6A01C013E05F
:1064B0004AE050E060E070E0C60185559C4E0F94C4
:1064C00011AA812F0F94595B0C94FD6A49E050E0AA
:1064D00065EB70E1C8010F945AAC892B61F5F601A8
:1064E000E655FC4E1081153431F01855143010F07B
:1064F0000C94FD6A01C013E04AE050E060E070E0F7
:10650000C60185559C4E0F9411AAE12FF0E0E05F83
:10651000F84F40E051E0008002C0569547950A943C
:10652000E2F7842F880F880F81506823812F0F9402
:10653000075D0C94FD6A49E050E06BEA70E1C80128
:106540000F945AAC892B11F00C94FD6AF601E655B4
:10655000FC4E8081853449F008EA902E980EF3E0D5
:10656000F91510F40C94FD6A02C013E0912EE92C89
:10657000F12C5701AA0CBB1CF501EF5CFD4F1081FB
:10658000012F0F70712E7294BFE07B22272D277090
:10659000722E111F1127111F61816770660F162B54
:1065A000F501EE5CFD4F8081882E8694869486945A
:1065B000382D3370832E1A821982C60185559C4E60
:1065C000DC012C912223E1F14AE050E0BE016F5F33
:1065D0007F4F0F9411AA062F0F7089819A8100971F
:1065E00079F1FC012081222359F14AE050E0BE01FB
:1065F0006F5F7F4F0F9411AA6770762E89819A8101
:106600000097F1F0DC012C912223D1F04AE050E018
:10661000BE016F5F7F4F0F9411AA162F1F708981E3
:106620009A81009769F0FC012081222349F04AE019
:1066300050E0BE016F5F7F4F0F9411AA6370862EEA
:10664000F501EF5CFD4F972D97709295907F612F2C
:10665000679566276795902B962B9083612F66959B
:106660001181107E882D8370880F880F880F162B5C
:10667000182B1183C701875E9D4FD701A35EBD4FC5
:10668000B701605F784FFC0120814C91DB016C9178
:10669000892D0E94D5C60C94FD6A87E693E00E947E
:1066A0009DA7882321F00E94FF9E0C94FD6A87E736
:1066B00093E00E949DA7882309F4B5C18DE793E07C
:1066C0000E949DA7882391F08091C80F882311F420
:1066D0000C94FD6A0F94138860937A1670937B165E
:1066E00080937C1690937D160C94FD6A82E893E06B
:1066F0000E949DA7882349F08091E50E8F93809199
:10670000E40E8F938BEC97E03DC086E893E00E9407
:106710009DA7882329F140917813509179132CE398
:10672000249FC001259F900D11249F938F9340912A
:10673000761350917713249FC001259F900D11244B
:106740009F938F9384EB97E09F938F930F9487ADE4
:106750000F900F900F900F900F900F900C94FD6A78
:106760008AE893E00E949DA78823C9F08091C80F12
:10677000882391F080912A078F93809129078F9326
:1067800081EB97E09F938F930F9487AD0F900F90BD
:106790000F900F900C94FD6A8FE997E0F0C08DE8A0
:1067A00093E00E949DA7882321F0109228070C9463
:1067B000FD6A81E993E00E949DA7882349F060E08B
:1067C00085EA9FE00F9469B361E087EA90E1FCCD30
:1067D00086E993E00E949DA7882321F00F944E261E
:1067E0000C94FD6A8DE993E00E949DA7882319F11E
:1067F0008091C80F8823C9F08AEA95E5DC0180936F
:10680000FC1F9093FD1FA093FE1FB093FF1F88E015
:106810008093FB1F98E10FB6F894A89590936000C1
:106820000FBE80936000F894FFCF83EA93E00E944C
:106830009BAE0C94FD6A85EB93E00E949DA7882394
:1068400039F180912B0D90912C0D41E061E0039680
:106850000F94D3438091AE189091AF18A091B018C7
:10686000B091B11880935B1990935C19A0935D1956
:10687000B0935E1986EA98E10E9429E38C010E9498
:1068800062AD0A30110531F70F9425570C94FD6A5B
:1068900088EB93E00E949DA7882381F00F94AD665A
:1068A00081E080933B0780912B0D90912C0D41E06E
:1068B00060E004960F94D3430C94FD6A8CEB93E054
:1068C0000E949DA7882309F45EC08091C80F882389
:1068D00009F453C010928B156091D1197091D2199F
:1068E0008BE390E00F9402AD6091D1197091D219B1
:1068F00083E590E00F9402AD19821B821A82CE01CB
:1069000001960E94E1DC00E010E0FF24F394809106
:10691000EF0D9091F00D2091F10D3091F20D821B51
:10692000930B8F779927892B81F00E94BEACF09250
:106930008B156091D1197091D21990E00F9402AD2E
:106940000F5F1F4F10928B15E2CF64E670E0CE010F
:1069500001960E94B8DC811103C003311105BCF21D
:1069600081E080938B156091D1197091D2198AE0E2
:1069700090E00F9402AD0C94FD6A83ED95E00F94C6
:10698000AFAD0C94FD6A8FEB93E00E949DA7882326
:1069900061F003EC13E0F80181918F01882311F479
:1069A0000C948A690E9462ADF6CF82ED93E00E945A
:1069B0009DA7882361F006ED13E0D8018D918D012C
:1069C000882311F40C948A690E9462ADF6CF85EF9A
:1069D00093E00E949DA781110C94FD6A8AEF93E0D9
:1069E0000E949DA7882341F060E070E088EF9FE05F
:1069F0000E94ACFD0C94FD6A8DEF93E00E949DA770
:106A0000882321F00F9413880C94FD6A82E094E0AF
:106A10000E949DA7882311F40C94FD6A80E00E94D7
:106A200093A90C94FD6A8EE50F947E9B8AAF811129
:106A30000C94FD6A87E40F947E9BF82E882311F452
:106A40000C94BB420F94759B0F9442B56C34710546
:106A500009F404C27CF56430710509F4FCC054F4F7
:106A60006230710509F4E2C00CF0E9C077FF6DC037
:106A70000C94AF426C31710509F43FC15CF46A308B
:106A8000710509F435C16B30710511F00C94AF42FA
:106A900080E02FC16E31710509F471C16B3471054D
:106AA00011F00C94AF4208E210E0FAE7EF2EF7E0A5
:106AB000FF2EB5C16835710511F40C94FD6AECF434
:106AC0006135710511F40C94764154F46F347105FD
:106AD00009F431C76035710509F459C70C94AF4208
:106AE0006635710511F40C941F426735710511F07C
:106AF0000C94AF4281E00C9420426C35710511F486
:106B00000C9428427CF46A35710511F40C942442EB
:106B10006B35710511F00C94AF4281E08093FA0E51
:106B20000C94FD6A6236710511F40C948842633648
:106B3000710511F00C94AF421092C80F60E084EC24
:106B40009FE00F9469B30C94AA4280915E0F81116B
:106B50000C94FD6A0F949EA36091480E7091490EAB
:106B600080914A0E90914B0E0F9480AE6B017C0188
:106B7000409041105090421060904310709044102B
:106B80008090D50F9090D60FA090D70FB090D80FCF
:106B9000A5019401C301B2010F94E2B320E030E0FB
:106BA00048EC52E40F94E9A79B01AC01C701B60180
:106BB0000F942EB61816D4F4A3019201C501B401A6
:106BC0000F94E2B320E030E048EC52E40F94E9A7E0
:106BD000A70196010F94E3B30F9448B56093480E54
:106BE0007093490E80934A0E90934B0E8091FB1048
:106BF000882311F40C94FB6A88E50F947E9B811125
:106C00000C94FB6A89E50F947E9B81110C94FB6ABE
:106C10008AE50F947E9B81110C94FB6A85E40F94A6
:106C20007E9B81110C94D26A0C94FB6A80915E0F5A
:106C300081110C94FD6A0F945FA481E008C08091DB
:106C40005E0F81110C94FD6A0F945FA480E00F9495
:106C5000609D0C94FD6A80E50F947E9B882339F03B
:106C60000F94759B0F9448B56B017C0103C0C12C38
:106C7000D12C760183E50F947E9B882361F00F94DD
:106C8000759B20E030E04AE754E40F94E9A70F94A5
:106C900048B56B017C01C114D104E104F10421F079
:106CA0008EEB93E10F94DC510F9486830F9413883D
:106CB000C60ED71EE81EF91E0F9413886093FF0EB0
:106CC0007093000F8093010F9093020F0F9413881D
:106CD0006C157D058E059F0510F00C94FD6A0F94D0
:106CE000AA7D80E00F945C0E80E00F94812FEECFA0
:106CF00081E00F94F0A40C94FD6A88E50F947E9BCC
:106D00008EAF0F946A9B1B012C0189E50F947E9B2B
:106D1000682E0F946A9B26966CAF7DAF8EAF9FAFA7
:106D200026978AE50F947E9BD82E0F946A9B4B0181
:106D30005C0187E50F947E9B782E83E40F947E9B05
:106D40007F928F93CD2C2696ECACFDAC0EAD1FAD93
:106D50002697262DB201A1018EAD0F94C76B0F901F
:106D60000F90BEADB1110C94FD6A61100C94FD6AD8
:106D700071100C94FD6AD1100C94FD6A08C60F9432
:106D8000868381E00E94CFA58C0180E090E0A8E49A
:106D9000B4E480937E0290937F02A0938002B0932C
:106DA000810260E070E080E291EC0F948B42809170
:106DB00040108F9380913F108F9380913E108F935E
:106DC00080913D108F9380913C108F9380913B1068
:106DD0008F9380913A108F93809139108F93809187
:106DE00038108F93809137108F93809136108F9346
:106DF000809135108F938DE99FE29F938F9383E865
:106E000097E09F938F930F9487ADC8010E94AEA522
:106E10000FB6F894DEBF0FBECDBF0C94FD6AB8016B
:106E2000012E000C880B990B0F9482AE0F949C08D6
:106E30009F938F937F936F931F930F93FF92EF9284
:106E40000F9487AD0F5F1F4F0FB6F894DEBF0FBED4
:106E5000CDBF0F36110519F70C94FD6A0E94BAAC2C
:106E60008A3F30F08CE993E10F9435080C94FD6A69
:106E70008091FF0C882341F08091000D882321F040
:106E80008091010D811106C081E08093971380EA03
:106E900090E197C585E593E10F94350840E060E007
:106EA00082EB9BE10F949407882309F493C080E060
:106EB00090E0A0EAB0E480933D1090933E10A09340
:106EC0003F10B09340102091391030913A1040910A
:106ED0003B1050913C1060913510709136108091AC
:106EE000371090913810FEEF6F2EFCE07F2E7F92CE
:106EF0006F92812C912CA8E4AA2EA2E4BA2EB1E4C0
:106F0000CB2EB0E1DB2EE12CF12C00EA10E40E9444
:106F1000458780923D1090923E10A0923F10B09213
:106F2000401080E090E0A4E3B3E4809339109093A4
:106F30003A10A0933B10B0933C10609135107091C3
:106F4000361080913710909138107F926F928501A2
:106F5000740120E030E044E353E40E9445870F943D
:106F600086838AE89BE10F943508EEEEFEE12591D9
:106F70003591459154912093391030933A104093B4
:106F80003B1050933C10EAEEFEE1659175918591BE
:106F900094916093351070933610809337109093CE
:106FA0003810E0903D10F0903E1000913F1010918D
:106FB00040107F926F920E9445870F94868341E034
:106FC00060E080E00F94A96E0F900F900F900F90EB
:106FD0000F900F9020E030E04CE052E46091A10E61
:106FE0007091A20E8091A30E9091A40E0F942EB6D4
:106FF00018160CF0A4C08091C80F8111A0C080E0C9
:1070000090E0A8ECB2E480933D1090933E10A093E2
:107010003F10B09340102091391030913A104091B8
:107020003B1050913C10609135107091361080915A
:10703000371090913810EEEFFCE0FF93EF93812C26
:10704000912C18E4A12E12E4B12E01E4C02E00E12F
:10705000D02EE12CF12C08EC12E40E94458780E050
:1070600090E0ACE0B2E48F8F98A3A9A3BAA30F94E9
:10707000303219821A821B821C82CE0101960F9433
:107080006D761092030D1092020D19821A821B82E6
:107090001C821D82CE0101960E9432DD0F900F905E
:1070A0002F8D38A149A15AA16091A10E7091A20E15
:1070B0008091A30E9091A40E0F942EB6181694F5FD
:1070C00089E692E10F94870764E080E00F945C32D8
:1070D00082E00E94919A81EA9EE00E943AA00F9479
:1070E000FE3085E094E00F94FE30CE014F960E9472
:1070F0003AA00F94FE3087E094E00F94FE3088EEC3
:1071000093E00F94B1120E94BBF240E053E567E0B8
:1071100070E0CE0101960E94EDDC882309F4C0CF17
:1071200010E001C011E06BE47BE581E00F941132C7
:1071300081E00F941537111102C080E0F8C381E09F
:107140000F94153781E090E0909323028093220200
:10715000E2E8F0E184918F01882339F00E9462AD6A
:107160000F5F1F4FF8018491F7CF8AE00E9462AD54
:107170001A821982C090A10ED090A20EE090A30EA8
:10718000F090A40E20E030E040EA50E4C701B601E0
:107190000F94D1B40F9442B525E0269FA001279FFC
:1071A000500D1124BA01550F880B990B0F9482AE24
:1071B0003B01382E292E20E030E04CE052E40F94C1
:1071C0007CAE87FF06C0612C712CACE03A2EB2E495
:1071D0002B2EC101262D372D492F522DC701B60167
:1071E0000F942EB6181674F420E030E040EA50E414
:1071F000F101662D772D8F2F922D0F94E3B33B0174
:10720000382E292E2F923F927F926F9281E697E03F
:107210009F938F930F9487AD20E030E040EF51E4CF
:10722000F101662D772D8F2F922D0F94E2B320E080
:1072300030E04CE852E40F94E3B30F9442B57093FE
:10724000030D6093020D84E090E09093410E8093D3
:10725000400E81E090E09093260F8093250F86E109
:107260009DE20F94DC5180E090E0A0EAB0E48093CE
:107270003D1090933E10A0933F10B093401020918A
:10728000391030913A1040913B1050913C10609170
:107290003510709136108091371090913810BEEFF4
:1072A0004B2EBCE05B2E5F924F92812C912C18E408
:1072B000A12E12E4B12E01E4C02E00E1D02EE12C6B
:1072C000F12C00EA10E40E94458780E090E0A0EAFB
:1072D000B1E48093351090933610A0933710B0939B
:1072E000381080E090E0A0E7B2E4809339109093EA
:1072F0003A10A0933B10B0933C10E0903D10F090FA
:107300003E1000913F10109140105F924F929C01EF
:10731000AD0160E070E080EA91E40E9445878AE96F
:1073200099E9A9E1BEE380933D1090933E10A093AC
:107330003F10B09340102091391030913A10409195
:107340003B1050913C106091351070913610809137
:107350003710909138105F924F921AE9E12E19E997
:10736000F12E09E11EE30E9445870F9486830FB634
:10737000F894DEBF0FBECDBF2091A10E3091A20EBA
:107380004091A30E5091A40EF101662D772D8F2F01
:10739000922D0F942EB618163CF488EE93E00F94BD
:1073A000B1120E94BBF2E8CF60E086EA9FE00F9442
:1073B00069B380E090E0A0EAB0E480933D10909340
:1073C0003E10A0933F10B09340102091391030919F
:1073D0003A1040913B1050913C10609135107091E3
:1073E000361080913710909138100EEF402E0CE03F
:1073F000502E5F924F92812C912CE8E4AE2EE2E465
:10740000BE2EF1E4CF2EF0E1DF2EE12CF12C00EACC
:1074100010E40E944587EAEEFEE165917591859141
:107420009491609335107093361080933710909339
:107430003810EEEEFEE1259135914591549120935F
:10744000391030933A1040933B1050933C10E09029
:107450003D10F0903E1000913F10109140105F924F
:107460004F920E9445870F94868360E070E080E829
:107470009FEB0F948B420F900F900F900F908823EB
:1074800009F45BCE30913D1027963FAF279740918E
:107490003E102B964FAF2B9750913F102F965FAF1A
:1074A0002F976091401063966FAF63976F935F93D0
:1074B0004F933F9384E597E09F938F930F9487AD0D
:1074C0000F900F900F900F900F900F908EEA9FE00B
:1074D0009FAF8EAF44244A94542C13E2C12ED12C7A
:1074E000E12CF12C8201B6010D2C000C880B990BBC
:1074F0000F9482AE4B015C0197012F5F3F4F3BAF72
:107500002AAFDF92CF923F932F9348E157E05F93EA
:107510004F930F9487AD0F900F900F900F900F9097
:107520000F908FEF4816580611F40C94D06FBE01DF
:107530006F5F7F4F8EAD9FAD0E94ACFDA5019401A2
:10754000F101662D772D8F2F922D0F947CAE18169A
:10755000A4F495E0E916F10471F095E0C90ED11C90
:10756000AFEF4A1A5A0AEEADFFAD3296FFAFEEAF5B
:10757000EAACFBACB7CF05E010E0C8018752984FEA
:10758000DC01AA0FBB1FBFAFAEAF3801B3E06B0E7B
:10759000711C25E0209FC001219F900D11241BAE7E
:1075A0001AAEFC01BD966696FFAFEEAF6697AEEFE2
:1075B0004A2EACE05A2EC301029705970CF0B6C1D3
:1075C00066966EAD7FAD66978AAC9BAC680D791DF3
:1075D000072E000C880B990B0F9482AE26966CAF89
:1075E0007DAF8EAF9FAF26977F926F92FBE0AF2E5D
:1075F000F7E0BF2EBF92AF920F9487AD7092260F27
:107600006092250F20E030E040EF51E426966CAD0B
:107610007DAD8EAD9FAD26970F94E2B320E030E0B4
:1076200040E251E40F94E9A720E030E040EA50E462
:107630000F94D1B420E030E048E452E40F94E3B377
:107640000F9442B57093030D6093020D80E090E0BB
:10765000A0EAB0E480933D1090933E10A0933F10B9
:10766000B09340102091391030913A1040913B1066
:1076700050913C1060913510709136108091371008
:10768000909138105F924F92812C912CA8E4AA2EF1
:10769000A2E4BA2EB1E4CB2EB0E1DB2EE12CF12C2A
:1076A00000EA10E40E94458780E090E0A0EAB1E49F
:1076B0008093351090933610A0933710B093381004
:1076C000812C912CF0E7AF2EF2E4BF2E809239107E
:1076D00090923A10A0923B10B0923C10E0903D1076
:1076E000F0903E1000913F10109140105F924F9229
:1076F000812C912C28E4A22E22E4B22E20E030E04E
:1077000040E752E4BC01CD010E9445872AE939E9EE
:1077100049E15EE320933D1030933E1040933F10CB
:10772000509340102091391030913A1040913B1005
:1077300050913C1060913510709136108091371047
:10774000909138105F924F921AE9E12E19E9F12ECB
:1077500009E11EE30E9445870F9486830FB6F894D3
:10776000DEBF0FBECDBF2091A10E3091A20E409181
:10777000A30E5091A40E26966CAD7DAD8EAD9FAD3F
:1077800026970F942EB618163CF488EE93E00F94CB
:10779000B1120E94BBF2E7CF80E090E0A0EAB0E433
:1077A00080933D1090933E10A0933F10B0934010F3
:1077B0002091391030913A1040913B1050913C107B
:1077C000609135107091361080913710909138107B
:1077D0005F924F92812C912CB8E4AB2EB2E4BB2E79
:1077E00011E4C12E10E1D12EE12CF12C00EA10E4BD
:1077F0000E944587EAEEFEE165917591859194912D
:107800006093351070933610809337109093381032
:10781000EEEEFEE12591359145915491209339107A
:1078200030933A1040933B1050933C10E0903D1041
:10783000F0903E1000913F10109140105F924F92D7
:107840000E9445870F94868360E070E080E89FEB9C
:107850000F948B42AAADBBAD1596BBAFAAAFBFEFDD
:107860006B1A7B0A0F900F900F900F90811103C03D
:107870000F94C39C5BC027967FAD27972B966FAD67
:107880002B972F969FAD2F9763968FAD6397272FDA
:10789000362F492F582F60913D1070913E108091E6
:1078A0003F10909140100F94E2B3162F072FF82E3F
:1078B000E92E2091851030918610409187105091CB
:1078C0008810D801F7016B2F7A2F8F2F9E2F0F94DE
:1078D000E9A70F9442B57A836983EF92FF920F93E1
:1078E0001F938091A40E8F938091A30E8F9380910C
:1078F000A20E8F938091A10E8F93EFEDF6E0FF9390
:10790000EF930F9487ADBE016F5F7F4F8EAD9FAD3C
:107910000E94ACFD2EAD3FAD2E5F3F4F3FAF2EAF6F
:107920000FB6F894DEBF0FBECDBF45CE81E00F94F9
:10793000C39C0C94FD6A0FEF10E0A7EDCA2EA6E0E1
:10794000DA2E1093BC190093BB19F4E6EF2EF12C3C
:1079500084E690E00F94B11251E0E51AF108C1F706
:10796000809179138F93809178138F931F930F9346
:10797000DF92CF920F9487AD055011090F900F90B1
:107980000F900F900F900F90E1F60C94FD6A81E03C
:107990008093590E2091FF0C80910110909102105C
:1079A000222341F02091000D222321F05090010D5F
:1079B00051100FC0029749F081E0809397138BE735
:1079C00090E10F949F760C94FD6A1092590E0C94DE
:1079D000FD6A0297D1F38091400E9091410E289656
:1079E0009FAF8EAF2897A091250FB091260F2C96B0
:1079F000BFAFAEAF2C9781E090E09093410E8093A3
:107A0000400E83E190E09093260F8093250F81E054
:107A10000F94812F0F94E3600F94562A80E090E03A
:107A2000A0EAB0E480933D1090933E10A0933F10E5
:107A3000B09340102091391030913A1040913B1092
:107A400050913C1060913510709136108091371034
:107A500090913810EEEF6E2EECE07E2E7F926F92BA
:107A6000F5E58F2E982CA82CF1E4BF2EA1E4CA2EA8
:107A7000A0E1DA2EE12CF12C00EA10E40E94458707
:107A8000E0E1F3E5659175918591949160933510EE
:107A9000709336108093371090933810E4E1F3E53B
:107AA00025913591459154912093391030933A1096
:107AB00040933B1050933C10E0903D10F0903E10EE
:107AC00000913F10109140107F926F92812C912C69
:107AD000E8ECAE2EE2E4BE2E0E9445870F9486832A
:107AE0000F900F900F900F9005EC1FE0C8010F94BE
:107AF00064B3019639F00E5F1F4F053DEFE01E079E
:107B0000A9F75AAE80E00E94CFA560969FAF8EAFD6
:107B1000609780E1482E83E5582E612C712CC301BB
:107B200063E070E00F9495B824967FAF6EAF249712
:107B30001C0160FF06C002E0802E912C881A990A71
:107B400014019AAC9920A1F16114710489F1249671
:107B50008EAD9FAD2497880F991F2496AEACBFAC15
:107B600024978A0D9B1D820D931D880F991F8D539D
:107B7000904F0F9464B3BC01990F880B990B0F942D
:107B800082AE2AE037ED43E25CE30F94E9A720914F
:107B90008D1530918E1540918F15509190150F9441
:107BA000E3B322966CAF7DAF8EAF9FAF229706C036
:107BB00022961CAE1DAE1EAE1FAE229720E030E016
:107BC00040EA50E420933D1030933E1040933F1024
:107BD000509340102091391030913A1040913B1051
:107BE00050913C1060913510709136108091371093
:107BF00090913810AEEFBCE0BF93AF93812C912CE5
:107C0000B0EAAB2EB1E4BB2E11E4C12E10E1D12EAF
:107C1000E12CF12C00EA10E40E9445870F94868342
:107C2000F20185919591A591B4918093351090932F
:107C30003610A0933710B0933810F2013496859126
:107C40009591A591B4918093391090933A10A09397
:107C50003B10B0933C1069E370E185E390E10E9432
:107C60005FA8E0903D10F0903E1000913F10109101
:107C700040102091391030913A1040913B105091B2
:107C80003C106091351070913610809137109091B2
:107C90003810FEEF8F2EFCE09F2E9F928F92812C4A
:107CA000912CA6E1AA2EA3E4BA2E0E9445870F9438
:107CB00086830F900F900F900F90BAACBB2081F08D
:107CC0006114710469F020E030E040E85FE322963F
:107CD0006CAD7DAD8EAD9FAD22970F94E2B304C025
:107CE00060E070E080E291EC0F948B42882309F40D
:107CF0008BC0C0903D10D0903E10E0903F10F090AF
:107D00004010A701960160E070E080EA90E40F94D3
:107D1000E2B32DEC3CEC4CEC5DE30F947CAE87FDC4
:107D200073C02AAD2223A1F0A701960122966CAD63
:107D30007DAD8EAD9FAD22970F94E2B39F7720E08B
:107D400030E040E85FE30F942EB618160CF45CC0E8
:107D5000C090A10ED090A20EE090A30EF090A40EC1
:107D600080910F078823A9F00E9484A9882389F0B5
:107D7000C701B6010F949C082091851030918610A0
:107D800040918710509188100F94D1B49B01AC01A1
:107D900003C020E030E0A901A7E024968EAD9FAD9E
:107DA0002497A89F8001A99F100D1124020D131D77
:107DB000000F111F000F111F04571A4E60913D1044
:107DC00070913E1080913F10909140100F94E2B35B
:107DD000F80161837283838394838091250F90914E
:107DE000260F01979093260F8093250FFFEF6F1AB0
:107DF0007F0A81E00F94812F28E0420E511C39E068
:107E00006316710409F08BCE80E090E0A0EAB0E444
:107E100080933D1090933E10A0933F10B09340107C
:107E20002091391030913A1040913B1050913C1004
:107E30006091351070913610809137109091381004
:107E4000EEEFFCE0FF93EF93812C912C00EAA02E43
:107E500001E4B02EE1E4CE2EE0E1DE2EE12CF12CA7
:107E600000EA10E40E9445870F9486830F900F90DC
:107E700049E06416710409F47AC080910107909179
:107E800002078130910531F018F0029719F005C012
:107E900080E001C081E00E94D9BC212C312CB0EAE5
:107EA0004B2EB0E45B2E1EEF612E1CE0712E82E2A1
:107EB00093E10F9487078EE190E00F94609C0E94FD
:107EC00008A65091DB0F5AAF61E06093DB0F109270
:107ED000DA0F20923D1030923E1040923F105092A7
:107EE00040102091391030913A1040913B10509140
:107EF0003C10609135107091361080913710909140
:107F000038107F926F92812C912CE0EAAE2EE1E442
:107F1000BE2EF1E4CF2EF0E1DF2EE12CF12C00EAB1
:107F200010E40E9445870F9486838AAD8093DB0F0F
:107F30001092DA0F82E00F9473830F900F90A801D4
:107F400097010F942EB618160CF4B1CF1092410E73
:107F50001092400E81E00F94153740E061E081E01F
:107F60000F94A96E81E0809397130C94FD6A60963C
:107F70008EAD9FAD60970E94AEA50F94032A6091CD
:107F8000FC0C7091FD0C072E000C880B990B0F94C4
:107F900082AE9058209185103091861040918710C4
:107FA000509188100F94D1B40F94142A80EC9FE064
:107FB0000F9457B3082FDE0111961D0110E0809039
:107FC000870290908802A0908902B0908A028AAEBF
:107FD0009BAEACAEBDAE50EE852E55E1952E2AADD2
:107FE0003BAD4CAD5DAD29833A834B835C83D101BE
:107FF0008D911D010F947E9B882319F00F946A9B2D
:108000001BC0013009F026C1123028F4112341F0C1
:108010008EEB9FE00AC0123031F08CEB9FE005C080
:108020008FEB9FE002C08DEB9FE00F9457B3682F5A
:10803000880F770B880B990B6115710581059105E8
:1080400009F408C10F9482AE2FE632E143E85AE307
:108050000F94E9A76B017C019F7727E139ED4EEC86
:108060005DE30F942EB618160CF033C0E4E7FEE57E
:1080700084915F01882341F00E9462ADFFEFAF1A47
:10808000BF0AF5018491F6CFE7E5F0E184915F0145
:10809000882341F00E9462ADFFEFAF1ABF0AF501DD
:1080A0008491F6CF42E0C701B6010E9405AEEEE42E
:1080B000F0E184917F01882341F00E9462ADFFEFDF
:1080C000EF1AFF0AF7018491F6CF8AE00E9462ADB1
:1080D000C1C020E030E040E05FE3C701B6011230EC
:1080E00009F461C0133009F48AC0113071F10F94A2
:1080F000E9A72B013C014CE8A42E45E1B42EA301D5
:108100009201D50115966D917D918D919C91189755
:108110000F94E3B3F5016583768387839087A70186
:10812000960161817281838194810F94E3B3D501BB
:1081300011966D937D938D939C931497BCE1AB0E38
:10814000B11C8A149B04D9F685C00F94E9A72B01B2
:108150003C013CE8A32E35E1B32EA3019201F501C9
:1081600065817681878190850F94E3B3D50115965B
:108170006D937D938D939C931897A7019601199603
:108180006D917D918D919C911C970F94E3B3F501B6
:108190006187728783879487FCE1AF0EB11C8A14D4
:1081A0009B04D9F657C00F94E9A72B013C012DE899
:1081B000A22E25E1B22EA3019201D5015C966D910C
:1081C0007D918D919C915F970F94E3B3F501648F3E
:1081D000758F868F978FA70196016081718182814B
:1081E00093810F94E3B3D5016D937D938D939D930C
:1081F0005D01B9E9AB16B5E1BB06E9F62BC00F94FA
:10820000E9A72B013C0199EAA92E95E1B92EA3011A
:108210009201F50160817181828193810F94E3B3B2
:10822000D5016D937D938D939D935D01A70196017B
:1082300058966D917D918D919C915B970F94E3B3CE
:10824000F501608F718F828F938FF5EBAF16F5E19B
:10825000BF06E9F61F5F143009F0C1CE0F94FB6032
:1082600081E080938C150F94AF2AE091FE0C24E0FE
:10827000E29FF0011124E452F04F20E030E04FE2A1
:1082800053E460817181828193810F942EB6181618
:1082900084F480910F07882361F00E9484A98823C9
:1082A00041F08091020D9091030DC29714F00C944F
:1082B000536B81E090E090932302809322028FEB36
:1082C00094E10F94DC5128964EAD5FAD2897509302
:1082D000410E4093400E2C968EAD9FAD2C979093FF
:1082E000260F8093250F1092590E34C180918C1562
:1082F000882309F495C0E4E4F0E184918F01882398
:1083000039F00E9462AD0F5F1F4FF8018491F7CFE3
:1083100067E070E080E090E00E94EBADE2E4F0E125
:1083200084918F01882339F00E9462AD0F5F1F4F47
:10833000F8018491F7CF67E070E080E090E00E9460
:10834000EBADEFE2F0E184918F01882339F00E94D8
:1083500062AD0F5F1F4FF8018491F7CF65E070E0C9
:1083600080E090E00E94EBADEDE1F0E184918F01BF
:10837000882339F00E9462AD0F5F1F4FF80184918E
:10838000F7CF8AE00E9462AD00E010E0BAE16B2E08
:10839000B0E17B2E88E1A82E80E1B82EE12CF12CF3
:1083A0004801F8EA8F0E911CF3018491AAE1CA2ECC
:1083B000A0E1DA2E882341F00E9462ADFFEFCF1AD0
:1083C000DF0AF6018491F6CFF401EE0DFF1DE457AC
:1083D000FA4E618172818381948145E00E9405AEED
:1083E000F4E0EF0EF11C2CE1E216F104E9F6F501E0
:1083F0008491F8E1EF2EF0E1FF2E882341F00E94F6
:1084000062ADFFEFEF1AFF0AF7018491F6CF0C512E
:1084100011090C33FFEF1F0709F0C0CF0C94FD6A60
:10842000EAEFFFE084918F01882311F40C948A69AC
:108430000E9462AD0F5F1F4FF8018491F5CF86EE69
:108440000E948EA90C94FD6A1092FA0E0C94FD6A9B
:1084500085E40F947E9B811102C00F94868369EF9F
:10846000662E62E0762E75E3A72E70E1B72EE1ED61
:108470008E2EE0E19E2ED12CD3018D913D010F94E3
:108480007E9B8823C9F1B3E0DB120CC00F94759B6F
:10849000F501608371838283938381E490E10E947C
:1084A000C9BD2AC00F94759B9B01AC01D4016D918D
:1084B0007D918D919C910F94E3B3F501608371835D
:1084C00082839383E0903D10F0903E1000913F1026
:1084D000109140102091391030913A1040913B108A
:1084E00050913C106091351070913610809137108A
:1084F000909138100F94A859D394F4E0AF0EB11CAA
:1085000024E0820E911C34E0D312B6CF0C94FD6AA5
:1085100081E08093C80F0F94138860937A1670934C
:108520007B1680937C1690937D166091C80F84EC27
:108530009FE00F9469B369E277E081EC9FE00E94CD
:10854000ACFD1092420E60E08FEF9FE00F9469B394
:108550000C94FD6A82E00F94812F0C94FD6A809147
:1085600087159091881583569C4E9F938F9385EE27
:108570009FE00C94C2338DE40F947E9B882311F40A
:108580000C946D68E0912B0DF0912C0D319681913A
:108590008032E9F38930D9F380538A3060F08091DA
:1085A00087159091881583569C4E9F938F9380EDED
:1085B0009FE00C94C2330F94759B0F9442B5AB01AE
:1085C000BC01CA0150932D0F40932C0F4937510520
:1085D00011F40C94B4500CF0DCC04F32510509F486
:1085E000AAC60CF061C04931510509F451C33CF5EC
:1085F0004431510509F4BDC294F44131510509F4E7
:10860000AEC234F44230510508F4F6C10C945668F9
:108610004231510511F40C94A94D0C945668463121
:10862000510509F4EAC20CF4E4C24731510509F4DA
:10863000EAC24831510509F4FEC20C9456684E3125
:10864000510509F45BC48CF44B31510509F43BC36B
:108650000CF42BC34C31510509F424C44D315105A0
:1086600011F40C9468680C9456684A32510509F468
:108670000CC654F44F31510509F4ACC540325105D4
:1086800009F40DC50C9456684C32510509F444C6E2
:108690004D32510511F00C9456688AE50F947E9B7B
:1086A0000E94F96F0C9468684936510509F41BC79C
:1086B000A4F54435510511F40C94A94DDCF4413571
:1086C000510511F40C948B4D34F44934510509F4DF
:1086D00078C60C9456684235510511F40C94A54D9A
:1086E0004335510511F00C94566881E08093320FA8
:1086F0000C9468684635510511F40C940B4E14F433
:108700000C94F04D4C35510511F40C942A4E48361A
:10871000510509F4B3C60C9456684037510509F465
:10872000CCC69CF44B36510511F40C94854D14F4D1
:108730000C94554D4D36510509F4F4C74E3651058C
:1087400011F40C94AE4E0C9456684337510511F455
:108750000C94FE4E84F44137510511F40C94C14E33
:108760004237510511F00C945668E2E6FDE0849121
:108770008F010C94D74F4737510511F40C94B95021
:108780004837510511F00C945668109221020C9450
:1087900068688E3541E0940711F40C949C670CF0E6
:1087A0007FC0803D910511F40C942A54CCF58B3C8C
:1087B000910511F40C948752FCF48E3B910511F451
:1087C0000C942C4C34F48C38910509F47BC60C9431
:1087D0005668883C910511F40C94D651893C91055A
:1087E00011F00C94566849EFE42E42E0F42E09E7AC
:1087F00010E1D12C0C9442528D3C910511F40C9453
:10880000255314F40C94E0528E3C910511F40C9411
:10881000D4538F3C910511F40C94F3530C94566887
:10882000803F910511F40C946868CCF48C3D91055F
:1088300011F40C94A7543CF4813D910511F40C946F
:1088400052540C9456688D3D910511F40C94B85413
:10885000823E910511F40C94D9540C9456688E32D2
:1088600061E0960711F40C94C8566CF48C32B1E0B8
:108870009B0711F40C943C558D32914011F40C94EB
:1088800074550C9456688F32F1E09F0711F40C94E4
:10889000DD568033914011F40C9430560C94566898
:1088A0008A3532E0930711F40C9429630CF047C029
:1088B000853F51E0950711F40C94EB5AECF48039A4
:1088C000A1E09A0711F40C94A35A3CF48F3591401F
:1088D00011F40C9468680C9456688339F1E09F0792
:1088E00011F40C94A75A843F914011F00C945668EF
:1088F0000E9485B00C9468688D3F31E0930711F4B5
:108900000C94AB5D6CF4863F51E0950711F40C9428
:10891000EF5A873F914011F40C94F35A0C94566827
:108920008835A2E09A0711F40C94865E893592404E
:1089300011F00C9456680F94228B0C9468688D3556
:10894000E3E09E0711F40C94FD63DCF48E3B22E01F
:10895000920711F40C9445683CF48D3B924011F45D
:108960000C9439680C945668833553E0950711F4DC
:108970000C94C75D8C35934011F40C942C630C94CB
:1089800056688C38A3E09A0711F40C94686894F444
:108990008438E3E09E0711F40C9419668B389340F9
:1089A00011F00C94566809EFA02E02E0B02E00E002
:1089B0000C947C67803A23E0920709F4DCC3873E7D
:1089C000934011F00C94566810925E0F1092F50FC0
:1089D0008091030F9091040FA091050FB091060FA5
:1089E00080932D0D90932E0DA0932F0DB093300DED
:1089F0000F94D3120C946868E0912B0DF0912C0D1C
:108A00008F010E5F1F4F80E50F947E9B882371F0CE
:108A10000F94759B0F9448B56B017C01AA24A39415
:108A2000672B682B692B31F4A12C04C0A12CC12C1D
:108A3000D12C760183E50F947E9B882391F00F94CF
:108A4000759B20E030E04AE754E40F94E9A70F94C7
:108A500048B56B017C01BB24B394672B682B692B51
:108A600009F4B12C6AE270E0C8010F9427B90097AD
:108A700011F0DC011C92F801CF0121912032E1F3C9
:108A8000A11007C0B11005C0222319F00F944E5356
:108A900004C081E193E10F94DC5181E08093470EA3
:108AA0001092460E0F9486830F9413886093FF0EE6
:108AB0007093000F8093010F9093020FC114D104A3
:108AC000E104F10419F10F941388C60ED71EE81EB5
:108AD000F91E84E090E090932302809322020F9489
:108AE00013886C157D058E059F0510F00C94956B11
:108AF0000F94593081110C94956B0F94AA7D81E0ED
:108B00000F945C0E80E00F94812FE9CF84E090E019
:108B100090932302809322020F945930811109C04F
:108B20000F94AA7D81E00F945C0E80E00F94812F5A
:108B3000F3CF82E090E09093230280932202809111
:108B40008016882331F085EB9DE20F94DC510C9464
:108B500068688FEB94E10F94DC510C94686888E0AE
:108B600093E10F94DC5117981698159814980C946B
:108B70006868E7ECF6E084918F01882339F00E9461
:108B800062AD0F5F1F4FF8018491F7CF8AE00E941A
:108B900062AD109261191092601984ED96E10E9405
:108BA00098E08BE1E4EDF6E1DE01119601900D9283
:108BB0008A95E1F740E050E0BE016F5F7F4F88E0AB
:108BC00094E00F94667BCE0101960E94B1A7E9EB79
:108BD000F6E084918F01882339F00E9462AD0F5F27
:108BE0001F4FF8018491F7CF8AE00E9462AD0C9488
:108BF00068680F94A9480C946868109280161092C7
:108C000081160C94686880912B0D90912C0D6AE26E
:108C100070E004960F9427B9009711F0DC011C92C4
:108C200080912B0D90912C0D41E061E004960F9402
:108C3000D3430C94686880918216811114C060E05F
:108C400086E69FE00F9469B360E088E69FE00F94AA
:108C500069B360E085E69FE00F9469B360E084E665
:108C60009FE00F9469B380918116882329F081E0F9
:108C700080938016109282160F9413886093500E82
:108C80007093510E8093520E9093530E0C9468681B
:108C900080918016882311F40C94686810928016D5
:108CA00081E0809382160C946868809181168823F5
:108CB00011F40C94686883E50F947E9B81110C94E9
:108CC000A16B0C94686880918016882309F4B8C061
:108CD0000CE916E1F80181918F01882319F00E94B7
:108CE00062ADF8CFEFEDFDE084918F01882339F07C
:108CF0000E9462AD0F5F1F4FF8018491F7CFE1EC46
:108D0000F5E084918F01882339F00E9462AD0F5FF6
:108D10001F4FF8018491F7CF60915B1970915C1936
:108D200080915D1990915E194AE00E947AADEDED57
:108D3000FDE084918F01882339F00E9462AD0F5FBE
:108D40001F4FF8018491F7CF609153197091541916
:108D500080915519909156194AE00E947AAD8AE0A7
:108D60000E9462AD0F94138840E6C42E4AEED42EC2
:108D7000E12CF12CA70196010F94A7B349015A01E8
:108D80006091500E7091510E8091520E9091530E41
:108D9000A70196010F94A7B38401021B130BC8010E
:108DA0006CE370E00F9481B8CB019927EAE0F0E022
:108DB000BF010F9495B8282FCB01BF010F9495B830
:108DC000805D8093B319205D2093B4191092B5197A
:108DD00053EBE52E59E1F52E6701D6018D916D011A
:108DE000882319F00E9462ADF8CF8AE30E9462AD39
:108DF000C8016CE370E00F9481B86AE070E00F94F2
:108E000095B8605D6093B319805D8093B41910923A
:108E1000B519F70181917F01882319F00E9462AD95
:108E2000F8CFEBEDFDE084918F01882311F40C94D1
:108E300068680E9462AD0F5F1F4FF8018491F5CF03
:108E400080918216882371F0EBECFDE084918F0114
:108E5000882309F4C9CE0E9462AD0F5F1F4FF8014D
:108E60008491F6CF80913F0E882371F0EFEBFDE007
:108E700084918F01882309F4B7CE0E9462AD0F5F01
:108E80001F4FF8018491F6CFEFEAFDE084918F0146
:108E9000882309F4A9CE0E9462AD0F5F1F4FF8012D
:108EA0008491F6CF80912B0D90912C0D6AE270E0A9
:108EB00004960F9427B98C01892BA9F0809187150E
:108EC000909188156EE470E083569C4E0F9427B9FC
:108ED00060E270E00F9427B9019690932C0D809377
:108EE0002B0DD8011C9280912B0D90912C0D41E0FF
:108EF00060E004960F94D3430C94686880918116C7
:108F0000882311F40C9468680F94255780912B0DD9
:108F100090912C0D6AE270E004960F9427B98C01B1
:108F2000892BA9F080918715909188156EE470E0E7
:108F300083569C4E0F9427B960E270E00F9427B9D6
:108F4000019690932C0D80932B0DF8011082C09008
:108F50002B0DD0902C0D86010C5F1F4F8091811638
:108F6000882311F40C94686886EA98E10E94BEE3B5
:108F7000109280161F8E1AA284ED96E19093F0163F
:108F80008093EF160115110591F0D60114968C917E
:108F90008F3239F4BE01615E7F4FC8010F941959B9
:108FA00006C081EF96E19093F0168093EF166091E2
:108FB000EF167091F01619821C8222E0A801CE01F2
:108FC00001960E9485E58823A1F0CE0101960F94B9
:108FD000D47A882371F061E0CE0101960E943FE3CC
:108FE000009739F025EEFC0120831C820E94C3DD2E
:108FF000F82ECE0101960E94B1A7FF2021F1E1EAEF
:10900000FDE084917F01882341F00E9462ADFFEF73
:10901000EF1AFF0AF7018491F6CFD8018D918D01E7
:10902000882319F00E9462ADF8CF8AE00E9462ADF9
:1090300010925B1910925C1910925D1910925E19D2
:109040000F94964626C0E9E8FDE084917F018823CD
:1090500041F00E9462ADBFEFEB1AFB0AF701849169
:10906000F6CFD8018D918D01882319F00E9462AD51
:10907000F8CFE7E8FDE084918F01882339F00E9462
:1090800062AD0F5F1F4FF8018491F7CF8AE00E9415
:1090900062ADCE014F960E94B1A70C946868809192
:1090A000801681110F94868300912B0D10912C0D49
:1090B0000C5F1F4F6AE270E0C8010F9427B97C0172
:1090C00061E270E0C8010F9427B9009719F08C0194
:1090D0000F5F1F4FE114F10411F0D7011C9280E5DE
:1090E0000F947E9BF82E80912B0D90912C0D0817DC
:1090F000190708F4F12C80918116882311F40C943F
:10910000686841E04F2561E0C8010F94D34383E5CF
:109110000F947E9B8823B9F080912B0D90912C0D9C
:109120008017910780F40F946A9BAB01BC014093B8
:109130005B1950935C1960935D1970935E1986EA10
:1091400098E10E9402E080918116882329F081E055
:109150008093801610928216F1100C9468680F9418
:1091600013886093500E7093510E8093520E90931B
:10917000530E0C94686880912B0D90912C0D6AE22F
:1091800070E005960F9427B98C01892BA9F0809186
:109190008715909188156EE470E083569C4E0F946D
:1091A00027B960E270E00F9427B9019690932C0DD7
:1091B00080932B0DF801108280912B0D90912C0D36
:1091C00021E020937F1641E060E005960F94D343A1
:1091D0000C9468680F9413880091500E1091510EF2
:1091E0002091520E3091530E6B017C01C01AD10AAE
:1091F000E20AF30AC701B60128EE33E040E050E08E
:109200000F94A7B3CA01B9012CE330E040E050E06D
:109210000F94A7B37F936F93C701B60120E63AEE90
:1092200040E050E00F94A7B33F932F9381EC9FE071
:109230009F938F938E010F5F1F4F1F930F930F9478
:10924000E0ADE6E9FEE584910FB6F894DEBF0FBE0F
:10925000CDBF7F01882341F00E9462AD3FEFE31A4A
:10926000F30AF7018491F6CF7801D7018D917D0142
:10927000882319F00E9462ADF8CF8AE00E9462ADA7
:10928000C8010F944E530C94686883E50F947E9B3D
:10929000882311F40C9468680F94759B0F9442B561
:1092A000F62EE72E862F9E2D8C0180E50F947E9B57
:1092B000882331F00F3F110509F010F40C94B26BC4
:1092C0000DE010E0EBE8F2E08191919180179107B9
:1092D00011F40C946868B2E0E33CFB07A9F7063090
:1092E000110539F48F2D9E2D9093BC198093BB19D5
:1092F00004C017FF02C00C94686861E0802F0F94CF
:10930000F8856F2D802F0F94CA856F2D7E2D802FAD
:109310000F9434860C9468688FEF0E948EA960E0E9
:1093200070E088EF9FE00F9483B30F94072D0F94A4
:10933000E92C0C94686884E090E090932302809379
:1093400022020F940B370F94AA7D81E00F945C0EDC
:1093500060E080E00F945C3288E79DE00F948331F9
:1093600061E080E00F945C321E9903C082E79DE0CB
:1093700002C085E79DE00F94833162E080E00F94A6
:109380005C321D9903C08CE69DE002C08FE69DE033
:109390000F94833163E080E00F945C321C9903C02A
:1093A00086E69DE002C089E69DE00F9483310F942C
:1093B0005930882341F20F940B370F94268A0C946E
:1093C000686880E50F947E9B882331F00F94759B2D
:1093D0000F9448B560933A0282E50F947E9B8823F0
:1093E00041F00F94759B0F9448B570933E026093C3
:1093F0003D0281E50F947E9B882331F00F94759B8D
:109400000F9448B56093390283E50F947E9B8823BF
:1094100041F00F94759B0F9448B570933C02609394
:109420003B0280913E028F9380913D028F93809109
:109430003A021F928F9385E796E09F938F930CE7F4
:1094400016E01F930F930F9487AD80913C028F938A
:1094500080913B028F93809139021F928F938EE609
:1094600096E09F938F931F930F930F9487AD0FB642
:10947000F894DEBF0FBECDBF0C946868BE016F5F6D
:109480007F4F88E690E00F9424A381110C946868C4
:1094900083E50F947E9B882311F40C9468681981EE
:1094A0000F94759B11110C9468680F9442B57093DA
:1094B0008A15609389150C94686863E08DE696E0E0
:1094C0000F94FE0D83E50F947E9B882311F40C947A
:1094D00068680F94759B0F9442B57093030D609369
:1094E000020D0C946868BE016F5F7F4F89E690E0C3
:1094F0000F9424A381110C946868EBEBFFE0849136
:109500008F01882339F00E9462AD0F5F1F4FF80171
:109510008491F7CFE98124E0E29FF0011124E45225
:10952000F04F608171818281938141E00E9405AE9C
:10953000E8EBFFE084918F01882339F00E9462AD4F
:109540000F5F1F4FF8018491F7CFE981F0E0EE0F34
:10955000FF1FE757FA4E60817181072E000C880BC0
:10956000990B0F9482AE41E00E9405AEE4EBFFE060
:1095700084918F01882339F00E9462AD0F5F1F4FE5
:10958000F8018491F7CF60910807709109078091E5
:109590000A0790910B0741E00E9405AEE1EBFFE066
:1095A00084918F01882339F00E9462AD0F5F1F4FB5
:1095B000F8018491F7CF6091020D7091030D072E91
:1095C000000C880B990B0F9482AE41E00E9405AE0F
:1095D000EEEAFFE084918F01882339F00E9462ADAA
:1095E0000F5F1F4FF8018491F7CF60E070E0CB016F
:1095F0000E94EBADECEAFFE084918F01882339F003
:109600000E9462AD0F5F1F4FF8018491F7CF609108
:10961000DC0F7091DD0F8091DE0F9091DF0F41E044
:109620000E9405AEE9EAFFE084918F01882339F0BA
:109630000E9462AD0F5F1F4FF8018491F7CF6091D8
:10964000891570918A15072E000C880B990B0F94C1
:1096500082AE41E00E9405AEE5EAFFE084918F0111
:10966000882339F00E9462AD0F5F1F4FF80184918B
:10967000F7CFE981F0E0E45AF04F608170E080E0DC
:1096800090E00E94EBADE0EAFFE084918F01882337
:1096900039F00E9462AD0F5F1F4FF8018491F7CF40
:1096A00060915B0F70E080E090E00E94EBADECE930
:1096B000FFE084918F01882339F00E9462AD0F5F33
:1096C0001F4FF8018491F7CF6091A10E7091A20E07
:1096D0008091A30E9091A40E41E00E9405AEE8E9AE
:1096E000FFE084918F01882339F00E9462AD0F5F03
:1096F0001F4FF8018491F7CF60919D0E70919E0EDF
:1097000080919F0E9091A00E41E00E9405AE8AE0EC
:109710000E9462AD81E090E0909323028093220248
:109720000C94DF6FBE016F5F7F4F8DE690E00F946A
:1097300024A381110C9468688DE69DE20F94DC519E
:1097400081E090E09093340E8093330E8091C80FA7
:10975000882329F060E081E090E00F94B20283E575
:109760000F947E9B882379F019810F94759B1111BA
:1097700006C00F9442B570938A156093891581E0F5
:109780008093040212C082E50F947E9B882369F0C7
:1097900019810F94759B111106C00F9442B57093F7
:1097A0008A1560938915109204020F9413884B0157
:1097B0005C01F9800F2D10E0F801EE0FFF1FE75755
:1097C000FA4E60817181072E000C880B990B0F9463
:1097D00082AEF801EE0FFF1FEE0FFF1FE452F04FB5
:1097E00011E020813181428153810F942EB61816E9
:1097F0000CF010E01093070F81E090E090932302AB
:109800008093220210925A0E4F2DC501B4010F947D
:109810005F118FE59DE20F94DC5182E090E0909320
:109820002302809322029093340E8093330E809112
:10983000C80F882329F060E082E090E00F94B20224
:109840000F9413886093FF0E7093000F8093010FA5
:109850009093020F0C94686883E59DE20F94DC51AD
:1098600083E090E09093340E8093330E8091C80F84
:10987000882329F060E081E090E00F94B20283E554
:109880000F947E9B882361F00F94759B0F9442B5D3
:109890007093030D6093020D81E0809304020FC06A
:1098A00082E50F947E9B882351F00F94759B0F9453
:1098B00042B57093030D6093020D109204020F9451
:1098C00013884B015C0110925A0E6091020D709149
:1098D000030D072E000C880B990B0F9482AE11E03C
:1098E000209108073091090740910A0750910B0712
:1098F0000F942EB618160CF010E01093070F81E0AD
:1099000090E0909323028093220205E91FE0B1E9E1
:10991000EB2EBFE0FB2E8DE8C82E8FE0D82E809175
:10992000070F6091020D7091030D8823B9F08091AB
:109930005A0E811113C0072E000C880B990B0F943F
:1099400082AE209108073091090740910A07509193
:109950000B070F942EB61816BCF08BC0072E000C08
:10996000880B990B0F9482AE20910807309109075C
:1099700040910A0750910B070F947CAE87FF79C086
:1099800080910402811175C00F941388DC01CB0112
:1099900088199909AA09BB09893E9340A105B10517
:1099A00008F45EC08091C80F811156C0E091FE0C92
:1099B00024E0E29FF0011124E452F04F40805180F6
:1099C00062807380F8018491A5E9AA2EAFE0BA2ED7
:1099D000882341F00E9462ADFFEFAF1ABF0AF50184
:1099E0008491F6CF42E0C301B2010E9405AEF701B7
:1099F0008491F1E9AF2EFFE0BF2E882341F00E9451
:109A000062ADFFEFAF1ABF0AF5018491F6CF609106
:109A1000FE0C70E080E090E00E94EBADF6018491D6
:109A2000EDE8AE2EEFE0BE2E882341F00E9462AD3D
:109A3000FFEFAF1ABF0AF5018491F6CF60910807D6
:109A40007091090780910A0790910B0741E00E94ED
:109A500005AE8AE00E9462AD0F9413884B015C0151
:109A60000F94AA7D80E00F945C0E80E00F94812F0C
:109A700056CF8AE49DE20F94DC5182E090E090930F
:109A800023028093220284E090E09093340E80932E
:109A9000330E0F9413886093FF0E7093000F809322
:109AA000010F9093020F0C94686883E50F947E9BDE
:109AB000882319F10F94759B20E030E0A9010F94E1
:109AC0007CAE87FD0FC00F94759B20E030E04FE720
:109AD00053E40F942EB6181644F00F94759B0F9410
:109AE00042B505C060E070E002C06FEF70E07093B7
:109AF000BC196093BB190C9468688FEF90E0909349
:109B0000BC198093BB190C9468681092BC19109210
:109B1000BB190C9468680F94943A0F948683149A36
:109B20000F94DF831092BC191092BB1968EE73E09A
:109B300080E090E00F94FB8689E094E00F94DC5184
:109B400080E00F94812F0C9468681092320F0C946F
:109B5000686883E50F947E9B882399F00F94759B2A
:109B600020E030E04AE754E40F94E9A70F9448B5A9
:109B700060937602709377028093780290937902D3
:109B80001DC088E50F947E9B81110C94B96B89E50B
:109B90000F947E9B81110C94B96B8AE50F947E9B88
:109BA00081110C94B96B85E40F947E9B81110C9408
:109BB000B96B0F948683149A0F94DF838FEF9FEF16
:109BC00090933E0280933D0290933C0280933B022F
:109BD00080933A02809339021092330F0C94686894
:109BE00083E50F947E9B882311F40C9468680F948E
:109BF000759B20E030E04AE754E40F94E9A70F9406
:109C000048B56093FB0E7093FC0E8093FD0E90930D
:109C1000FE0E0C94686883E50F947E9B882311F4F4
:109C20000C9468680F94759B20E030E04AE754E498
:109C30000F94E9A70F9448B5609372027093730272
:109C4000809374029093750289E696E10E9432DD5A
:109C50000C94686829EF32E03BAF2AAF09E710E1C6
:109C60007FE5C72E7DE0D72EF12CAAADBBAD8D913F
:109C7000BBAFAAAF0F947E9B882309F463C0B3E007
:109C8000FB1259C00F94759B2B013C0120E030E082
:109C900040EA51E40F947CAE87FF45C0A3019201D6
:109CA000F80164817581868197810F94D1B44B014D
:109CB0005C019B01AC016091CD107091CE10809140
:109CC000CF109091D0100F94E9A76093CD107093AE
:109CD000CE108093CF109093D01020902B02309014
:109CE0002C02A5019401D1011C966D917D918D915D
:109CF0009C911F970F94E9A7F10164877587868768
:109D00009787D6016D917D918D919C910F9480AE36
:109D1000A50194010F94E9A70F9448B5F60160835B
:109D2000718382839383D80114964D925D926D92D4
:109D30007C92179707C00F94759BF8016483758315
:109D400086839783F3940C5F1F4FF4E0CF0ED11CF2
:109D500064E0862EF81089CF0C9468688EE40F9426
:109D60007E9B882311F40C9468680F946A9B60931F
:109D70002D0D70932E0D80932F0D9093300D0C941C
:109D8000686883E50F947E9B882379F080912B0D82
:109D900090912C0D4AE050E060E070E001960F9445
:109DA00011AA60934F020C946868E6E9FEE584917D
:109DB0008F01882339F00E9462AD0F5F1F4FF801B9
:109DC0008491F7CFC0904F02D12CE12CF12CE6E822
:109DD000FFE084918F01882339F00E9462AD0F5F0C
:109DE0001F4FF8018491F7CF4AE0C701B6010E94E6
:109DF0007AAD8AE00E9462AD0C94686886E50F94A3
:109E00007E9B882379F0E3ECFBE584918F01882326
:109E100011F40C94F4450E9462AD0F5F1F4FF801DE
:109E20008491F5CF85E50F947E9B382E8823D9F158
:109E3000E0902B0DF0902C0DFFEFEF1AFF0AF0923F
:109E40002C0DE0922B0D270167014601D6018D9163
:109E50006D0190ED980F9A30C0F38E3211F00C9492
:109E600068685D013501F50181915F0190ED980F02
:109E70009A30C0F38E3211F00C946868CF018C01D7
:109E8000DC012C90019620ED220D2A30C0F3822DAA
:109E90000F94B25181110C94D86BBDE22B120C942B
:109EA00068680C94D86BE8E6FFE084918F01882302
:109EB00039F00E9462AD0F5F1F4FF8018491F7CF18
:109EC000E3ECFBE584918F01882339F00E9462ADB9
:109ED0000F5F1F4FF8018491F7CFEEE0FFE0849110
:109EE0008F01882339F00E9462AD0F5F1F4FF80188
:109EF0008491F7CFEAE0FFE084918F01882339F065
:109F00000E9462AD0F5F1F4FF8018491F7CFEBEF16
:109F1000FEE084918F01882339F00E9462AD0F5FCB
:109F20001F4FF8018491F7CFEEEEFEE084918F0190
:109F3000882339F00E9462AD0F5F1F4FF8018491B2
:109F4000F7CFEDEDFEE084918F01882339F00E9478
:109F500062AD0F5F1F4FF8018491F7CFEBEDFEE08C
:109F600084918F01882339F00E9462AD0F5F1F4FEB
:109F7000F8018491F7CFE4EDFEE084918F0188230E
:109F800039F00E9462AD0F5F1F4FF8018491F7CF47
:109F9000EFEAFEE084918F01882311F40C94F445DC
:109FA0000E9462AD0F5F1F4FF8018491F5CF8823A7
:109FB00039F00E9462AD0F5F1F4FF8018491F7CF17
:109FC0006091351070913610809137109091381053
:109FD00042E00E9405AEEEE5FDE084918F0188230A
:109FE00039F00E9462AD0F5F1F4FF8018491F7CFE7
:109FF0006091391070913A1080913B1090913C1013
:10A0000042E00E9405AEEAE5FDE084918F018823DD
:10A0100039F00E9462AD0F5F1F4FF8018491F7CFB6
:10A0200060913D1070913E1080913F1090914010D2
:10A0300042E00E9405AEE6E5FDE084918F018823B1
:10A0400039F00E9462AD0F5F1F4FF8018491F7CF86
:10A050006091411070914210809143109091441092
:10A0600042E00E9405AEE6EBF5E084918F01882383
:10A0700039F00E9462AD0F5F1F4FF8018491F7CF56
:10A0800080E00F9465830F9482AE20917D10309113
:10A090007E1040917F10509180100F94D1B442E017
:10A0A0000E9405AEE2E5FDE084918F01882339F03E
:10A0B0000E9462AD0F5F1F4FF8018491F7CF81E0DE
:10A0C0000F9465830F9482AE20918110309182109D
:10A0D00040918310509184100F94D1B442E00E94BB
:10A0E00005AEEEE4FDE084918F01882339F00E94F3
:10A0F00062AD0F5F1F4FF8018491F7CF82E00F949C
:10A1000065830F9482AE2091851030918610409126
:10A110008710509188100F94D1B442E00E9405AE90
:10A12000EAE4FDE084918F01882339F00E9462AD5A
:10A130000F5F1F4FF8018491F7CF83E00F94658381
:10A140000F9482AE2091891030918A1040918B102B
:10A1500050918C100F94D1B442E00E9405AE8AE079
:10A160000E9462AD0C94686881E0809321020C9497
:10A170006868E4E5F6E084918F01882339F00E9455
:10A1800062AD0F5F1F4FF8018491F7CF8AE00E9404
:10A1900062ADECE4F6E084918F01882339F00E94EF
:10A1A00062AD0F5F1F4FF8018491F7CF1E9B0DC06A
:10A1B000EEEFF2E184918F018823A1F00E9462AD5D
:10A1C0000F5F1F4FF8018491F7CFE9EFF2E184911F
:10A1D0008F01882339F00E9462AD0F5F1F4FF80195
:10A1E0008491F7CF8AE00E9462ADE4E4F6E08491C6
:10A1F0008F01882339F00E9462AD0F5F1F4FF80175
:10A200008491F7CF8091060182FF0DC0EEEFF2E15D
:10A2100084918F018823A1F00E9462AD0F5F1F4FD0
:10A22000F8018491F7CFE9EFF2E184918F0188235F
:10A2300039F00E9462AD0F5F1F4FF8018491F7CF94
:10A240008AE00E9462ADECE3F6E084918F018823FE
:10A2500039F00E9462AD0F5F1F4FF8018491F7CF74
:10A260001D9B0DC0EEEFF2E184918F018823A1F0D8
:10A270000E9462AD0F5F1F4FF8018491F7CFE9EFA5
:10A28000F2E184918F01882339F00E9462AD0F5F63
:10A290001F4FF8018491F7CF8AE00E9462ADE4E39A
:10A2A000F6E084918F01882339F00E9462AD0F5F40
:10A2B0001F4FF8018491F7CF8091060187FF0DC0F1
:10A2C000EEEFF2E184918F018823A1F00E9462AD4C
:10A2D0000F5F1F4FF8018491F7CFE9EFF2E184910E
:10A2E0008F01882339F00E9462AD0F5F1F4FF80184
:10A2F0008491F7CF8AE00E9462ADECE2F6E08491AF
:10A300008F01882339F00E9462AD0F5F1F4FF80163
:10A310008491F7CF1C9B0DC0EEEFF2E184918F0189
:10A320008823A1F00E9462AD0F5F1F4FF801849156
:10A33000F7CFE9EFF2E184918F01882339F00E9491
:10A3400062AD0F5F1F4FF8018491F7CF8AE00E9442
:10A3500062ADE4E2F6E084918F01882339F00E9437
:10A3600062AD0F5F1F4FF8018491F7CF01990FC0C5
:10A37000EEEFF2E184918F01882311F40C94F445FF
:10A380000E9462AD0F5F1F4FF8018491F5CFE9EF96
:10A39000F2E184918F01882311F40C94F4450E941A
:10A3A00062AD0F5F1F4FF8018491F5CF1091FE0C45
:10A3B00084E50F947E9B882301F10F94759B0F9485
:10A3C00048B5162F6623C9F0E6E9FEE584918F01B2
:10A3D000882339F00E9462AD0F5F1F4FF80184910E
:10A3E000F7CF02EE12E1D8018D918D01882311F48F
:10A3F0000C9468680E9462ADF6CF84E40F947E9B53
:10A40000882311F40C9468680F94759B20E030E069
:10A41000A9010F947CAE811103C0109210112EC0BF
:10A420000F94759BB4E01B9FF0011124EF5EFE4E6C
:10A430006083718382839383C0901111D090121135
:10A44000E0901311F090141120E030E0A901C70151
:10A45000B6010F947CAE811106C0C12CD12C50EEF8
:10A46000E52E5FE3F52EC0921111D0921211E09209
:10A470001311F092141181E0809310110F94CE0CFF
:10A480000C946868F70181917F010F947E9B88236B
:10A49000A1F10F94759B0F9448B5F1E0FD15ACF058
:10A4A000653C29E0720781059105A0F4562F472FDE
:10A4B000382F292F613CA3E07A078105910590F0A0
:10A4C00050EC43E030E020E00DC0562F472F382FEE
:10A4D000292F08C050EC43E030E020E064EC79E044
:10A4E00080E090E0F80164A375A386A397A3E455E8
:10A4F000FF4F5083418332832383D3940C5F1F4FDC
:10A50000F4E0DF12BFCF0E946BBD0C94686829EFA6
:10A51000A22E22E0B22E39E7C32E30E1D32E912CA9
:10A52000D5018D915D010F947E9B882309F43EC077
:10A530000F94759B7B018C01B1E0B91514F120E0FB
:10A5400030E048E453E40F942EB618163CF4512C36
:10A55000612C88E4782E93E4892E04C05E2C6F2C45
:10A56000702E812E20E030E048EC52E4B701C801A3
:10A570000F942EB618164CF4E12CF12C08EC12E4D2
:10A5800004C0562E6F2C782E812E852D962DA72D4A
:10A59000B82DF601848B958BA68BB78BC701D8019C
:10A5A000E456FF4F80839183A283B3839394F4E0B6
:10A5B000CF0ED11C14E0812E9810B2CF0C94686895
:10A5C00083E50F947E9B8823E9F00F94759B60933D
:10A5D000AD107093AE108093AF109093B01084E5DF
:10A5E0000F947E9B882311F40C9468680F94759BDC
:10A5F0006093B1107093B2108093B3109093B41025
:10A600000C94686880E50F947E9B882351F00F942A
:10A61000759B6093AD107093AE108093AF109093C4
:10A62000B01082E50F947E9B882351F00F94759BA8
:10A630006093B1107093B2108093B3109093B410E4
:10A6400084E50F947E9B0C94686883E50F947E9B51
:10A65000882351F00F94759B6093B5107093B610DA
:10A660008093B7109093B81084E50F947E9B882355
:10A6700051F00F94759B6093B9107093BA1080934A
:10A68000BB109093BC1082E40F947E9B882361F0F2
:10A690000F94759B0F9448B56093BD107093BE10D6
:10A6A0008093BF109093C01088E50F947E9B882301
:10A6B00091F00F94759B6093C5107093C6108093B2
:10A6C000C7109093C8106093C1107093C21080930C
:10A6D000C3109093C41089E50F947E9B882351F09A
:10A6E0000F94759B6093C5107093C6108093C7102C
:10A6F0009093C8108AE50F947E9B882351F00F94A5
:10A70000759B6093C9107093CA108093CB1090937F
:10A71000CC1085E40F947E9B882351F00F94759B99
:10A720006093CD107093CE108093CF109093D01083
:10A7300020E030E040E251E46091C1107091C2101D
:10A740008091C3109091C4100F942EB6181664F423
:10A7500080E090E0A0E2B1E48093C1109093C21039
:10A76000A093C310B093C41020E030E040E251E465
:10A770006091C5107091C6108091C7109091C8105B
:10A780000F942EB6181614F00C94686880E090E0D0
:10A79000A0E2B1E48093C5109093C610A093C710B7
:10A7A000B093C8100C946868A9EFEA2EA2E0FA2EC4
:10A7B00001ED10E1BDEDCB2EB0E1DB2ED7018D9187
:10A7C0007D010F947E9B882339F00F94759BF801CF
:10A7D00060837183828393830C5F1F4FC016D10601
:10A7E00069F70C94686883E50F947E9B882351F089
:10A7F0000F94759B6093FC107093FD108093FE1076
:10A800009093FF1086E40F947E9B882381F00F9431
:10A81000759B20E030E040E752E40F94D1B46093A0
:10A8200000117093011180930211909303118AE536
:10A830000F947E9B882311F40C9468680F94759B89
:10A840006093041170930511809306119093071182
:10A850000C94686883E50F947E9B882351F00F94D5
:10A86000759B609308117093091180930A1190935E
:10A870000B1186E40F947E9B882311F40C94686876
:10A880000F94759B20E030E040E752E40F94D1B480
:10A8900060930C1170930D1180930E1190930F1112
:10A8A0000C94686883E50F947E9B882311F40C94C4
:10A8B00068680F94759B0F9442B56115710551F04E
:10A8C0006130710569F481E08093FB101092D90F1B
:10A8D0000C9468681092FB101092D90F0C94686861
:10A8E000E6E9FEE584918F01882339F00E9462AD8C
:10A8F0000F5F1F4FF8018491F7CFE1E1F6E08491FB
:10A900008F01882339F00E9462AD0F5F1F4FF8015D
:10A910008491F7CF009187151091881503561C4E2E
:10A92000D8018D918D01882319F00E9462ADF8CF76
:10A93000EAEAFEE084918F01882311F40C94F44537
:10A940000E9462AD0F5F1F4FF8018491F5CF83E540
:10A950000F947E9B882311F40C9468680F94759B68
:10A960000F9442B570934402609343020C9468685C
:10A9700083E50F947E9B882309F480CD0F94759B0B
:10A980000F9442B56B017C0184E50F947E9B882374
:10A9900059F0BE016F5F7F4F8DED90E00F9424A3BF
:10A9A00081110C9468686ACDD0928302C0928202B1
:10A9B00065CD80E50F947E9B882311F40C94686824
:10A9C0000F94759B0F9442B5D62E862F972F7C013E
:10A9D00083E50F947E9B882331F00F94759B0F9431
:10A9E00042B58B0102C00FEF1FEFC801019603971C
:10A9F00010F00C946868EBE8F2E083EC92E02191AF
:10AA00003191E216F30611F40C9468688E179F07D3
:10AA1000B1F7F7FE02C00C9468680F948683FD2C92
:10AA200060E08D2D0F94F8850F3FFFEF1F0731F089
:10AA30000130110571F401E010E00DC08D2D0F946F
:10AA4000BDA731E020E0892B09F030E0032F122F61
:10AA500002C000E010E08F2D0F94BDA78017910772
:10AA600011F40C9468680F94AA7D80E00F945C0E3A
:10AA700080E00F94812FEFCF83E50F947E9B882396
:10AA800031F00F94759B0F9442B58B0102C00EE616
:10AA900010E080E50F947E9B882329F00F94759B2E
:10AAA0000F9442B502C068EE73E06B01770FEE08B9
:10AAB000FF081016110694F4809101079091020787
:10AAC000029718F4C8010F94065EC701B6010F94EF
:10AAD000FB8684E50F94404D0C946868C701B6016D
:10AAE0000F94FB860C94686880E50F947E9B882306
:10AAF00051F00F94759B6093E1107093E210809376
:10AB0000E3109093E41089E40F947E9B882381F0F6
:10AB10000F94759B2CEA35EC47E25EE30F94E9A7AE
:10AB20006093E5107093E6108093E7109093E8101F
:10AB300084E40F947E9B882381F00F94759B2CEA0C
:10AB400035EC47E25EE30F94D1B46093E910709363
:10AB5000EA108093EB109093EC1083E40F947E9BAB
:10AB6000882351F00F94759B60930002709301024B
:10AB700080930202909303020F943D82EDE5F7E18A
:10AB800084918F01882339F00E9462AD0F5F1F4FBF
:10AB9000F8018491F7CF06E114E0D8018D918D0181
:10ABA000882319F00E9462ADF8CF6091E110709196
:10ABB000E2108091E3109091E41042E00E9405AE13
:10ABC0000AE114E0F80181918F01882319F00E94B5
:10ABD00062ADF8CF2CEA35EC47E25EE36091E51018
:10ABE0007091E6108091E7109091E8100F94D1B425
:10ABF00042E00E9405AE0EE114E0D8018D918D0176
:10AC0000882319F00E9462ADF8CF2CEA35EC47E2B8
:10AC10005EE36091E9107091EA108091EB109091E1
:10AC2000EC100F94E9A742E00E9405AE02E214E0A6
:10AC3000F80181918F01882319F00E9462ADF8CF4D
:10AC400060910002709101028091020290910302D2
:10AC500042E00E9405AE8AE00E9462AD0C946868F2
:10AC600080E50F947E9B882351F00F94759B609331
:10AC7000ED107093EE108093EF109093F01089E434
:10AC80000F947E9B882381F00F94759B2CEA35EC02
:10AC900047E25EE30F94E9A76093F1107093F2101E
:10ACA0008093F3109093F41084E40F947E9B882398
:10ACB00081F00F94759B2CEA35EC47E25EE30F942C
:10ACC000D1B46093F5107093F6108093F7109093C1
:10ACD000F8100F943D82EDE5F7E184918F01882310
:10ACE00039F00E9462AD0F5F1F4FF8018491F7CFDA
:10ACF00006E114E0D8018D918D01882319F00E949E
:10AD000062ADF8CF6091ED107091EE108091EF1070
:10AD10009091F01042E00E9405AE0AE114E0F801C3
:10AD200081918F01882319F00E9462ADF8CF2CEA3F
:10AD300035EC47E25EE36091F1107091F210809182
:10AD4000F3109091F4100F94D1B442E00E9405AE3C
:10AD50000EE114E0D8018D918D01882319F00E9435
:10AD600062ADF8CF2CEA35EC47E25EE36091F51076
:10AD70007091F6108091F7109091F8100F94E9A758
:10AD800042E00E9405AE8AE00E9462AD0C946868C1
:10AD900083E50F947E9B882319F00F94759B03C065
:10ADA00060E070E0CB0160932402709325028093F1
:10ADB0002602909327020C94686885E40F947E9B8A
:10ADC000882359F00F94759B0F9442B524967FAF5A
:10ADD0006EAF249777FF05C013C024961FAE1EAE3A
:10ADE000249763961FAE639765961FAE659726E11D
:10ADF00067962FAF679733E468963FAF68970EC0AA
:10AE000063961FAE639765961FAE65974CE867968D
:10AE10004FAF679752E468965FAF689783E50F94EA
:10AE20007E9B882371F00F94759B63966FAF639739
:10AE300065967FAF659767968FAF679768969FAF68
:10AE4000689783E40F947E9B882349F00F94759B49
:10AE50000F9442B5A6967FAF6EAFA69706C085E069
:10AE600090E0A6969FAF8EAFA697A6968EAC9FACAD
:10AE7000A6979092300E80922F0E1092240F10926F
:10AE8000320E1092310E0F94138862966CAF7DAF24
:10AE90008EAF9FAF62972496AEACBFAC2497B7FC41
:10AEA00005C02AE0A7962FAFA79704C03DE2A7965A
:10AEB0003FAFA7970F941388E3966CAF7DAF8EAF2B
:10AEC0009FAFE39724968EAC9FAC24971814190477
:10AED000B4F406E214E0D8018D918D01882319F0B5
:10AEE0000E9462ADF8CF8AE00E9462AD81E080935B
:10AEF000240F1092320E1092310E0C94686800E507
:10AF000014E0F80181918F01882319F00E9462AD4D
:10AF1000F8CF8AE00E9462AD0F94943A24968EACEA
:10AF20009FAC24978FE7892809F451C080935B0F69
:10AF300062968CAC9DACAEACBFAC62976C968CAE9E
:10AF40009DAEAEAEBFAE6C97AF968CAE9DAEAEAEC4
:10AF5000BFAEAF972B961FAE2B976D961FAE6D971A
:10AF600020E46E962FAF6E973CE16F963FAF6F97E0
:10AF700046E4A0964FAFA097A1961FAEA197A296C8
:10AF80001FAEA297A3961FAEA397A4961FAEA49739
:10AF9000EFE78E2E912CA12CB12C2A968CAE9DAE73
:10AFA000AEAEBFAE2A97FFE74F2E512C612C712C0D
:10AFB000AB961CAE1DAE1EAE1FAEAB9721E0E89661
:10AFC0002FAFE8971AAE1EAE212C312C06C080930D
:10AFD0005C0FAECF80E00F94812FA89580915D0F1C
:10AFE000882309F474C10F94B84124968EAC9FACA9
:10AFF0002497892859F49090DC0F9AAEA090DD0F29
:10B00000AEAE2090DE0F3090DF0F0AC0B090080780
:10B01000BAAE809009078EAE20900A0730900B07D9
:10B020002AAD3EADA101A1966FADA197A2967FADCD
:10B03000A297A3968FADA397A4969FADA4970F94C4
:10B040002EB6181674F09AACA1969FAEA197AEAC2E
:10B05000A296AFAEA297A3962FAEA397A4963FAEAB
:10B06000A4976D962FAD6D976E963FAD6E976F96C8
:10B070004FAD6F97A0965FADA0976AAD7EADC10151
:10B080000F942EB6181674F0BAAC6D96BFAE6D97CD
:10B090008EAC6E968FAE6E976F962FAE6F97A09612
:10B0A0003FAEA0970F941388DC01CB01E3968CACE4
:10B0B0009DACAEACBFACE39788199909AA09BB094E
:10B0C000853C9940A105B10550F00F94887D0F94FF
:10B0D0001388E3966CAF7DAF8EAF9FAFE397E89692
:10B0E0008FACE897882009F474C02AAD3EADA10169
:10B0F00063966FAD639765967FAD659767968FADE5
:10B10000679768969FAD68970F947CAE87FFDFC006
:10B110000F941388DC01CB0162968CAC9DACAEAC75
:10B12000BFAC629788199909AA09BB09893893416C
:10B13000A105B10508F4CBC0D301C2012A968CAC9D
:10B140009DACAEACBFAC2A9788199909AA09BB0976
:10B150002496AEACBFAC2497B595A79597958795E7
:10B16000AB2819F080935B0F02C080935C0F0F94A3
:10B1700013886C966CAF7DAF8EAF9FAF6C974B0111
:10B180005C0162962CAD3DAD4EAD5FAD6297821A0B
:10B19000930AA40AB50AAB968CAE9DAEAEAEBFAE16
:10B1A000AB9763968FAC6397A1968FAEA197659688
:10B1B0009FAC6597A2969FAEA2976796AFAC679734
:10B1C000A396AFAEA3976896BFAC6897A496BFAEA0
:10B1D000A4972AAD3EADA10163966FAD63976596C6
:10B1E0007FAD659767968FAD679768969FAD6897B7
:10B1F0000F942EB6181614F00C94C56E0F94138885
:10B20000DC01CB016C968CAC9DACAEACBFAC6C974A
:10B2100088199909AA09BB0989389341A105B10583
:10B2200010F40C94C56E0F94138862966CAF7DAFCA
:10B230008EAF9FAF6297DC01CB0188199909AA09EB
:10B24000BB092091310E3091320E1216130614F400
:10B250000C94F06C2A968CAD9DADAEADBFAD2A9727
:10B26000840D951DA61DB71D24968EAC9FAC24970A
:10B27000B595A79597958795892811F40C94C16E7B
:10B2800080935B0F8091310E9091320E01969093D6
:10B29000320E8093310E63969FAC63976D969FAE8E
:10B2A0006D976596AFAC65976E96AFAE6E976796E5
:10B2B000BFAC67976F96BFAE6F9768968FAC689775
:10B2C000A0968FAEA09721E0E8962FAFE89720E0F8
:10B2D00030E040EA51E463966FAD639765967FADC9
:10B2E000659767968FAD679768969FAD68970F943F
:10B2F000E3B32AAD3EADA1010F947CAE87FF0EC033
:10B30000E9EDFCE084918F01882309F4ECCD0E94E3
:10B3100062AD0F5F1F4FF8018491F6CF0F94138831
:10B32000DC01CB01AF968CAC9DACAEACBFACAF97A3
:10B3300088199909AA09BB09813D9740A105B10562
:10B3400008F4B4C024968EAC9FAC2497892881F071
:10B35000E0905B0FF12CE6EDFCE084918F018823F7
:10B36000B9F00E9462AD0F5F1F4FF8018491F7CFD3
:10B37000E0905C0FF12CE3EDFCE084918F018823D9
:10B3800039F00E9462AD0F5F1F4FF8018491F7CF33
:10B3900042E06AAD7EADC1010E9405AEEFECFCE07B
:10B3A00084918F01882339F00E9462AD0F5F1F4F97
:10B3B000F8018491F7CFB701FF0C880B990B0E941D
:10B3C000EBAD8AE00E9462AD2B968FAC2B97882064
:10B3D00009F452C0A7969FACA797891418F4282D9A
:10B3E0002F5F59C02B968FAC2B97A7969FACA79732
:10B3F000891054C0282D2F5F2B962FAF2B97E496E2
:10B400002FADE497E5963FADE597E6964FADE6970D
:10B41000E7965FADE7976AAD7EADC1010F94E2B3E9
:10B420006B017C0120E030E0A9010F942EB61816C4
:10B430005CF420E030E040EA50E4C701B6010F942C
:10B440007CAE87FF2BC00AC020E030E040EA50EC21
:10B45000C701B6010F942EB6181604F524966FADE9
:10B460002497661F6627661F80E00F94C73D81E022
:10B470008093240F0C9468688AACE4968FAEE497AE
:10B480009EACE5969FAEE597E6962FAEE697E796DB
:10B490003FAEE79721E02B962FAF2B970F941388A1
:10B4A000AF966CAF7DAF8EAF9FAFAF970F94138801
:10B4B0006B017C010F9413886C960CAD1DAD2EAD05
:10B4C0003FAD6C9762968CAC9DACAEACBFAC629756
:10B4D000080D191D2A1D3B1DC01AD10AE20AF30AE4
:10B4E000DC01CB018C0D9D1DAE1DBF1D81389F441D
:10B4F000A241B10570F0E2EBFCE084918F0188235A
:10B5000009F4F1CC0E9462AD0F5F1F4FF8018491E6
:10B51000F6CF8091310E9091320EA6968EAC9FACF4
:10B52000A697881699060CF055CDE6E5FCE08491C7
:10B530008F01882309F4D7CC0E9462AD0F5F1F4FA3
:10B54000F8018491F6CF0F9486830C9468688091FB
:10B550007B13882311F40C94686885E40F947E9B18
:10B56000882331F00F94759B0F9448B5162F01C0B6
:10B570001FEF86E40F947E9B882331F00F94759B18
:10B580000F9448B5062F01C00FEF1F920F931F9223
:10B590001F9385E49CE09F938F930F9487AD1F9238
:10B5A0000F931F921F938BEB9BE59F938F930F94A9
:10B5B000D5A60FB6F894DEBF0FBECDBF1AE00F942C
:10B5C0005C26181614F40C946868115011F00C9451
:10B5D000CA6E0C9468680E9414AF0C9468680E944C
:10B5E000DEAE0C9468688091DC108F938091DB1044
:10B5F0008F938091DA108F938091D9108F938091DF
:10B60000D8108F938091D7108F938091D6108F93FD
:10B610008091D5108F938091D4108F938091D31007
:10B620008F938091D2108F938091D1108F9306E9E0
:10B630001EE51F930F931F930F938091D0108F934C
:10B640008091CF108F938091CE108F938091CD10E9
:10B650008F938091CC108F938091CB108F9380919A
:10B66000CA108F938091C9108F938091C8108F93C7
:10B670008091C7108F938091C6108F938091C510D1
:10B680008F938091C4108F938091C3108F9380917A
:10B69000C2108F938091C1108F938091C0108F93AF
:10B6A0008091BF108F938091BE108F938091BD10B9
:10B6B0008F938091BC108F938091BB108F9380915A
:10B6C000BA108F938091B9108F938091B8108F9397
:10B6D0008091B7108F938091B6108F938091B510A1
:10B6E0008F931F930F931F930F938091B4108F9399
:10B6F0008091B3108F938091B2108F938091B1108D
:10B700008F938091B0108F938091AF108F93809121
:10B71000AE108F938091AD108F931F930F931F9353
:10B720000F93809134118F93809133118F93809177
:10B7300032118F93809131118F93809130118F93BB
:10B7400080912F118F9380912E118F9380912D11C5
:10B750008F9380912C118F9380912B118F938091D7
:10B760002A118F93809129118F93809128118F93A3
:10B77000809127118F93809126118F9380912511AD
:10B780008F931F930F931F930F938091AC108F9300
:10B790008091AB108F938091AA108F938091A91004
:10B7A0008F938091A8108F938091A7108F93809191
:10B7B000A6108F938091A5108F938091A4108F93E2
:10B7C0008091A3108F938091A2108F938091A110EC
:10B7D0008F938091A0108F9380919F108F93809171
:10B7E0009E108F9380919D108F931F930F931F93A3
:10B7F0000F93809124118F93809123118F938091C7
:10B8000022118F93809121118F93809120118F931A
:10B8100080911F118F9380911E118F9380911D1124
:10B820008F9380911C118F9380911B118F93809126
:10B830001A118F93809119118F93809118118F9302
:10B84000809117118F93809116118F93809115110C
:10B850008F931F930F931F930F9380919C108F933F
:10B8600080919B108F9380919A108F938091991063
:10B870008F93809198108F93809197108F938091E0
:10B8800096108F93809195108F93809194108F9341
:10B89000809193108F93809192108F93809191104B
:10B8A0008F93809190108F9380918F108F938091C0
:10B8B0008E108F9380918D108F931F930F931F93F2
:10B8C0000F9380918C108F9380918B108F93809128
:10B8D0008A108F93809189108F93809188108F9315
:10B8E000809187108F93809186108F93809185101F
:10B8F0008F93809184108F93809183108F93809188
:10B9000082108F93809181108F93809180108F93FC
:10B9100080917F108F9380917E108F9380917D1006
:10B920008F931F930F931F930F9385E999E09F9334
:10B930008F930F9487AD0FB6F894DEBF0FBECDBFC7
:10B940002CEA35EC47E25EE36091E9107091EA1071
:10B950008091EB109091EC100F94E9A79F938F9337
:10B960007F936F932CEA35EC47E25EE36091E5103C
:10B970007091E6108091E7109091E8100F94D1B487
:10B980009F938F937F936F938091E4108F93809117
:10B99000E3108F938091E2108F938091E1108F9349
:10B9A0001F930F931F930F9388E699E09F938F93B4
:10B9B0000F9487AD2CEA35EC47E25EE36091F51019
:10B9C0007091F6108091F7109091F8100F94E9A7FC
:10B9D0009F938F937F936F932CEA35EC47E25EE35E
:10B9E0006091F1107091F2108091F3109091F41029
:10B9F0000F94D1B49F938F937F936F938091F010A6
:10BA00008F938091EF108F938091EE108F938091A0
:10BA1000ED108F931F930F931F930F9383E399E080
:10BA20009F938F930F9487AD0FB6F894DEBF0FBE30
:10BA3000CDBF8091FB101F928F931F930F931F9385
:10BA40000F9320E030E040E752E460910C117091D8
:10BA50000D1180910E1190910F110F94E9A79F93F2
:10BA60008F937F936F9380910B118F9380910A1125
:10BA70008F93809109118F93809108118F931F9359
:10BA80000F931F930F93809107118F93809106114D
:10BA90008F93809105118F93809104118F9320E0F3
:10BAA00030E040E752E46091001170910111809103
:10BAB0000211909103110F94E9A79F938F937F93A5
:10BAC0006F938091FF108F938091FE108F938091E0
:10BAD000FD108F938091FC108F931F930F931F93F2
:10BAE0000F9382E398E09F938F930F9487AD0FB6E7
:10BAF000F894DEBF0FBECDBF809110118823E9F00E
:10BB0000809114118F93809113118F938091121152
:10BB10008F93809111118F931F930F931F930F9306
:10BB20008CE098E09F938F930F9487AD0FB6F894B5
:10BB3000DEBF0FBECDBF0C9468681F930F938DEED0
:10BB400097E09F938F930F9487AD0F900F900F9076
:10BB50000F900C946868E6E9FEE584918F018823D4
:10BB600039F00E9462AD0F5F1F4FF8018491F7CF4B
:10BB7000EAE9FEE084918F01882311F40C9468684F
:10BB80000E9462AD0F5F1F4FF8018491F5CF8AE5E7
:10BB90000F947E9B882309F489C00F94759B6B01D9
:10BBA0007C0120E030E040E751EC0F942EB687FD99
:10BBB00038C020E030E040EA50ECC701B6010F94F5
:10BBC0007CAE181674F1F7FAF094F7F8F094C0927E
:10BBD000DD10D092DE10E092DF10F092E010E6E986
:10BBE000FEE584918F01882339F00E9462AD0F5FDA
:10BBF0001F4FF8018491F7CFE8E0F6E084918F01C0
:10BC0000882339F00E9462AD0F5F1F4FF8018491C5
:10BC1000F7CF8AE00E9462AD8AE00E9462AD0C9488
:10BC20006868E6E9FEE584918F01882339F00E9477
:10BC300062AD0F5F1F4FF8018491F7CFE8E0F6E0A7
:10BC400084918F01882339F00E9462AD0F5F1F4FEE
:10BC5000F8018491F7CFECE2F6E084918F0188231C
:10BC600039F00E9462AD0F5F1F4FF8018491F7CF4A
:10BC700061EF7FEF8FEF9FEF0E94EBADE4E2F6E024
:10BC800084918F01882339F00E9462AD0F5F1F4FAE
:10BC9000F8018491F7CF6BEF7FEF8FEF9FEF0E945A
:10BCA000EBAD8AE00E9462AD0C946868E6E9FEE5BF
:10BCB00084918F01882339F00E9462AD0F5F1F4F7E
:10BCC000F8018491F7CFE8E0F6E084918F018823B2
:10BCD00039F00E9462AD0F5F1F4FF8018491F7CFDA
:10BCE0008AE00E9462AD8091DD109091DE10A091FB
:10BCF000DF10B091E010BC01CD01905842E00E94ED
:10BD000005AE8AE00E9462AD0C9468680F94868349
:10BD100085E40F947E9B882329F00F94759B6B011B
:10BD20007C0105C0C12CD12CE12C00ECF02E8CE460
:10BD30000F947E9B81110F94759B8AE50F947E9BD7
:10BD4000882329F00F94759B2B013C011CC020E037
:10BD500030E048EC51E460913D1070913E108091CC
:10BD60003F10909140100F947CAE87FF07C0412C8C
:10BD7000512C18ED612E11E4712E05C0412C512C6F
:10BD8000612CB0E47B2E88E50F947E9B882339F0EC
:10BD90000F94759B6AAF7BAF8CAF9DAF0AC0812CAF
:10BDA000912CA3E5AA2EA3E4BA2E8AAE9BAEACAE2C
:10BDB000BDAE89E50F947E9B882349F00F94759B57
:10BDC00022966CAF7DAF8EAF9FAF229706C02296B2
:10BDD0001CAE1DAE1EAE1FAE229780917B13882332
:10BDE00011F40C94D06E83E694E00E949DA7882302
:10BDF00011F40C94D06E332433940F9486831092F4
:10BE00002E0F8091C80F882329F060E086E190E032
:10BE10000F94B202909043022F969FAE2F972090DE
:10BE20004402E091FE0CF0E0EE0FFF1FE757FA4EE0
:10BE3000A080B1806496BFAEAEAE64972091BB196E
:10BE40003091BC1966963FAF2EAF66978091351042
:10BE500090913610A0913710B091381026968CAF83
:10BE60009DAFAEAFBFAF269789839A83AB83BC8368
:10BE70008090391090903A10A0903B10B0903C10F8
:10BE80002A968CAE9DAEAEAEBFAE2A978D829E82B4
:10BE9000AF82B88620913D1030913E1040913F1006
:10BEA000509140102E962CAF3DAF4EAF5FAF2E9706
:10BEB00029873A874B875C87209141103091421047
:10BEC00040914310509144102D873E874F87588BE7
:10BED000C701B6010F94E3B3609341107093421011
:10BEE00080934310909344104EEF5CE05F934F9328
:10BEF000812C912C68EEA62E62E4B62E71E4C72E3A
:10BF000070E1D72E2E96ECACFDAC0EAD1FAD2E978A
:10BF10002A962CAD3DAD4EAD5FAD2A9726966CAD01
:10BF20007DAD8EAD9FAD26970E9445870F94868389
:10BF300020913D1030913E1040913F1050914010A3
:10BF4000C301B2010F94E3B37B018C0160933D10F8
:10BF500070933E1080933F109093401020913910C1
:10BF600030913A1040913B1050913C106091351047
:10BF7000709136108091371090913810AEEFBCE080
:10BF8000BF93AF93812C912CE0E7AE2EE1E4BE2E5F
:10BF90000E9445870F9486838AAC9BACACACBDAC49
:10BFA0008092351090923610A0923710B0923810CF
:10BFB00022962CAD3DAD4EAD5FAD2297209339104A
:10BFC00030933A1040933B1050933C10E0903D105A
:10BFD000F0903E1000913F10109140104EEF5CE049
:10BFE0005F934F93812C912CF8E4AF2EF2E4BF2E97
:10BFF00022962CAD3DAD4EAD5FAD22976AAD7BADC7
:10C000008CAD9DAD0E9445870F9486830F900F9055
:10C010000F900F900F900F9080917B13811124C08F
:10C0200084E090E090932302809322020F9413887F
:10C030004B015C0180E091E10F948707CC24C3940D
:10C04000D12CE12CF12CD1100C94146F0F94593099
:10C05000882311F40C94146F9FB7F8948091020117
:10C060008B7F809302019FBF1092B60680917B1355
:10C07000882319F00F949E2502C00E94D0D40F94FB
:10C08000868380917B13811160C084E090E090935F
:10C0900023028093220241E060E089E192E10F9463
:10C0A00094078093B60681114BC00F940B3762E062
:10C0B00080E00F945C3286E799E40F94833120E0AE
:10C0C00030E048EC52E46091351070913610809168
:10C0D0003710909138100F94E2B36093351070933D
:10C0E00036108093371090933810E0903D10F09008
:10C0F0003E1000913F101091401020913910309166
:10C100003A1040913B1050913C10EEEFFCE0FF9351
:10C11000EF93812C912CE8E4AE2EE2E4BE2EF1E404
:10C12000CF2EF0E1DF2E0E9445870F94868389EEA3
:10C1300091E10F94350881E00F9415370F900F901F
:10C1400080917B13882309F477C0311071C08091EE
:10C150003F0E882329F060E080912D0E0F94692412
:10C1600084E090E0909323028093220289E291E19F
:10C170000F948707FF24F39400E010E00F945930E8
:10C18000811139C00F94AA7D81E00F945C0E043FA9
:10C1900041E0140711F400E010E080910101846097
:10C1A0008093010101151105A1F48091010790917F
:10C1B0000207009721F00197B9F4FF20A9F09FB77B
:10C1C000F894809102018460809302019FBFF12C5A
:10C1D0000BC00431110541F49FB7F894809102011E
:10C1E0008B7F809302019FBF0F5F1F4F84E090E021
:10C1F0000F94B112C3CF9FB7F894809102018B7F47
:10C20000809302019FBF80913F0E882389F00F9495
:10C210000B3762E080E00F945C3286E799E40F947C
:10C22000833180E60F945E2460E080E00F944F211C
:10C23000832D0F9491A456C00F940B3761E080E0DA
:10C240000F945C3282E891E10F94833162E080E0E8
:10C250000F945C328FE691E10F94833184E090E09B
:10C2600090932302809322020E94629D0F94593082
:10C2700081111AC00F94AA7D81E00F945C0E0E9478
:10C28000AD9D882399F38091010790910207029751
:10C2900020F488EE93E00F94065E82E390E00F9422
:10C2A000B11284E50F94404D0E94009C82E090E022
:10C2B00090932302809322020F94DD9B80910107CB
:10C2C00090910207029720F484EF91E00F94065EAC
:10C2D00082E390E00F94B11284E50F94404D80E02A
:10C2E0000F9415373110F1C01092B606A4E0CA2E93
:10C2F000D12CB2E0AB2EB12C8091B606813009F47E
:10C30000E4C01092B606D0922302C09222020F948B
:10C310000B3760E080E00F945C3288EB91E10F9482
:10C32000833161E081E00F945C328FEB9FE20F94E8
:10C33000833162E081E00F945C3284EA91E10F94F2
:10C34000833163E081E00F945C3282E991E10F94E4
:10C35000833161E080E00F945C3288E694E00F94D2
:10C36000FE30E090BD190E2C000CFF0801E010E03B
:10C370008091B606811168C00F94AA7D81E00F9468
:10C380005C0E8091BD19082E000C990B9701281B9B
:10C39000390B37FF03C0319521953109253031051F
:10C3A0000CF444C08E159F0514F401501109E816D1
:10C3B000F90634F40F5F1F4F0430110564F009C013
:10C3C0000430110534F40115110529F401E010E0E1
:10C3D00002C003E010E061E080E00F945C3289E588
:10C3E00096E00F94FE3062E080E00F945C3289E5C5
:10C3F00096E00F94FE3063E080E00F945C3289E5B4
:10C4000096E00F94FE30602F80E00F945C3288E657
:10C4100094E00F94FE30E090BD190E2C000CFF0844
:10C4200064E670E080E090E00F94FB860F94593052
:10C43000882309F49DCF0093B60664EF71E080E095
:10C4400090E00F94FB8694CF0F940B370F94268ABD
:10C45000B0922302A09222028091B6068230F9F0B7
:10C46000833041F50F9486830E9462EA0F940B3764
:10C4700060E080E00F945C328BEC91E10F948331AB
:10C4800062E080E00F945C3286E799E40F94833198
:10C4900087E99DE10F943C9C0F9486832DCF80917A
:10C4A0007B13882321F080E00F9491A425CF0F9473
:10C4B000DD9B22CF0F940B3762E080E00F945C325B
:10C4C00089ED91E10F94833117CF81E00F941537F7
:10C4D00066968EAD9FAD66979093BC198093BB19FD
:10C4E00031103FC020E030E040EA50E4609141105C
:10C4F0007091421080914310909144100F94E3B3D7
:10C5000060934110709342108093431090934410B5
:10C51000E0903D10F0903E1000913F1010914010BF
:10C520002091391030913A1040913B1050913C10BD
:10C5300060913510709136108091371090913810BD
:10C54000EEEFFCE0FF93EF93812C912CA12CE0E423
:10C55000BE2EF1E4CF2EF0E1DF2E0E9445870F9032
:10C560000F90E0903D10F0903E1000913F10109120
:10C5700040102D813E814F81588569817A818B8160
:10C580009C81EEEF6E2EECE07E2E7F926F92812CDE
:10C59000912CF8E4AF2EF2E4BF2EA1E4CA2EA0E164
:10C5A000DA2E0E9445870F948683E984FA840B85EE
:10C5B0001C852D813E814F81588569817A818B81CF
:10C5C0009C817F926F92812C912CB0E7AB2EB1E4CD
:10C5D000BB2E0E9445870F948683CE010D960E9444
:10C5E000C9BD80E1FE013196A5E3B0E101900D9255
:10C5F0008A95E1F780E1E5E3F0E1A9ECBFE0019085
:10C600000D928A95E1F72F969FAD2F979093430255
:10C61000209244022F929F9384EE97E09F938F93F2
:10C620008E01015E1F4F1F930F930F94E0AD60E0EA
:10C63000C8010E9459DB8FEB94E10F94DC511092FA
:10C64000410E1092400E0FB6F894DEBF0FBECDBF64
:10C650003FC50E946CCE3CC583E50F947E9B88232A
:10C6600009F436C50F94759B0F9442B56B017C019C
:10C670002B0186E799E40F94DC51E7E7FEE0849113
:10C680008F01882339F00E9462AD0F5F1F4FF801C0
:10C690008491F7CF0D2C000CEE08FF08C701B601FE
:10C6A0000E94EBAD8AE00E9462AD0F9413884B01AB
:10C6B0005C0110925A0E6091020D7091030D072ECD
:10C6C000000C880B990B0F9482AE20E030E0A9019A
:10C6D0000F947CAE811111C06091891570918A15FB
:10C6E000072E000C880B990B0F9482AE11E020E00E
:10C6F00030E0A9010F947CAE811110E0052C000CF4
:10C700006608770882E7282E8EE0382E111115C0B2
:10C7100080915A0E81116CC0C301B2010F9482AE98
:10C720002091A10E3091A20E4091A30E5091A40E23
:10C730000F942EB618168CF05BC0C301B2010F9493
:10C7400082AE2091A10E3091A20E4091A30E509185
:10C75000A40E0F947CAE87FF4BC00F941388DC01AE
:10C76000CB0188199909AA09BB09893E9340A10503
:10C77000B10508F434C0E4E7FEE084915F0188234A
:10C7800041F00E9462ADFFEFAF1ABF0AF50184913C
:10C79000F6CF6091A10E7091A20E8091A30E9091A0
:10C7A000A40E41E00E9405AEF101849102E7A02EA3
:10C7B0000EE0B02E882341F00E9462ADFFEFAF1A69
:10C7C000BF0AF5018491F6CFC701B6010E94EBAD17
:10C7D0008AE00E9462AD0F9413884B015C010F94B4
:10C7E000AA7D80E00F945C0E80E00F94812F8ECFA5
:10C7F0008DE597E10F94DC516BC48FE30F947E9B22
:10C80000882309F4BCC00E9484A91A821982882353
:10C8100081F00AE614E0D8018D918D01882319F08A
:10C820000E9462ADF8CF8AE00E9462AD0EE714E08C
:10C830000AC005E914E0F80181918F01882399F37A
:10C840000E9462ADF8CFD8018D918D01882319F037
:10C850000E9462ADF8CF8AE00E9462AD88248A947B
:10C86000982C5401A3E24A2E512C612C712CB0EB70
:10C870002B2EBFE03B2E1AAE69817A81072E000C69
:10C88000880B990B0F9482AE209185103091861001
:10C8900040918710509188100F94D1B46B017C01A6
:10C8A0002AAD21110DC0EEE6FEE084918F018823B0
:10C8B00059F00E9462AD0F5F1F4FF8018491F7CFCE
:10C8C000C501B4010E94EBADEBE6FEE084918F015F
:10C8D000882339F00E9462AD0F5F1F4FF8018491E9
:10C8E000F7CFC301B2010E94EBADE8E6FEE0849110
:10C8F0008F01882339F00E9462AD0F5F1F4FF8014E
:10C900008491F7CF69817A81072E000C880B990BEF
:10C910000E94EBADE5E6FEE084918F01882339F0BB
:10C920000E9462AD0F5F1F4FF8018491F7CF20E0A6
:10C9300030E04AE754E4C701B6010F94E9A742E0AA
:10C940000E9405AE8AE00E9462ADFAADFF5FFAAFC9
:10C95000F63009F4BDC3BE016F5F7F4FC1010E9475
:10C9600092FDB2E02B0E311CE5E04E0E511C611C15
:10C97000711CFFEF8F1A9F0AAF0ABF0A7DCF81E2B9
:10C980000F947E9B882309F44AC061E086EA9FE009
:10C990000F9487B388E090E09A838983BE016F5F2C
:10C9A0007F4F80EB9FE00E94ACFD88E190E09A838E
:10C9B0008983BE016F5F7F4F82EB9FE00E94ACFDD9
:10C9C00080E390E09A838983BE016F5F7F4F84EBA1
:10C9D0009FE00E94ACFD80E590E09A838983BE01D0
:10C9E0006F5F7F4F86EB9FE00E94ACFD88E790E091
:10C9F0009A838983BE016F5F7F4F88EB9FE00E941F
:10CA0000ACFD09EA14E0D8018D918D01882319F05D
:10CA10000E9462ADF8CF8AE00E9462AD59C38AE5F8
:10CA20000F947E9B882319F161E086EA9FE00F94C2
:10CA300087B31A82198200EB1FE0BE016F5F7F4F40
:10CA4000C8010E94ACFD0E5F1F4F0A3BBFE01B07F1
:10CA5000A1F70AEB14E0F80181918F01882319F006
:10CA60000E9462ADF8CF8AE00E9462AD31C383E5D7
:10CA70000F947E9B882309F4CEC00F94759B0F946E
:10CA800042B57A83698389E40F947E9B882309F4F5
:10CA90001FC30F94759B0F9448B5653008F018C3F9
:10CAA000862F90E08852984FBE016F5F7F4F880FAE
:10CAB000991F0E94ACFD04EC14E0D8018D918D010A
:10CAC000882319F00E9462ADF8CF8AE00E9462AD1F
:10CAD0000EE714E0F80181918F01882319F00E947C
:10CAE00062ADF8CF8AE00E9462AD3EEA232E3FE0BD
:10CAF000332E44244A94542C320153E2852E912C37
:10CB0000A12CB12C1AAE1A821982FAADFF2331F092
:10CB1000BE016F5F7F4FC1010E9492FD69817A81E2
:10CB2000072E000C880B990B0F9482AE2091851074
:10CB30003091861040918710509188100F94D1B495
:10CB40006B017C012AAD21110DC0E1E6FEE084916C
:10CB50008F01882359F00E9462AD0F5F1F4FF801CB
:10CB60008491F7CFC301B2010E94EBADEEE5FEE088
:10CB700084918F01882339F00E9462AD0F5F1F4FAF
:10CB8000F8018491F7CFC501B4010E94EBADEBE54C
:10CB9000FEE084918F01882339F00E9462AD0F5F1F
:10CBA0001F4FF8018491F7CF69817A81072E000C1D
:10CBB000880B990B0E94EBADE8E5FEE084918F01B4
:10CBC000882339F00E9462AD0F5F1F4FF8018491F6
:10CBD000F7CF20E030E04AE754E4C701B6010F94F4
:10CBE000E9A742E00E9405AE8AE00E9462ADFAAD7C
:10CBF000FF5FFAAF25E0820E911CA11CB11C3FEF34
:10CC0000431A530A630A730A42E0240E311CF630B9
:10CC100009F079CF5DC2E7E4FEE084918F018823BB
:10CC200009F456C20E9462AD0F5F1F4FF801849154
:10CC3000F6CF0F9486838BE40F947E9B882399F024
:10CC40000F943F9B6B017C0120E030E0A9010F9421
:10CC50002EB687FD08C0C092180DD092190DE09233
:10CC60001A0DF0921B0D82E50F947E9B882361F0D4
:10CC70000F943F9B6B017C0120E030E0A9010F94F1
:10CC80007CAE87FF89C006C0C12CD12C20E8E22EE3
:10CC90002FEBF22E84E40F947E9B882329F00F94CF
:10CCA0003F9B4B015C0106C0812C912C90E8A92E82
:10CCB0009FEBB92E87E50F947E9B882329F00F9474
:10CCC0003F9B2B013C0106C0412C512C80E8682E73
:10CCD0008FEB782E88E40F947E9B882339F00F9495
:10CCE0003F9B6AAF7BAF8CAF9DAF08C020E030E0C8
:10CCF00040E85FEB2AAF3BAF4CAF5DAF20E030E0E8
:10CD0000A901C501B4010F942EB687FD45C020E0EE
:10CD100030E0A901C301B2010F942EB687FD3CC0DB
:10CD200020E030E0A9016AAD7BAD8CAD9DAD0F94E4
:10CD30002EB687FD31C020E030E0A901C501B40165
:10CD40000F947CAE882391F120E030E040E05FE377
:10CD5000C501B4010F94E9A76B017C012AAD3BAD7D
:10CD60004CAD5DADC301B2010F94E9A74B015C016D
:10CD7000A7019601C701B6010F94E9A72BED3FE08B
:10CD800049E450E40F94E9A79B01AC01C501B4014B
:10CD90000F94D1B46B017C0120E030E0A901C70100
:10CDA000B6010F942EB687FF04C00BC0C12CD12C46
:10CDB0007601C092140DD092150DE092160DF092EE
:10CDC000170DE6E9FEE584918F01882339F00E9472
:10CDD00062AD0F5F1F4FF8018491F7CFE9EDF7E0E7
:10CDE00084918F01882339F00E9462AD0F5F1F4F3D
:10CDF000F8018491F7CF6091180D7091190D809111
:10CE00001A0D90911B0D42E00E9405AE8AE00E942F
:10CE100062ADE3EDF7E084918F01882339F00E9441
:10CE200062AD0F5F1F4FF8018491F7CFC090140DD2
:10CE3000D090150DE090160DF090170D20E030E029
:10CE4000A901C701B6010F947CAE882349F042E0E6
:10CE5000C701B6010E9405AE8AE00E9462AD38C1EA
:10CE6000EEECF7E084918F01882311F40C94F445E3
:10CE70000E9462AD0F5F1F4FF8018491F5CF0F94B0
:10CE80006A9B0F9482AE6B017C0120E030E0A90127
:10CE90000F947CAE87FD40C020E030EA40E854E4C7
:10CEA000C701B6010F942EB6181674F120E030E0D9
:10CEB00047E054E4C701B6010F942EB687FD2FC09A
:10CEC00020E030E04CE752E4C701B6010F94E9A737
:10CED00020E030EA40E854E40F94D1B40F9448B510
:10CEE000162F802F0F94AD9B612F802F0F949C9B4A
:10CEF0000F5F043009F4ECC0D5018D915D010F94F2
:10CF00007E9B8823A9F3BBCFC12C10EAD12E10E859
:10CF1000E12E14E4F12ED4CFC12CD12C760120E0E7
:10CF200030E04CE752E4C701B6010F94E9A720E0D6
:10CF300034EB40E954E4D0CF85E40F947E9B882302
:10CF400009F4C6C00F94759B0F9448B56B017C0122
:10CF50008B016830710569F06031710551F0603204
:10CF6000710539F06034710521F06038710509F000
:10CF7000AFC00F94868380E091E05C0100901307BE
:10CF800002C0B694A7940A94E2F7C6010E94B2C602
:10CF90008093130720911C0240912002682F83E0A8
:10CFA0000E94D5C640907510509076106090771012
:10CFB00070907810A016B10670F5C801B5010F94F5
:10CFC00081B86B01E12CF12CC701B6010F9480AE42
:10CFD0009B01AC016091891070918A1080918B1037
:10CFE00090918C100F94E9A76093891070938A1028
:10CFF00080938B1090938C10A3019201C701B6010E
:10D000000F9498B360937510709376108093771097
:10D01000909378105DC0C501B8010F9481B86B0181
:10D02000E12CF12CC701B6010F9480AE9B01AC013D
:10D030006091891070918A1080918B1090918C1062
:10D040000F94D1B46093891070938A1080938B10E1
:10D0500090938C10C301B201A70196010F94A8B858
:10D06000209375103093761040937710509378107A
:10D070002FC080917B13882329F085E40F947E9B39
:10D0800081117BC70F944B6523C083E40F947E9B73
:10D0900090917B13882329F09923D1F00F949E253A
:10D0A00017C09111FBCF0E94D0D412C08091871578
:10D0B0009091881583569C4E9F938F9382E39EE0B8
:10D0C0009F938F930F9487AD0F900F900F900F90B9
:10D0D00010922D0F10922C0F90C284E50F947E9B1E
:10D0E000882309F41BC120912B0D30912C0DF901DF
:10D0F00031968F01021B130B7F0181918032C9F39E
:10D100008930B9F3082E000C990B0F94E4B8F7019D
:10D110008083E0912B0DF0912C0DE00FF11F8081A9
:10D1200090ED980F953008F458C08F3309F43CC047
:10D13000883781F0833649F1E2E2FEE084918F0185
:10D14000882309F4E7C00E9462AD0F5F1F4FF8010A
:10D150008491F6CF80917B13882309F44EC240E07E
:10D1600050E067EA70E381ED92E10E94F1D580938F
:10D170002C0E0F94868380912C0E805F0F945E247A
:10D1800061E081E00F944F2138C280917B138823A6
:10D1900009F433C20F94868380E30F945E24809158
:10D1A0002C0E80932D0E45C080917B1340E050E003
:10D1B000882351F067EA70E381ED92E10E94F1D596
:10D1C00080932C0E11E010C067EB72E180EC92E1CD
:10D1D0000E94F1D580932C0E06C00F94759B0F947E
:10D1E00048B560932C0E10E00F94868380912C0E2E
:10D1F00021E030E0082E01C0220F0A94EAF7909156
:10D20000330F292B2093330F90917B139923A1F097
:10D21000805F0F945E2461E081E00F944F2180E3F2
:10D220000F945E2480912C0E80932D0E112309F40F
:10D23000E4C10F942B20E1C1882309F432C0E6E950
:10D24000FEE584918F01882339F00E9462AD0F5F63
:10D250001F4FF8018491F7CFE0E2FEE084918F0147
:10D26000882339F00E9462AD0F5F1F4FF80184914F
:10D27000F7CF60912C0E70E080E090E00E94EBAD63
:10D280008AE00E9462ADE7EFF5E084918F01882388
:10D2900009F440C00E9462AD0F5F1F4FF8018491F6
:10D2A000F6CF86E40F947E9B882399F00F94759BAC
:10D2B0006B017C0120E030E0A9010F942EB6181616
:10D2C00044F4C0927E02D0927F02E0928002F092FB
:10D2D0008102E6E9FEE584918F01882339F00E94FE
:10D2E00062AD0F5F1F4FF8018491F7CFE5EEF5E0D7
:10D2F00084918F01882339F00E9462AD0F5F1F4F28
:10D30000F8018491F7CF6091FE0C70E080E090E02E
:10D310000E94EBAD8AE00E9462AD6FC184E40F947D
:10D320007E9B882309F408C10F94759B0F9442B526
:10D330006330710509F061C18EE995E09F938F9389
:10D340000F9487AD81E40F947E9B0F900F908823FC
:10D35000B9F080912B0D90912C0DDC0111962C9140
:10D36000283741F440E150E060E070E002960F940D
:10D3700011AA04C00F94759B0F9442B58B0102C093
:10D3800000E010E083E40F947E9B882339F00F9433
:10D39000759B0F9442B5262F872F02C020E080E1B5
:10D3A0001F71A22EB82EB1E0AB16B0E1BB0618F08B
:10D3B000A12CB0E1BB2EC501800F911F813090419F
:10D3C00028F080E090E15C01A01AB10A88E50F9492
:10D3D0007E9B882309F475C020912B0D30912C0D74
:10D3E000A9014F5F5F4F9E012F5F3F4F6901F90118
:10D3F000E12CF12C9A01D9018C912F5F3F4F8823AA
:10D40000A1F140E1E416F10469F18032A1F38A3020
:10D4100061F190ED980F9A3018F48295807F07C0E3
:10D420009FE9980F9630A8F48295807F8057AD01D0
:10D430004E5F5F4F11969C9120ED290F2A3010F41A
:10D44000822B0BC02FE9290F263018F49755892B12
:10D4500004C0F194E194F10808C081936FEFE61ADB
:10D46000F60AC8CFA0E1EA2EF12C5701E114F1042D
:10D4700041F1812C912CD6016D916D01C401800F79
:10D48000911F0F9487B3BFEF8B1A9B0AE814F9041E
:10D4900091F71F930F93FF92EF9281E795E09F938F
:10D4A0008F930F9487AD6091D1197091D2198AE052
:10D4B00090E00F9402AD0F900F900F900F900F908F
:10D4C0000F906801E12CF12CA114B10409F495C06E
:10D4D0008D2D0F94939B8C2D0F94939B6091D1195C
:10D4E0007091D21980E290E00F9402AD10E1EFEF5D
:10D4F000CE1ADE0AEE0AFE0AC60101970F9457B350
:10D50000082F6091D1197091D21980E290E00F94A8
:10D5100002AD802F0F94939B1150F1E0AF1AB10828
:10D5200011F01111E4CF6091D1197091D2198AE0F4
:10D5300090E00F9402ADC8CFE6E9FEE584918F013B
:10D54000882339F00E9462AD0F5F1F4FF80184916C
:10D55000F7CFE1E1F6E084918F01882339F00E9452
:10D5600062AD0F5F1F4FF8018491F7CF00918715CF
:10D570001091881503561C4ED8018D918D0188237A
:10D5800019F00E9462ADF8CFEBE1FEE084918F01CB
:10D59000882309F4BFCE0E9462AD0F5F1F4FF801D0
:10D5A0008491F6CFC090D50FD090D60FE090D70FD2
:10D5B000F090D80F209141103091421040914310CB
:10D5C00050914410C701B6010F94E2B34B015C01C6
:10D5D0002DEC3CEC4CEC5DEB0F947CAE87FD3AC03F
:10D5E0002DEC3CEC4CEC5DE3C501B4010F942EB680
:10D5F00018160CF438C00F94C8A081E090E0909306
:10D600002302809322020F9413886093FF0E70937D
:10D61000000F8093010F9093020FE0918715F09116
:10D620008815E656FC4E8081813019F0863009F06D
:10D63000C6C4EDE5F7E184918F01882339F00E949B
:10D6400062AD0F5F1F4FF8018491F7CF8AE00E940F
:10D6500062ADB5C4E091FE0CF0E0E752F04F80817E
:10D66000811192C409C0E091FE0CF0E0E752F04F46
:10D670008081882309F4BFCFC0924110D09242101C
:10D68000E0924310F092441081E490E10E94C9BD01
:10D69000E091FE0CF0E0E752F04F908181E08927A5
:10D6A0000F94F0A48CC420E030E040E85FE3609188
:10D6B00041107091421080914310909144100F944A
:10D6C000E3B36093411070934210809343109093A2
:10D6D0004410E0903D10F0903E1000913F101091EA
:10D6E00040102091391030913A1040913B105091E8
:10D6F0003C106091351070913610809137109091E8
:10D700003810EEEFFCE0FF93EF93812C912CE8ECC6
:10D71000AE2EE3E4BE2EF1E4CF2EF0E1DF2E0E9428
:10D7200045870F900F900C94594182E090E09093C0
:10D730002302809322021092470E1092460E0C9400
:10D740009F450F946A9BAB01BC0140935B195093BA
:10D750005C1960935D1970935E1986EA98E10E94E6
:10D7600002E0B6CC0F94759B0F9442B58B010C94DC
:10D7700062490F94868388E50F947E9B882319F075
:10D78000179A1092FF0C89E50F947E9B882319F05D
:10D79000169A1092000D8AE50F947E9B85E40F94F3
:10D7A0007E9B882311F40C94DE4D149A0C94DE4D6C
:10D7B0001A8219824AE050E0BE016F5F7F4FC701B5
:10D7C0000F9411AA78A36F8F89819A818816990680
:10D7D00009F07ECC4AE050E0BE016F5F7F4FC6018A
:10D7E0000F9411AA7AA369A389819A816816790690
:10D7F00009F06ECC4AE050E0BE016F5F7F4FC5017B
:10D800000F9411AA7CA36BA389819A810817190729
:10D8100009F05ECC8FE790E09EA38DA35801EFEF57
:10D82000AE1ABE0AD8018C918D3211F575016701CF
:10D83000BFEFCB1ADB0AF70180810F94B251382E6B
:10D84000811102C07601F3CFEA18FB08DE2CC70174
:10D8500099278330910569F543E050E06BED7BE556
:10D86000C5010F945AAC892B09F042C01EA21DA21B
:10D87000332009F42DCCCE0101960F94FF63882349
:10D8800009F426CCFE017F96DE011196AE01495DBA
:10D890005F4F219131918D919D918217930708F4EB
:10D8A0004CC02817390708F413CC4E175F0789F7C7
:10D8B0000FCC8530910571F445E050E065ED7BE5D6
:10D8C000C5010F945AAC892B99F481E090E09EA396
:10D8D0008DA3CECF049761F444E050E060ED7BE58A
:10D8E000C5010F945AAC892B19F482E090E0EFCF78
:10D8F0008EEF8E0D823008F0EBCBD80111968C9113
:10D9000011978F7D823509F0E3CB12968C918F7D34
:10D91000833409F0DDCBB2E0DB1203C083E090E09A
:10D92000D6CFF801838190ED980F9A3008F0D0CBD4
:10D93000082E000C990B8E97CACF89E492E10F94C0
:10D94000870745E65DE062E080E00F940037D20192
:10D950001D912D01812F0F94B251811108C067ECE8
:10D9600076E0812F110F990B0F9402ADF0CF49E3B0
:10D9700052E163E080E00F940037809101079091BD
:10D980000207029720F488EE93E00F94065E82E38C
:10D9900090E00F94B11284E50F94404D84EF91E034
:10D9A0000F94B1128091010790910207029720F421
:10D9B00088EE93E00F94065E82E390E00F94B1123C
:10D9C00084E50F94404D80E090E00F94609C81E0EE
:10D9D0000F9415370F940B3780E00F94812F78CB7D
:10D9E000AB96CCACDDACEEACFFACAB97C80ED91EA1
:10D9F000EA1EFB1EAB962CAD3DAD4EAD5FADAB97B9
:10DA0000281B390B4A0B5B0B2A966CAD7DAD8EAD96
:10DA10009FAD2A970F9498B3A70196010F94A8B8C9
:10DA2000DA01C901840D951DA61DB71D843191052C
:10DA3000A105B105E4F02C013D018C3E9105A10545
:10DA4000B1052CF06BEE462E512C612C712C40E868
:10DA50004416510461047104DCF05EEF852E912CB4
:10DA6000A12CB12C84189508A608B7080AC034E187
:10DA7000432E512C612C712C44E1842E912CA12C2D
:10DA8000B12C2A968CAE9DAEAEAEBFAE2A9706C024
:10DA90002A964CAE5DAE6EAE7FAE2A97E2E4FDE014
:10DAA00084918F01882339F00E9462AD0F5F1F4F70
:10DAB000F8018491F7CFC301B2010E94EBADEDE311
:10DAC000FDE084918F01882339F00E9462AD0F5FE1
:10DAD0001F4FF8018491F7CF2A966CAD7DAD8EADC6
:10DAE0009FAD2A970E94EBADE6E3FDE084918F01A4
:10DAF000882339F00E9462AD0F5F1F4FF8018491B7
:10DB0000F7CF42E06D966FAD6D976E967FAD6E97D5
:10DB10006F968FAD6F97A0969FADA0970E9405AEB0
:10DB2000EFE2FDE084918F01882339F00E9462AD1D
:10DB30000F5F1F4FF8018491F7CF42E0A1966FADC0
:10DB4000A197A2967FADA297A3968FADA397A49617
:10DB50009FADA4970E9405AE8AE00E9462AD8091BD
:10DB6000310E9091320E039714F40C942A592A9690
:10DB70006CAD7DAD8EAD9FAD2A970F9482AE20E047
:10DB800030E040E850E40F94E9A74B015C016D964A
:10DB90002FAD6D976E963FAD6E976F964FAD6F97A9
:10DBA000A0965FADA097A1966FADA197A2967FAD0D
:10DBB000A297A3968FADA397A4969FADA4970F9419
:10DBC000E2B320ED3FE049E450E40F94E9A720E000
:10DBD00030E040E05FE30F94E9A79B01AC01C50191
:10DBE000B4010F94D1B44B015C01C701B6010F948D
:10DBF00082AE20E030E04AE754E40F94D1B46B01E8
:10DC00007C01E9E2FDE084918F01882339F00E94D4
:10DC100062AD0F5F1F4FF8018491F7CF42E0C5015D
:10DC2000B4010E9405AEE3E2FDE084918F018823F8
:10DC300039F00E9462AD0F5F1F4FF8018491F7CF5A
:10DC400042E0C701B6010E9405AE8AE00E9462ADC3
:10DC50002AE939E949E15FE3C501B4010F94E9A775
:10DC60004B015C016093200F7093210F8093220F72
:10DC70009093230F9B01AC010F94E3B3A70196018E
:10DC80000F94D1B460931C0F70931D0F80931E0FDF
:10DC900090931F0FA5019401C701B6010F94E9A746
:10DCA00020E030E040E05EE30F94E9A76093180FB6
:10DCB0007093190F80931A0F90931B0FE5E1FDE00D
:10DCC00084918F01882339F00E9462AD0F5F1F4F4E
:10DCD000F8018491F7CF8AE00E9462ADEFE0FDE0A9
:10DCE00084918F01882339F00E9462AD0F5F1F4F2E
:10DCF000F8018491F7CF6091200F7091210F8091EE
:10DD0000220F9091230F42E00E9405AE8AE00E940C
:10DD100062ADE9E0FDE084918F01882339F00E9433
:10DD200062AD0F5F1F4FF8018491F7CF60911C0F18
:10DD300070911D0F80911E0F90911F0F42E00E9465
:10DD400005AE8AE00E9462ADE3E0FDE084918F01C0
:10DD5000882339F00E9462AD0F5F1F4FF801849154
:10DD6000F7CF6091180F7091190F80911A0F909151
:10DD70001B0F42E00E9405AE8AE00E9462AD0C9447
:10DD80002A5980935C0F0C944259E8961FAEE8978D
:10DD90000C94675984E690E00F94B1120C94DF5A0A
:10DDA000312C0C94FD5EE12CF12C809101018460FA
:10DDB00080930101E114F10409F04EC08091010744
:10DDC000909102070097F1F10197D1F19FEFE91AC5
:10DDD000F90AA1E0DA1609F452C0DA1608F04AC0CE
:10DDE00084E090E00F94B1120F94138895018401A0
:10DDF0000054184D264F3F4F0617170728073907BD
:10DE000010F00C94236085ED90E10F9487071F8E2E
:10DE100018A219A21AA2CE014F960F946D760F94F4
:10DE20008683149ADD24D3940F94AA7D81E00F9405
:10DE30005C0EF4EFEF16F1E0FF0609F0B6CFB3CFBA
:10DE4000CC2021F29FB7F8948091020184608093E6
:10DE500002019FBFC12CBACF84E1E816F10409F09A
:10DE6000B5CF9FB7F894809102018B7F8093020118
:10DE70009FBFACCFB2E0DB16E1F00C94236084E0EE
:10DE800090E00F94B1120F945930882369F2E09119
:10DE9000FE0CF0E0EE0FFF1FE757FA4E64962EAD32
:10DEA0003FAD6497318320830E9441FD42E0D42E30
:10DEB000BBCF0091FE0C10E0F801EE0FFF1FE757FB
:10DEC000FA4E60817181072E000C880B990B0F941C
:10DED00082AE000F111F000F111FF801E452F04F26
:10DEE00020813181428153810F94E2B32B013C01A7
:10DEF00020E030E0A9010F942EB618165CF420E063
:10DF000030E040E85FE3C301B2010F947CAE87FFCD
:10DF100016C00AC020E030E040E85FEBC301B20168
:10DF20000F942EB618165CF480E091E10F948707E9
:10DF30000F9413884B015C01D12C0C94266064E093
:10DF400081E00F945C32E091FE0C34E0E39FF0013D
:10DF50001124E452F04F80819181A281B3818F8F8F
:10DF600098A3A9A3BAA3CE014F960E943AA00F94FA
:10DF7000FE30A4E1EA2EF12C57CF0F94759B0F943D
:10DF800048B560932C0E7EC82DEC3CEC4CEC5DE368
:10DF9000C501B4010F942EB618160CF46DCB2BCB23
:10DFA000A5019401F101662D772D8F2F922D0F94ED
:10DFB0007CAE181614F40C94AD3A0C94BD3AC958C2
:10DFC000DF4F0FB6F894DEBF0FBECDBFDF91CF910C
:10DFD0001F910F91FF90EF90DF90CF90BF90AF9087
:10DFE0009F908F907F906F905F904F903F902F9079
:10DFF00008952F923F924F925F926F927F928F92ED
:10E000009F92AF92BF92CF92DF92EF92FF920F93C7
:10E010001F93CF93DF93CDB7DEB7C95CD1090FB69D
:10E02000F894DEBF0FBECDBF782E81E00F948A66D4
:10E03000711025C01092030D1092020D19821A82E0
:10E040001B821C82CE0101960F946D7661E080ECFC
:10E050009FE00F9469B360E08FEB9FE00F9469B38A
:10E0600060E08EEB9FE00F9469B360E08DEB9FE082
:10E070000F9469B360E08CEB9FE00F9469B380E08C
:10E080000F9415370F94E3600F94E92C1092FD0C58
:10E090001092FC0C83E0EFEFFCE0DF011D928A950B
:10E0A000E9F781E00E94CFA5C855DF4F99838883A7
:10E0B000C85AD04083E69CE10F9487070E94FEA5D2
:10E0C00040E050E061E080E090E00F94CB6640E0FB
:10E0D00050E061E081E090E00F94CB66E0903D106D
:10E0E000F0903E1000913F10109140102091391097
:10E0F00030913A1040913B1050913C106091351096
:10E100007091361080913710909138100F94A85963
:10E110000E94C6BC1092210220E030E040EA50E4A8
:10E1200060913510709136108091371090913810B1
:10E130000F94E3B31B012C016093351070933610DC
:10E14000809337109093381020E030E040EA50E49C
:10E150006091391070913A1080913B1090913C1071
:10E160000F94E3B39B01AC016093391070933A10A4
:10E1700080933B1090933C10E0903D10F0903E1047
:10E1800000913F10109140108EEF9CE09F938F9371
:10E19000812C912CA0EAAA2EA1E4BA2EB1E4CB2EB8
:10E1A000B0E1DB2EC201B1010E9445870F94868346
:10E1B0000E9408A60F900F90882311F40C94D88326
:10E1C00089E29CE10F943508772089F089EF9BE183
:10E1D0000F94870763E080E00F945C3261E070E0A9
:10E1E00080E090E00F94E33083EF9BE110C083ED7B
:10E1F0009BE10F94870762E080E00F945C3261E05E
:10E2000070E080E090E00F94E3308DEC9BE10F94A0
:10E2100083310F94C06671102EC084E090E090931B
:10E2200023028093220240E060E082EB9BE10F94A6
:10E230009407882321F08AE89BE10F94350884EF46
:10E240009AE10F94350882E090E090932302809346
:10E25000220283ED9BE10F94870762E080E00F9438
:10E260005C3261E070E080E090E00F94E3308DEC90
:10E270009BE10F94833180E090E0A0EAB0E48093CA
:10E280003D1090933E10A0933F10B09340106090CB
:10E29000210281E08093210284E00F94ED37E09029
:10E2A0003D10F0903E1000913F10109140102091D1
:10E2B000391030913A1040913B1050913C106091D0
:10E2C0003510709136108091371090913810EEEF24
:10E2D000FCE0FF93EF93812C912CE0EAAE2EE1E479
:10E2E000BE2EF1E4CF2EF0E1DF2E0E9445870F9481
:10E2F00086830F9452376092210282E00F947383D9
:10E300000F900F9020E030E040EA50E40F947CAE94
:10E3100081110C94D4837720E9F0C855DF4F8881B0
:10E320009981C85AD0400E94AEA50F94D82E0F9460
:10E33000EB2A0F948A32882311F40C9484830E9470
:10E34000BAAC803F11F00C94D08381E00E948EA97A
:10E350000C94D0838AEF0E948EA960E070E088EF71
:10E360009FE00F9483B30F94C06684ECEDE8F5E171
:10E37000DF011D928A95E9F7EAE0FFE184918F01C0
:10E38000882339F00E9462AD0F5F1F4FF80184911E
:10E39000F7CF61E070E080E090E00E94EBAD0E947A
:10E3A00097AEBE016F5A7F4F83ED9BE10F947507C7
:10E3B00062968FAD6297843020F083E062968FAFD3
:10E3C000629780E090E0A0EAB0E480933D109093E3
:10E3D0003E10A0933F10B09340102AEE3EE1C65786
:10E3E000DF4F39832883CA58D0408CE895E1CE5757
:10E3F000DF4F99838883C258D040A0969FAF8EAFDD
:10E40000A097A8963FAF2EAFA89781E090E0A0E03C
:10E41000B0E0AE968CAF9DAFAEAFBFAFAE970F94EE
:10E42000C06662966FAD629780E00F945C32AE96E4
:10E430006CAD7DAD8EAD9FADAE970F94E3308DEC9E
:10E440009BE10F94833165E575E585E591E40F94D3
:10E450007D2AA896EEADFFADA89785919591A591DF
:10E46000B4918093351090933610A0933710B093E9
:10E470003810A896EEADFFADA8973496859195918A
:10E48000A591B4918093391090933A10A0933B10CA
:10E49000B0933C1060E070E088E492E40F947D2A31
:10E4A00000912D1010912E1020912F1030913010CE
:10E4B0004091291050912A1060912B1070912C10CE
:10E4C0008091251090912610A0912710B0912810CE
:10E4D0003F932F931F930F937F936F935F934F936C
:10E4E000BF93AF939F938F9386E79EE19F938F9304
:10E4F0000F9487AD0F94868340912510509126107C
:10E5000060912710709128108091291090912A1005
:10E51000A0912B10B0912C10C0902D10D0902E10E7
:10E52000E0902F10F090301021E00FB6F894DEBF8D
:10E530000FBECDBF413157420CF420E081319742EC
:10E5400014F00C94DA83822F90E0880F991FFC015D
:10E55000E259F14EA590B490FC01EA59F14E859034
:10E560009490DF92CF929F928F92BF92AF921F9220
:10E570002F938DE49EE19F938F930F9487AD8DE64B
:10E580009CE19F938F930F9487AD0F94943A809161
:10E590006E008B7F80936E00EF9880916F008D7F6F
:10E5A00080936F000FB6F894A89580916000886101
:10E5B00080936000109260000FBE1092FB0C1092CE
:10E5C000FA0C88ED91E09093F90C8093F80C8CEAAA
:10E5D00091E09093F70C8093F60C00E028EC30E08B
:10E5E000A601B401C5010F94E34D00912D101091C7
:10E5F0002E1020912F103091301040912910509101
:10E600002A1060912B1070912C1080912510909100
:10E610002610A0912710B09128103F932F931F939D
:10E620000F937F936F935F934F93BF93AF939F939A
:10E630008F938DE09DE19F938F930F9487AD809191
:10E64000251090912610A0912710B0912810782EB7
:10E65000692E8091291090912A10A0912B10B091D1
:10E660002C10582E492EC0902D10D0902E10E090D6
:10E670002F10F09030100FB6F894DEBF0FBECDBF54
:10E6800044E8242E4CE1342E95E0C91697EFD906C4
:10E690000CF46FC01A8219821F921F92A3E0AF93ED
:10E6A000B4E8BF931F92E4E6EF93DF92CF924F92CC
:10E6B0005F926F927F923F922F920F9487AD0FB629
:10E6C000F894DEBF0FBECDBF89819A81803D924014
:10E6D00030F089819A81803A954058F512C0FE0148
:10E6E00031967F0100E010E024E833E0A601652DBB
:10E6F000742D872D962D0F94AF6281110C94DF83BA
:10E70000E8CF9E012F5F3F4F790100E010E02CE73A
:10E710003CEFA60144565109652D742D872D962D89
:10E720000F94AF62882329F089819A8180539D4F8D
:10E730001CC089819A818037984008F04AC0CE0178
:10E7400001967C0104EB10E024E833E0A601485C6C
:10E750005109652D742D872D962D0F94AF62882356
:10E76000C1F189819A8180569A4F9A8389830C944A
:10E77000DF8300912D1010912E1020912F103091D9
:10E7800030104091291050912A1060912B107091F7
:10E790002C108091251090912610A0912710B091F7
:10E7A00028103F932F931F930F937F936F935F9343
:10E7B0004F93BF93AF939F938F938CEB9CE19F9369
:10E7C0008F930F9487AD0FB6F894DEBF0FBECDBF09
:10E7D000D4C389819A8180349B4098F4DE011196DC
:10E7E0007D0104EB10E02CE73CEFA6014C525140B8
:10E7F000652D742D872D962D0F94AF6281110C9489
:10E80000C68480E0E981FA81882311F40C94E283C4
:10E810008091251090912610A0912710B09128107A
:10E820004091291050912A1060912B1070912C105A
:10E8300000912D1010912E1020912F10309130103A
:10E84000FF93EF931F930F935F934F939F938F9338
:10E8500089EE9CE19F938F930F9487AD40912D108B
:10E8600050912E1060912F107091301000E028EC24
:10E8700030E0B401C5010F94E34D85E08F9380E74C
:10E880008F938DE19EE19F938F930F9487AD84E0EA
:10E890008F9388E38F938BE09EE19F938F930F94E8
:10E8A00087AD8091251090912610A0912710B091EE
:10E8B00028106A968CAF9DAFAEAFBFAF6A976896CF
:10E8C000CEACDFAC68978091291090912A10A0916E
:10E8D0002B10B0912C10E2968CAF9DAFAEAFBFAFB6
:10E8E000E29780912D1090912E10A0912F10B09151
:10E8F00030106E968CAF9DAFAEAFBFAF6E971C0160
:10E9000098E4291A310889E08F9380E68F933F922B
:10E910002F92E096AFADE097AF93AF96BFADAF97B4
:10E92000BF936896EFAD6897EF936796FFAD6797D3
:10E93000FF9386E39DE19F938F930F9487AD409162
:10E940002D1050912E1060912F10709130107A017F
:10E9500020E931E0E0966EAD7FADE09768968EAD30
:10E960009FAD68970F94E34DE0962EAD3FADE097D5
:10E970003450E4963FAF2EAFE4970FB6F894DEBF65
:10E980000FBECDBF812C912CD601B450EC96BFAFF9
:10E99000AEAFEC97F601FC5FC258DF4FF983E88316
:10E9A000CE57D040382D3170A3963FAFA39780FC4F
:10E9B00002C00C94E883EF968FADEF97C158DF4FFC
:10E9C0009881CF57D04000E020E931E0A701E496DC
:10E9D0006EAD7FADE4970F94E34DC0902910D090B9
:10E9E0002A10E0902B10F0902C108091251090911F
:10E9F0002610A0912710B091281001E028EC30E0FB
:10EA0000A101B6010F94E34DC0902910D0902A10B7
:10EA1000E0902B10F0902C108091251090912610F2
:10EA2000A0912710B09128100FEF28EC30E040E6BD
:10EA300059E0B6010F94E34D80912D1090912E1066
:10EA4000A0912F10B09130107C01A3968FADA397A9
:10EA5000882311F40C94F08380910B0181608093E2
:10EA60000B010000840195E0000F111F9A95E1F75A
:10EA7000A3969FADA397992311F40C94F58380EC92
:10EA8000482E55245A94652C752CC12CD12CA0E409
:10EA9000E796AFAFE797A12CB12C93B1A70142192C
:10EAA0005309292F207194FF02C00C94FC8388EE37
:10EAB0009FEF840F951F97FD02C00C94008480E0A7
:10EAC00090E0A80EB91E80910B0121110C940A84CC
:10EAD000846080930B01000021110C940D842E148E
:10EAE0003F0434F484E00E9432BDB1E0EB1AF10837
:10EAF00081E00E9432BD8BE599E00197F1F7E7963E
:10EB00002FADE7972150E7962FAFE7972111C5CF9B
:10EB1000A6E0B694A794AA95E1F7A3963FADA39774
:10EB2000332311F40C941C848FE190E08C199D091F
:10EB3000800F911FFC01EA57F84FA08280912510A9
:10EB400090912610A0912710B0912810840D951D4A
:10EB5000A61DB71D8093251090932610A093271013
:10EB6000B0932810C7010F2C000CAA0BBB0B80938D
:10EB70002D1090932E10A0932F10B09330108FEF84
:10EB8000C81AD80A90E2C916D10409F080CF0A57F2
:10EB9000184FE0E2BE2EF1E3CF2EFDE1DF2ED801CB
:10EBA0008D918D011F928F93DF92CF920F9487AD3D
:10EBB000BA940F900F900F900F90B110F0CF8FE29A
:10EBC0009DE19F938F930F9487ADBFEF8B1A9B0AA4
:10EBD000E496EEADFFADE497E05CFF4FE496FFAF47
:10EBE000EEAFE4970F900F90F0E28F16910409F0CA
:10EBF000D9CE76E8A72E7BE0B72E86EA9BE0F5011A
:10EC0000119211928E179F07D9F780E090E0DC01F6
:10EC100065E0AA0FBB1F6A95E1F7AA57B84F40E01D
:10EC2000ED91F0E034E0F595E7953A95E1F7EE0FD8
:10EC3000FF1FEA57F44F208131812F5F3F4F31830F
:10EC400020834F5F403261F7019680329105F9F6DB
:10EC500096E8C92E9BE0D92E00E010E02EE6E22EC9
:10EC60002DE1F22ED6018C9111969C91B2E0CB0E43
:10EC7000D11C9F938F931F930F93FF92EF920F944A
:10EC800087AD0F5F1F4F0F900F900F900F900F9059
:10EC90000F900031110531F78091880B9091890B0D
:10ECA000E8E8FBE031E021E04191519184179507BC
:10ECB00010F4322FCA012F5F2031B1F7032F1F92BA
:10ECC0003F939F938F9385E99DE19F938F930F943B
:10ECD00087ADE4EAFBE00F900F900F900F900F903C
:10ECE0000F908EE0329122912A30310510F40C946D
:10ECF0001F848295807F2091860B3091870B20376F
:10ED0000334010F00C942684000F000F000F182FD2
:10ED1000101B1F921F931F928F931F920F938EE7CA
:10ED20009DE19F938F930F9487AD86E8482E87E0EF
:10ED3000582E0FB6F894DEBF0FBECDBFF201202FC4
:10ED400030E0012F10E0808190E02817390710F0A3
:10ED50000C942984821B930B982F80E0B8010F94A8
:10ED600081B86F3F710519F010F06FEF70E061939B
:10ED7000AE16BF0641F700E010E0A9E7AA2EADE10C
:10ED8000BA2EB7E7CB2EBDE1DB2EC801F5E0880F28
:10ED9000991FFA95E1F7DC01AA57B84F7D01912C34
:10EDA000F70181917F011F928F93BF92AF920F94D1
:10EDB00087AD93940F900F900F900F90F0E29F12F9
:10EDC000EFCFDF92CF920F9487AD0F5F1F4F0F9061
:10EDD0000F9000321105C9F683EF9DE12EED3BE067
:10EDE000A6ECBBE0FC01459154914D935D930296D6
:10EDF0002A173B07B9F7612C712C812C912C10E05C
:10EE000000E050E060E070E0B62E26EC3BE0E496D7
:10EE10003FAF2EAFE497A0E0B0E080E090E040E0AC
:10EE200020E030E07D01E60EF71E1701260C371CAE
:10EE3000EEEFAE2EA40E41110C942D84FEEFFF2EAA
:10EE4000F20EE7E0EF1510F00C9433842F5F3F4F84
:10EE50002C30310581F74F5F9096E4962EAD3FAD93
:10EE6000E4972E5F3F4FE4963FAF2EAFE4974C30D0
:10EE7000B9F6881699061CF44C01052F1B2D6F5FFF
:10EE80007F4F6431710509F0BFCF5F5F30E2630EE1
:10EE9000711C543109F0B6CF9F928F921F920F933D
:10EEA0001F921F9389EA9DE19F938F930F9487ADE3
:10EEB0000FB6F894DEBF0FBECDBF93E48916910460
:10EEC00014F40C9468841F920F931F921F938AED81
:10EED0009DE19F938F930F9487AD1A5FE12EF12CE4
:10EEE000A0E1EA1AF108B6E0EE0CFF1CBA95E1F7D2
:10EEF0006896EEADFFAD6897EE0EFF1E0A5FC02E5E
:10EF0000D12CF0E1CF1AD10816E0CC0CDD1C1A95FB
:10EF1000E1F7E0962EAD3FADE097C20ED31E6C96A2
:10EF20003FAD6C973F936B968FAD6B978F93DF924E
:10EF3000CF92FF92EF9289EC9DE19F938F930F9474
:10EF400087AD00E028EC30E06C964EAD5FAD6C977D
:10EF5000B601C7010F94E34D0FB6F894DEBF0FBEA4
:10EF6000CDBF81E0F20111922F01F6EF4F16FCE0C8
:10EF70005F06C1F781110C946B8410E086E39EE17B
:10EF80009F938F930F9487AD0E94839580916E001D
:10EF9000846080936E00EF9A80916F00826080930E
:10EFA0006F0098E288E10FB6F894A895809360000E
:10EFB0000FBE909360001092FB0C1092FA0C10920E
:10EFC000F90C1092F80C1092F70C1092F60C0F90AE
:10EFD0000F90112311F40C940C8320E030E0A90170
:10EFE000A096AEADBFADA09711966D917D918D911C
:10EFF0009C9114970F94E9A7209135103091361009
:10F0000040913710509138100F94E3B3A096EEADB5
:10F01000FFADA0976183728383839483C09039107E
:10F02000D0903A10E0903B10F0903C1020E030E09F
:10F03000A90165817681878190850F94E9A7A70151
:10F0400096010F94E3B3A096AEADBFADA097159611
:10F050006D937D938D939C93189720E030E040E86A
:10F0600050ECC701B6010F947CAE87FF0CC080E066
:10F0700090E0A0E8B0EC8093391090933A10A09300
:10F080003B10B0933C1020E030E040E450E460914D
:10F090003D1070913E1080913F10909140100F9460
:10F0A000E3B360933D1070933E1080933F109093B4
:10F0B0004010AE968CAD9DADAEADBFADAE97019696
:10F0C000A11DB11DAE968CAF9DAFAEAFBFAFAE97D9
:10F0D000A896AEADBFADA8971896A896BFAFAEAF35
:10F0E000A897A096EEADFFADA0973896A096FFAF7B
:10F0F000EEAFA097AE968CAD9DADAEADBFADAE9769
:10F100000597A105B10509F08AC980E090E00F9448
:10F11000B11220E030E040E950EC6091911570911F
:10F12000921580919315909194150F947CAE87FF62
:10F1300043C0E9EEFEE184918F01882339F00E94FB
:10F1400062AD0F5F1F4FF8018491F7CF8AE00E94F4
:10F1500062ADE7EBFEE184918F01882339F00E94D4
:10F1600062AD0F5F1F4FF8018491F7CF6091911549
:10F1700070919215809193159091941542E00E94A0
:10F1800005AEE3EBFEE184918F01882339F00E9404
:10F1900062AD0F5F1F4FF8018491F7CF42E060E04E
:10F1A00070E080E990EC0E9405AE0E9497AEF2E01C
:10F1B000AF96FFAFAF9703C0AF961FAEAF97109259
:10F1C000BD151092BE151092BF151092C015109269
:10F1D000C1151092C2151092C3151092C41524E6E1
:10F1E000E3962FAFE397A2961CAE1DAE1EAE1FAEE8
:10F1F000A2976A961CAE1DAE1EAE1FAE6A97CE01D8
:10F20000019664969FAF8EAF6497DE01AF5BBF4FF0
:10F210006696BFAFAEAF66976A966CAD7DAD8EADAC
:10F220009FAD6A970F94CEB4AA966CAF7DAF8EAFA8
:10F230009FAFAA976A966CAD7DAD8EAD9FAD6A9774
:10F240000F945CB7C457DF4F688379838A839B83AD
:10F25000CC58D040A2966CAD7DAD8EAD9FADA2973F
:10F260000F94CEB4C057DF4F688379838A839B8322
:10F27000C059D040A2966CAD7DAD8EAD9FADA2972A
:10F280000F945CB7CC56DF4F688379838A839B8366
:10F29000C459D0406496EEADFFAD6497A0E4EA2E69
:10F2A0001192EA94E9F76696AEADBFAD6697E0E1DC
:10F2B0001D92EA95E9F780E090E00F94B1128091F9
:10F2C000BD159091BE15A091BF15B091C015C65542
:10F2D000DF4F88839983AA83BB83CA5AD040809129
:10F2E000C1159091C215A091C315B091C415C25516
:10F2F000DF4F88839983AA83BB83CE5AD040DE0137
:10F30000AF5BBF4FC856DF4FB983A883C859D04001
:10F31000FE013196AC96FFAFEEAFAC9700E0CC5655
:10F32000DF4F88819981AA81BB81C459D040B058F0
:10F33000EA968CAF9DAFAEAFBFAFEA97C057DF4F35
:10F3400088819981AA81BB81C059D040B058EE967E
:10F350008CAF9DAFAEAFBFAFEE97C457DF4F888184
:10F360009981AA81BB81CC58D040B058C258DF4F98
:10F3700088839983AA83BB83CE57D040AC962EACAA
:10F380003FACAC9710E07CE8472E75E1572EE4E0E7
:10F390007E2EC12CD12C7601013011F40C94EE8418
:10F3A000113011F40C94FA84002311F1023081F42D
:10F3B000D20111962D913D914D915C911497C258B7
:10F3C000DF4F688179818A819B81CE57D0400BC005
:10F3D000F2012581368147815085EE966CAD7DAD79
:10F3E0008EAD9FADEE970F94E9A74B015C0106C06F
:10F3F000812C912C60E8A62E6FE3B62E112301F12B
:10F40000123081F4D20111962D913D914D915C9174
:10F410001497C258DF4F688179818A819B81CE57CA
:10F42000D0400BC0F2012581368147815085EE9690
:10F430006CAD7DAD8EAD9FADEE970F94E9A704C086
:10F4400060E070E080E89FE39B01AC01C501B4017E
:10F450000F94E9A79B01AC01C701B6010F94E3B378
:10F460006B017C010023E1F11123D1F1023011F095
:10F470000C94CE84D20111962D913D914D915C91C9
:10F480001497AA966CAD7DAD8EAD9FADAA970F94E3
:10F49000E9A74B015C01113011F40C94E88412309F
:10F4A00011F00C94DB84D20111962D913D914D9178
:10F4B0005C911497AA966CAD7DAD8EAD9FADAA9769
:10F4C0000F94E9A79B01AC01C501B4010F94E9A712
:10F4D0009B01AC01C701B6010F94E3B36B017C0142
:10F4E0007A94F8E04F0E511C711056CFD101CD9295
:10F4F000DD92ED92FD921D011F5F143009F043CFA4
:10F500004CE8242E45E1342EEAEEFEE16C96FFAF86
:10F51000EEAF6C97CA57DF4F1882C658D040C4561A
:10F52000DF4F1882CC59D040C056DF4F1882C05AE6
:10F53000D04010E0002321F1013049F1023081F484
:10F54000D10111962D913D914D915C911497C25826
:10F55000DF4F688179818A819B81CE57D0400BC073
:10F56000F1012581368147815085EE966CAD7DADE8
:10F570008EAD9FADEE970F94E9A74B015C010AC0D9
:10F58000812C912C30E8A32E3FE3B32E03C0812CB5
:10F59000912C5401D10111964D905D906D907C900D
:10F5A0001497A3019201AA966CAD7DAD8EAD9FAD6F
:10F5B000AA970F94E9A76B017C01D10115968D9153
:10F5C0009D910D90BC91A02DA6968CAF9DAFAEAF36
:10F5D000BFAFA6976C96EEADFFAD6C9785919591F8
:10F5E000A591B491CC55DF4F88839983AA83BB83BF
:10F5F000C45AD040A6962CAD3DAD4EAD5FADA6979A
:10F60000CC56DF4F688179818A819B81C459D04073
:10F610000F94E9A79B01AC01C701B6010F94E2B3B7
:10F62000C655DF4F288139814A815B81CA5AD04053
:10F630000F94E3B3CC55DF4F288139814A815B8138
:10F64000C45AD0400F94E2B3A50194010F94E9A7E6
:10F65000CA57DF4F2881C658D040C456DF4F388183
:10F66000CC59D040C056DF4F4881C05AD040512FAE
:10F670000F94E3B3CA57DF4F688379838A839B83F0
:10F68000C658D0400023A9F00130B9F00230D9F0BB
:10F69000A6962CAD3DAD4EAD5FADA697EA966CAD8E
:10F6A0007DAD8EAD9FADEA970F94E9A76B017C010C
:10F6B0000AC0C12CD12C760106C0C12CD12C20E867
:10F6C000E22E2FE3F22E6C96EEADFFAD6C973496E2
:10F6D00085909590A590B490A3019201C457DF4FF7
:10F6E000688179818A819B81CC58D0400F94E9A7A9
:10F6F0002B013C01A6962CAD3DAD4EAD5FADA6975E
:10F70000C057DF4F688179818A819B81C059D04081
:10F710000F94E9A79B01AC01C301B2010F94E3B3BD
:10F72000C255DF4F288139814A815B81CE5AD04052
:10F730000F94E3B3A50194010F94E2B3A7019601DE
:10F740000F94E9A7CA57DF4F288139814A815B812D
:10F75000C658D0400F94E3B3CA57DF4F6883C658EA
:10F76000D040C456DF4F7883CC59D040C056DF4FCD
:10F770008883C05AD040192F6C96AEADBFAD6C9740
:10F7800018966C96BFAFAEAF6C97B8E02B0E311CDD
:10F79000ECEA2E16E5E13E0609F0CCCEDC01CB0109
:10F7A000B058C856DF4FE881F981C859D0408193DD
:10F7B0009193A193B193C856DF4FF983E883C85959
:10F7C000D0400F5FAC962EAD3FADAC97205F3F4F62
:10F7D000AC963FAF2EAFAC97043009F0CFCD259655
:10F7E0008CAD9DADAEADBFAD2597AA968CAF9DAF4C
:10F7F000AEAFBFAFAA978D819E81AF81B885AE961F
:10F800008CAF9DAFAEAFBFAFAE9789859A85AB8504
:10F81000BC85A6968CAF9DAFAEAFBFAFA6978D85CA
:10F820009E85AF85B889EA968CAF9DAFAEAFBFAF6E
:10F83000EA9789819A81AB81BC81EE968CAF9DAFAE
:10F84000AEAFBFAFEE9729968CAD9DADAEADBFAD5F
:10F850002997C258DF4F88839983AA83BB83CE57E9
:10F86000D04089899A89AB89BC89C457DF4F888386
:10F870009983AA83BB83CC58D040898D9A8DAB8D58
:10F88000BC8DC057DF4F88839983AA83BB83C0593F
:10F89000D0408D8D9E8DAF8DB8A1CC56DF4F888323
:10F8A0009983AA83BB83C459D0408D899E89AF892F
:10F8B000B88DC856DF4F88839983AA83BB83C85904
:10F8C000D0402D968CAD9DADAEADBFAD2D97CA5736
:10F8D000DF4F88839983AA83BB83C658D04089A110
:10F8E0009AA1ABA1BCA1C456DF4F88839983AA8398
:10F8F000BB83CC59D0408DA19EA1AFA1B8A5C05665
:10F90000DF4F88839983AA83BB83C05AD0408DA5DB
:10F910009EA5AFA5B8A9CC55DF4F88839983AA834C
:10F92000BB83C45AD04089A59AA5ABA5BCA5CE542B
:10F93000DF4F88839983AA83BB83C25BD0406196E3
:10F940008CAD9DADAEADBFAD6197CA54DF4F88831E
:10F950009983AA83BB83C65BD04089A99AA9ABA926
:10F96000BCA9C654DF4F88839983AA83BB83CA5B33
:10F97000D0408DA99EA9AFA9B8ADC254DF4F8883EE
:10F980009983AA83BB83CE5BD04089AD9AADABADE2
:10F99000BCADCE53DF4F88839983AA83BB83C25CFF
:10F9A000D04021968CAD9DADAEADBFAD2197CA5371
:10F9B000DF4F88839983AA83BB83C65CD04014E65B
:10F9C000C12CD12C76014601570126013701A30134
:10F9D0009201AE966CAD7DAD8EAD9FADAE970F949E
:10F9E000E9A79B01AC01AA966CAD7DAD8EAD9FAD34
:10F9F000AA970F94E2B32B013C01A5019401A696AE
:10FA00006CAD7DAD8EAD9FADA6970F94E9A79B0120
:10FA1000AC01C301B2010F94E2B32B013C01A70179
:10FA20009601EA966CAD7DAD8EAD9FADEA970F94D1
:10FA3000E9A79B01AC01C301B2010F94E2B3EE96BA
:10FA40002CAD3DAD4EAD5FADEE970F94D1B46E963B
:10FA50006CAF7DAF8EAF9FAF6E97C457DF4F2881DD
:10FA600039814A815B81CC58D0400F94E9A79B0132
:10FA7000AC01C258DF4F688179818A819B81CE5762
:10FA8000D0400F94E2B32B013C01A5019401C05773
:10FA9000DF4F688179818A819B81C059D0400F9462
:10FAA000E9A79B01AC01C301B2010F94E2B34B0182
:10FAB0005C01A7019601CC56DF4F688179818A816C
:10FAC0009B81C459D0400F94E9A79B01AC01C501AB
:10FAD000B4010F94E2B3C856DF4F288139814A81BF
:10FAE0005B81C859D0400F94D1B42B013C01C4565E
:10FAF000DF4F288139814A815B81CC59D0406E9695
:10FB00006CAD7DAD8EAD9FAD6E970F94E9A79B0157
:10FB1000AC01CA57DF4F688179818A819B81C658C1
:10FB2000D0400F94E2B34B015C01C056DF4F2881F7
:10FB300039814A815B81C05AD040C301B2010F9420
:10FB4000E9A79B01AC01C501B4010F94E2B34B01DD
:10FB50005C01A7019601CC55DF4F688179818A81CC
:10FB60009B81C45AD0400F94E9A79B01AC01C50109
:10FB7000B4010F94E2B3CE54DF4F288139814A811A
:10FB80005B81C25BD0400F94D1B44B015C01C65481
:10FB9000DF4F288139814A815B81CA5BD0406E96F4
:10FBA0006CAD7DAD8EAD9FAD6E970F94E9A79B01B7
:10FBB000AC01CA54DF4F688179818A819B81C65B21
:10FBC000D0400F94E2B36B017C01C254DF4F288117
:10FBD00039814A815B81CE5BD040C301B2010F9471
:10FBE000E9A79B01AC01C701B6010F94E2B36B0119
:10FBF0007C01CE53DF4F288139814A815B81C25C11
:10FC0000D040C501B4010F94E9A79B01AC01C70125
:10FC1000B6010F94E2B3CA53DF4F288139814A817C
:10FC20005B81C65CD0400F94D1B46B017C01115054
:10FC300009F0CDCE6E962CAD3DAD4EAD5FAD6E975D
:10FC4000C655DF4F688179818A819B81CA5AD0402D
:10FC50000F94E3B36093BD157093BE158093BF15E9
:10FC60009093C015A3019201C255DF4F688179813D
:10FC70008A819B81CE5AD0400F94E3B36093C11523
:10FC80007093C2158093C3159093C415A501940178
:10FC90006A966CAD7DAD8EAD9FAD6A970F94E3B360
:10FCA0006A966CAF7DAF8EAF9FAF6A97A701960142
:10FCB000A2966CAD7DAD8EAD9FADA2970F94E3B3D0
:10FCC000A2966CAF7DAF8EAF9FAFA297E3969FAD2C
:10FCD000E3979150E3969FAFE39791119DCA6A967F
:10FCE0006CAD7DAD8EAD9FAD6A970F94CEB4609331
:10FCF000AD157093AE158093AF159093B0156A96BD
:10FD00006CAD7DAD8EAD9FAD6A970F945CB760937F
:10FD1000B1157093B2158093B3159093B415A29654
:10FD20006CAD7DAD8EAD9FADA2970F945CB7DC013D
:10FD3000CB01B0588093B5159093B615A093B71525
:10FD4000B093B815A2966CAD7DAD8EAD9FADA29768
:10FD50000F94CEB46093B9157093BA158093BB1508
:10FD60009093BC156A962CAD3DAD4EAD5FAD6A97D4
:10FD7000A2966CAD7DAD8EAD9FADA2970F94E2B310
:10FD80006B017C01E894F7F8B701A60180E69FE0DB
:10FD90000F947BB32FE132E449E05BE3C701B60186
:10FDA0000F942EB618166CF425E33AEF4EE85BE399
:10FDB000C701B6010F942EB6181634F001E010E01A
:10FDC00005C000E010E002C002E010E025E33AEFD9
:10FDD0004EE85BE36A966CAD7DAD8EAD9FAD6A97E4
:10FDE0009F770F942EB618167CF025E33AEF4EE875
:10FDF0005BE3A2966CAD7DAD8EAD9FADA2979F7774
:10FE00000F942EB6181614F402E010E08091AD1590
:10FE10009091AE15A091AF15B091B015AE968CAF84
:10FE20009DAFAEAFBFAFAE978091B5159091B615AF
:10FE3000A091B715B091B815A6968CAF9DAFAEAF97
:10FE4000BFAFA6978091BD159091BE15A091BF152B
:10FE5000B091C015E6968CAF9DAFAEAFBFAFE69741
:10FE60008091B1159091B215A091B315B091B415D0
:10FE7000EA968CAF9DAFAEAFBFAFEA978091B91550
:10FE80009091BA15A091BB15B091BC15EE968CAFB0
:10FE90009DAFAEAFBFAFEE978091C1159091C215E7
:10FEA000A091C315B091C415C258DF4F88839983C0
:10FEB000AA83BB83CE57D040AAEEBEE16C96BFAFFB
:10FEC000AEAF6C979CE8292E95E1392EF101818027
:10FED0009280A380B48085819681A781B085AA96FF
:10FEE0008CAF9DAFAEAFBFAFAA976C96EEADFFAD36
:10FEF0006C97C590D590E590F490A5019401AE96CD
:10FF00006CAD7DAD8EAD9FADAE970F94E9A72B0183
:10FF10003C01AA962CAD3DAD4EAD5FADAA97A6961D
:10FF20006CAD7DAD8EAD9FADA6970F94E9A79B01FB
:10FF3000AC01C301B2010F94E3B3E6962CAD3DAD25
:10FF40004EAD5FADE6970F94E3B39B01AC01C701E3
:10FF5000B6010F94E2B36B017C016C96EEADFFAD80
:10FF60006C9734964590559065907490EA962CADB8
:10FF70003DAD4EAD5FADEA97C501B4010F94E9A761
:10FF80004B015C01EE962CAD3DAD4EAD5FADEE97F5
:10FF9000AA966CAD7DAD8EAD9FADAA970F94E9A7E3
:10FFA0009B01AC01C501B4010F94E3B3C258DF4F0C
:10FFB000288139814A815B81CE57D0400F94E3B3C9
:10FFC0009B01AC01C301B2010F94E2B34B015C0190
:10FFD000A7019601C701B6010F94E9A76B017C0147
:10FFE000A5019401C501B4010F94E9A79B01AC01DF
:10FFF000C701B6010F94E3B30F9467B72DEC3CEC47
:020000021000EC
:100000004CE45FE30F942EB6181614F40EEF1FEFB6
:10001000B8E02B0E311C6C96EEADFFAD6C973896A8
:100020006C96FFAFEEAF6C978CEAE82E85E1F82E68
:10003000E214F30409F04ACF0115110509F07AC161
:10004000A2962CAD3DAD4EAD5FADA2976A966CAD5C
:100050007DAD8EAD9FAD6A970F94E3B320E030E0A5
:1000600040E05FE30F94E9A76B017C010F94CEB4ED
:100070002B013C016093AD157093AE158093AF15C5
:100080009093B015C701B6010F945CB7A2966CAF00
:100090007DAF8EAF9FAFA2976093B1157093B215ED
:1000A0008093B3159093B415DC01CB01B058AA9698
:1000B0008CAF9DAFAEAFBFAFAA978093B5159093AD
:1000C000B615A093B715B093B8154092B9155092D4
:1000D000BA156092BB157092BC151092BD151092A6
:1000E000BE151092BF151092C0151092C115109236
:1000F000C2151092C3151092C4156E961CAE1DAE9B
:100100001EAE1FAE6E976A961CAE1DAE1EAE1FAE23
:100110006A97CE57DF4FA881B981C258D040119657
:100120008D909D90AD90BC90149715968D919D915A
:100130000D90BC91A02DAE968CAF9DAFAEAFBFAF72
:10014000AE97C657DF4FE881F981CA58D040C590B5
:10015000D590E590F490A5019401C301B2010F94EC
:10016000E9A7A6966CAF7DAF8EAF9FAFA697AE9670
:100170002CAD3DAD4EAD5FADAE97AA966CAD7DADED
:100180008EAD9FADAA970F94E9A79B01AC01A696EF
:100190006CAD7DAD8EAD9FADA6970F94E3B39B0183
:1001A000AC01C701B6010F94E2B32091BD153091A7
:1001B000BE154091BF155091C0150F94E3B36B016C
:1001C0007C016093BD157093BE158093BF1590930D
:1001D000C01520E030E040E85FE36A966CAD7DAD8D
:1001E0008EAD9FAD6A970F94E3B36A966CAF7DAF07
:1001F0008EAF9FAF6A97C657DF4FE881F981CA5823
:10020000D040349685919591A591B491A6968CAFE6
:100210009DAFAEAFBFAFA697A5019401A2966CADFE
:100220007DAD8EAD9FADA2970F94E9A74B015C0108
:10023000AE962CAD3DAD4EAD5FADAE97C301B201F4
:100240000F94E9A79B01AC01C501B4010F94E3B37E
:100250009B01AC01A6966CAD7DAD8EAD9FADA69712
:100260000F94E2B32091C1153091C2154091C3158E
:100270005091C4150F94E3B34B015C016093C11519
:100280007093C2158093C3159093C41520E030E09D
:1002900040E85FE36E966CAD7DAD8EAD9FAD6E9721
:1002A0000F94E3B36E966CAF7DAF8EAF9FAF6E973A
:1002B000CE57DF4FA881B981C258D0401896CE578B
:1002C000DF4FB983A883C258D040C657DF4FE881BB
:1002D000F981CA58D0403896C657DF4FF983E88372
:1002E000CA58D0402A163B0609F013CF6A962CADA7
:1002F0003DAD4EAD5FAD6A97C701B6010F94D1B465
:100300006093BD157093BE158093BF159093C01573
:100310006E962CAD3DAD4EAD5FAD6E97C501B4018F
:100320000F94D1B46093C1157093C2158093C31517
:100330009093C4154090AD155090AE156090AF15D8
:100340007090B015C090B915D090BA15E090BB155B
:10035000F090BC158091B1159091B215A091B31594
:10036000B091B415A2968CAF9DAFAEAFBFAFA297C0
:100370008091B5159091B615A091B715B091B815AB
:100380006A968CAF9DAFAEAFBFAF6A97A7019601DB
:10039000C301B2010F94E9A74B015C016A962CAD31
:1003A0003DAD4EAD5FAD6A97A2966CAD7DAD8EADA5
:1003B0009FADA2970F94E9A79B01AC01C501B401C1
:1003C0000F94E2B34B015C019B01AC01C701B60184
:1003D0000F94D1B46B017C016A966CAD7DAD8EAD8E
:1003E0009FAD6A979058A50194010F94D1B46A9675
:1003F0006CAF7DAF8EAF9FAF6A97A2966CAD7DADAF
:100400008EAD9FADA2979058A50194010F94D1B4E1
:10041000CE57DF4F688379838A839B83C258D0404D
:10042000A5019401C301B2010F94D1B44B015C0149
:100430004090BD155090BE156090BF157090C015CE
:100440008091C1159091C215A091C315B091C415AA
:10045000A2968CAF9DAFAEAFBFAFA297C092AD15C5
:10046000D092AE15E092AF15F092B015CE57DF4F97
:1004700088819981AA81BB81C258D0408093B115EF
:100480009093B215A093B315B093B4156A968CAD42
:100490009DADAEADBFAD6A978093B5159093B6157F
:1004A000A093B715B093B8158092B9159092BA156C
:1004B000A092BB15B092BC15C701B6019058A3011C
:1004C00092010F94E9A76B017C01A2962CAD3DAD82
:1004D0004EAD5FADA2976A966CAD7DAD8EAD9FAD12
:1004E0006A970F94E9A79B01AC01C701B6010F946D
:1004F000E2B36093BD157093BE158093BF159093C2
:10050000C015CE57DF4F688179818A819B81C2589F
:10051000D0409058A30192010F94E9A76B017C0190
:10052000A2962CAD3DAD4EAD5FADA297C501B40115
:100530000F94E9A79B01AC01C701B6010F94E2B388
:100540006093C1157093C2158093C3159093C41521
:1005500080E090E00F94B11217FD53C04DEB55E1D0
:1005600065EB75E18DEA95E10F94662B4091BD1521
:100570005091BE156091BF157091C01585EE9FE03A
:100580000F947BB34091C1155091C2156091C31572
:100590007091C41589EE9FE00F947BB34091AD1527
:1005A0005091AE156091AF157091B0158DED9FE033
:1005B0000F947BB34091B1155091B2156091B31572
:1005C0007091B41581EE9FE00F947BB34091B51507
:1005D0005091B6156091B7157091B81585ED9FE0F3
:1005E0000F947BB34091B9155091BA156091BB152A
:1005F0007091BC1589ED9FE00F947BB30F94EB2AAB
:1006000009C00E3F9FEF190729F4AF96AFADAF9722
:10061000A23049F038010BC0AF961FAEAF976624E9
:100620006A94762C04C0BEEF6B2E77247A94C8555A
:10063000DF4F88819981C85AD0400E94AEA580E0E2
:1006400090E0A0EAB0E480933D1090933E10A09318
:100650003F10B09340102091391030913A104091E2
:100660003B1050913C106091351070913610809184
:10067000371090913810EEEFFCE0FF93EF93812C50
:10068000912CE0EAAE2EE1E4BE2EF1E4CF2EF0E1B3
:10069000DF2EE12CF12C00EA10E4F7D30F948683CF
:1006A0000F900F9077FC22C020E030E046E153E449
:1006B00060913D1070913E1080913F1090914010DC
:1006C0000F94E3B360933D1070933E1080933F10FE
:1006D0009093401065E575E585E591E40F947D2ADA
:1006E00082E39AE10F9435080F948A3281E00F94E7
:1006F000153782E00F94812FBFEF6B167B0631F424
:1007000085EF99E10F94350810E04BC0EEEF6E16BF
:10071000EFEF7E0681F4AF96FFADAF97FF2329F090
:10072000F23031F08EEA98E1EDCF83E399E1EACF40
:1007300083EF98E1E7CFAF96EFACAF97E11007C03A
:1007400023E06216710498F083E399E117C0AF9635
:100750003FADAF97323019F480EB99E102C086E6E5
:1007600099E10F9435081614170454F309C0F301E6
:10077000EE0FFF1FE553FD4F808191810F943508E7
:100780006720609409F286EE0E948EA98FE59FE0B3
:100790000F9457B3813021F087E59AE10F94350823
:1007A00011E00F9452372BC186E19FE10F94350879
:1007B00010E025C183E0821B282F0C94A37281E0F6
:1007C0000C940274F0E9CF1AF1E0DF0A0C94447340
:1007D000EB968FADEB97EC969FADEC970C94E37492
:1007E00080910B018E7F0C942F75B0E44B2E512C11
:1007F000612C712C0C94457587E190E00C9459752F
:100800008F3F910509F014F40C9461758FEF90E01F
:100810000C9461758B7F0C946975E0E6EE16E9E047
:10082000FE0614F00C94787584E00E9432BDFFEF50
:10083000EF1AFF0A0C947875C6010C9498758150D4
:10084000883011F00C9472760C94797600E00C9458
:10085000877680E090E00C94AC764B3011F40C94E9
:100860001E77222311F02B3029F4F7E0FA1510F44B
:100870000C9426777101E20EF31EF701EA57F84F48
:10088000F081A396FFAFA397E496EEADFFADE4979A
:10089000E080F180CC24C394D12C022E02C0CC0C79
:1008A000DD1C0A94E2F7EC20FD20EF2831F0A3963E
:1008B000FFADA397F13148F005C0A396EFADA39724
:1008C000E13118F401960C94267701970C94267761
:1008D00080E00C94B27784EF91E00F94294F882345
:1008E00011F40C94BD7714E0812C912C5401C12C8F
:1008F000D12C760188EE93E00F94294F882311F4D0
:100900000C94BD778091251090912610A09127100E
:10091000B0912810092E000CAA0BBB0BC80ED91ED3
:10092000EA1EFB1E8091291090912A10A0912B1095
:10093000B0912C10092E000CAA0BBB0B880E991E2F
:10094000AA1EBB1E1150B1F640902D1050902E10D3
:1009500060902F1070903010C501B40122E0969580
:100960008795779567952A95D1F732E0F694E794C5
:10097000D794C7943A95D1F700E028EC30E0A20173
:10098000C6010F94E34D11E00C94BE7729813A81A2
:100990002059374F3A8329830C940274F201258140
:1009A000368147815085EA966CAD7DAD8EAD9FADA9
:1009B000EA970C94477AF201258136814781508568
:1009C000EA966CAD7DAD8EAD9FADEA970C94607AE2
:1009D00060E070E080E89FE30C94627A112311F4E8
:1009E0000C94707A812C912C50E8A52E5FE3B52EE3
:1009F0000C944B7A01110C94367A0C94707A81E045
:100A00000F94153780E00F948A66812FC753DF4F0C
:100A10000FB6F894DEBF0FBECDBFDF91CF911F910F
:100A20000F91FF90EF90DF90CF90BF90AF909F908D
:100A30008F907F906F905F904F903F902F90089590
:100A40002F923F924F925F926F927F928F929F92DE
:100A5000AF92BF92CF92DF92EF92FF920F931F93CC
:100A6000CF93DF93CDB7DEB76A970FB6F894DEBFAA
:100A70000FBECDBF1C0128013901FC01E45BFF4F13
:100A800080809180A280B3809A01AB01C501B4013E
:100A90000F94E9A70F94BAB40F9448B56B017C0189
:100AA000A3019201C501B4010F94E9A70F94BAB450
:100AB0000F9448B528E7C216D104E104F10428F4E4
:100AC00048E7C42ED12CE12CF12CD101D7968D9082
:100AD0009D90AD90BC90DA97C986DA86EB86FC864D
:100AE0008C149D04AE04BF0420F489869A86AB86DC
:100AF000BC86683771058105910520F468E770E0D0
:100B000080E090E06B017C0186169706A806B90686
:100B100010F475016401F101ED5BFF4F40805180DD
:100B20006280738049825A826B827C824528462883
:100B3000472841F4412C512C3201439449825A8276
:100B40006B827C8229853A854B855C85CA01B90117
:100B50000F9498B36D877E878F87988BA50194013A
:100B6000C501B4010F9498B34B015C01A701960134
:100B7000C701B6010F9498B3698B7A8B8B8B9C8BD2
:100B800049805A806B807C80440C551C661C771C05
:100B90004D825E826F827886D501C4010197A109DA
:100BA000B1094D845E846F84788884199509A609FB
:100BB000B7094D805E806F807884480E591E6A1E8A
:100BC0007B1EC301B2012D813E814F8158850F9458
:100BD000A7B329013A01C501B40129893A894B8992
:100BE0005C89621B730B840B950B2D813E814F81B9
:100BF00058850F94A7B3DA01C901840D951DA61D70
:100C0000B71DF10180889188A288B388881599055D
:100C1000AA05BB0528F4881A990AAA0ABB0A9CC02F
:100C200029813A814B815C8182E0220F331F441F6E
:100C3000551F8A95D1F7D501C40181709927AA273C
:100C4000BB2789839A83AB83BC83240135017694C7
:100C50006794579447944F8A588E698E7A8E4D8444
:100C60005E846F84788889899A89AB89BC89841568
:100C70009505A605B705C0F1D301C20180959095F1
:100C8000A095B09549885A886B887C88840D951DFD
:100C9000A61DB71DBC01CD01620F731F841F951FD8
:100CA00049805A806B807C8045284628472841F03F
:100CB0004D805E806F807884640D751D861D971D44
:100CC0000F94A7B38F89988DA98DBA8D820F931F2A
:100CD000A41FB51F2401350188159905AA05BB0578
:100CE000C0F52C013D0135C06D857E858F859889C5
:100CF00049885A886B887C88641975098609970920
:100D000049805A806B807C8045284628472841F0DE
:100D10004D805E806F807884640D751D861D971DE3
:100D20000F94A7B34F88588C698C7A8C420E531E4F
:100D3000641E751ED501C401481459046A047B045D
:100D400010F4D301C20124013501481A590A6A0A74
:100D50007B0A812C912C54018FB7F894F101E55B4B
:100D6000FF4F908191111FC0D1015A964D925D9213
:100D70006D927C925D97840C951CA61CB71CF101AA
:100D8000868E978EA0A2B1A249845A846B847C84FB
:100D9000DB964D925D926D927C92DE97FF96C082BB
:100DA000D182E282F3828FBF6A960FB6F894DEBFDB
:100DB0000FBECDBFDF91CF911F910F91FF90EF90AC
:100DC000DF90CF90BF90AF909F908F907F906F906B
:100DD0005F904F903F902F9008950F931F93CF9364
:100DE000C82F0F94B8828AEE0F946A820F9488827B
:100DF000811103C00F94AF8235C08C2F0F946A828B
:100E00000F948882882371F10F94AF820F94B88277
:100E10008BEE0F946A820F948882882319F1599A75
:100E200028E02A95F1F7519887E090E0C0E0589AC1
:100E300028E02A95F1F729B121FB002700F910E0FD
:100E40009801082E01C0220F0A94EAF7C22B589885
:100E500028E02A95F1F7019750F7519A0F94AF8245
:100E60008C2F06C08FEF80931D0D80931C0D80E0AA
:100E7000CF911F910F910895CF93C82F0F94042005
:100E8000C150E1F7CF910D940F202F923F924F92D6
:100E90005F926F927F928F929F92AF92BF92CF920A
:100EA000DF92EF92FF920F931F93CF93DF93CDB713
:100EB000DEB7C358D1090FB6F894DEBF0FBECDBF61
:100EC00069A37AA38BA39CA32DA33EA34FA358A7EA
:100ED000E496ECAEFDAE0EAF1FAFE497E696DFAE44
:100EE000CEAEE6978BA699A6AFA6B8AAC756DF4F97
:100EF00088809980C959D0409AAE89AE8091000708
:100F00008F5FA6968FAFA697803119F4A6961FAE75
:100F1000A697A6969FACA697092D990C110B8091C8
:100F2000FF0690E00817190709F452C0BE016B5D77
:100F30007F4FCE0181960E94B7A749A05AA06BA00F
:100F40007CA020917D1030917E1040917F105091B7
:100F50008010C301B2010F94E9A70F94DBB6AA96E3
:100F60006CAF7DAF8EAF9FAFAA978DA09EA0AFA0B4
:100F7000B8A420918110309182104091831050913B
:100F80008410C501B4010F94E9A70F94DBB6AE96A7
:100F90006CAF7DAF8EAF9FAFAE9780918C158823DD
:100FA00069F1A5019401C301B2010F947C77E49625
:100FB0002CAD3DAD4EAD5FADE4970F94E3B3209102
:100FC000851030918610409187105091881024C070
:100FD0001092260D0F94AA7D80E00F945C0E80E0A5
:100FE0000F94812F8091FF0690E00817190791F365
:100FF0008091260D81110C94699598CF20918510D0
:10100000309186104091871050918810E4966CAD15
:101010007DAD8EAD9FADE4970F94E9A70F94DBB63D
:101020006F966CAF7DAF8EAF9FAF6F97E696AEAD0C
:10103000BFADE697CD90DD90ED90FC9020918910AA
:1010400030918A1040918B1050918C10C701B601DD
:101050000F94E9A70F94DBB669966CAF7DAF8EAFA6
:101060009FAF69972091591030915A1040915B10B1
:1010700050915C10C301B2010F94E2B32B013C010B
:1010800020915D1030915E1040915F105091601082
:10109000C501B4010F94E2B34B015C01A3019201BD
:1010A000C301B2010F94E9A72B013C01A5019401F2
:1010B000C501B4010F94E9A79B01AC01C301B201C2
:1010C0000F94E3B30F9467B7C058DF4F68837983F9
:1010D0008A839B83C058D040209165103091661060
:1010E0004091671050916810C701B6010F94E2B3A8
:1010F000A5966CAF7DAF8EAF9FAFA5978091751011
:1011000090917610A0917710B091781069968CAC80
:101110009DACAEACBFAC699788169906AA06BB0613
:1011200009F4C4C0E091FE0C04E0E09FF00111243A
:10113000E452F04F20912402309125024091260282
:101140005091270260817181828193810F947CAEDE
:1011500087FF33C08092751090927610A09277101E
:10116000B0927810C0926510D0926610E09267102D
:10117000F0926810E6E9FEE584918F01882339F04A
:101180000E9462AD0F5F1F4FF8018491F7CFECEA28
:10119000FFE184918F01882339F00E9462AD0F5FD7
:1011A0001F4FF8018491F7CF8AE00E9462ADA596A7
:1011B0001CAE1DAE1EAE1FAEA5978091751090910E
:1011C0007610A0917710B091781069968CAC9DAC98
:1011D000AEACBFAC6997881A990AAA0ABB0AC501C6
:1011E000B401B7FE07C090958095709561957F4FCB
:1011F0008F4F9F4F0F9482AE6B017C0120E030EC4B
:101200004BEE53E46091891070918A1080918B109D
:1012100090918C100F94E9A79B01AC01C701B60116
:101220000F942EB618160CF041C06996ACACBDAC4C
:10123000CEACDFAC6997A0927510B0927610C092D8
:101240007710D0927810E696EEADFFADE6978081EC
:101250009181A281B3818093651090936610A093D1
:101260006710B0936810E6E9FEE584918F0188234A
:1012700039F00E9462AD0F5F1F4FF8018491F7CFE4
:10128000EEE8FFE184918F01882339F00E9462AD7E
:101290000F5F1F4FF8018491F7CF8AE00E9462AD83
:1012A000A5961CAE1DAE1EAE1FAEA5978091000781
:1012B000282E312CF7E58F9FC00111248A57984FB3
:1012C000FC01EB5AFF4F118210823A9710828090F6
:1012D000691090906A10A0906B10B0906C102196DD
:1012E0008CAE9DAEAEAEBFAE2197AA964CAD5DADB5
:1012F0006EAD7FADAA97481959096A097B0977FF36
:1013000007C070956095509541955F4F6F4F7F4F27
:1013100087E5829DF001839DF00D1124EA57F84F77
:10132000408351836283738340906D1050906E10A0
:1013300060906F1070907010AE960CAD1DAD2EAD1C
:101340003FADAE97041915092609370937FF07C0C5
:1013500030952095109501951F4F2F4F3F4FE7E592
:10136000E29DC001E39D900D1124FC01EA57F84F66
:101370000483158326833783A0907110B090721078
:10138000C0907310D0907410A9AABAAACBAADCAAF4
:101390006F968CAD9DADAEADBFAD6F978A199B09B1
:1013A000AC09BD09B7FF07C0B095A0959095819590
:1013B0009F4FAF4FBF4FF7E5BF2EB29CF001B39CDC
:1013C000F00D1124EA57F84F80879187A287B387E1
:1013D000C0907510D0907610E0907710F090781053
:1013E000CDAADEAAEFAAF8AE69968CAC9DACAEACE5
:1013F000BFAC69978C189D08AE08BF08B7FE08C03F
:10140000B094A09490948094811C911CA11CB11C58
:10141000E7E5EE2EE29CF001E39CF00D1124EA5783
:10142000F84F84869586A686B78688159905AA05FD
:10143000BB0514F4D501C4014A015B018017910773
:10144000A207B30744F0481759076A077B0754F40B
:101450004C015D0107C0401751076207730714F480
:101460004801590187E5829DF001839DF00D11240B
:10147000EA57F84F808A918AA28AB38A06E08016DA
:101480009104A104B10414F40C946995DF01A95BE3
:10149000BF4F8091BB199091BC198C01990F220B01
:1014A000330B0D931D932D933C931397AA968CACFD
:1014B0009DACAEACBFACAA972196CCACDDACEEAC8B
:1014C000FFAC21978C149D04AE04BF0414F0108E61
:1014D00002C081E0808FAE96ECACFDAC0EAD1FADCE
:1014E000AE97E414F504060517055CF487E5829DC4
:1014F000F001839DF00D1124EA57F84F808D826032
:10150000808F89A89AA8ABA8BCA86F96CCACDDAC9C
:10151000EEACFFAC6F97C814D904EA04FB045CF48A
:1015200087E5829DF001839DF00D1124EA57F84F65
:10153000808D8460808F6996ECACFDAC0EAD1FADE4
:1015400069978DA89EA8AFA8B8ACE814F9040A055D
:101550001B055CF487E5829DF001839DF00D11244D
:10156000EA57F84F808D8860808FA9ADBAAD8C9115
:1015700097E5929DF001939DF00D1124EA57F84FE5
:10158000818F452B462B472B09F0179887E5829DC5
:10159000F001839DF00D1124EA57F84F8481958165
:1015A000A681B781892B8A2B8B2B09F0169887E5AA
:1015B000829DF001839DF00D1124EA57F84F80853C
:1015C0009185A285B385892B8A2B8B2B09F01598E1
:1015D00087E5829DF001839DF00D1124EA57F84FB5
:1015E00084859585A685B785892B8A2B8B2B11F44D
:1015F0000C9463958091230D882319F0815080937A
:10160000230D8091240D882319F081508093240D9F
:101610008091250D882319F081508093250DE9AD27
:10162000FAAD8081813061F030F0823089F480E25F
:101630008093250D08C0149880E28093230D08C084
:1016400080E28093240D8091230D811128C0149A8B
:1016500087E5829DF001839DF00D1124EA57F84F34
:1016600084849584A684B78489AE9AAEABAEBCAEB2
:1016700089288A288B2819F5E090B910F090BA10C3
:101680000091BB101091BC102BA539A54FA558A9EE
:10169000B701C8010F942EB618163CF522C087E595
:1016A000829DF001839DF00D1124EA57F84F848448
:1016B0009584A684B78489AE9AAEABAEBCAEE090FA
:1016C000B510F090B6100091B7101091B8109701B6
:1016D000A8016BA579A58FA598A90F947CAE87FF6B
:1016E00004C0EBA6F9A60FA718AB809169109091E2
:1016F0006A10A0916B10B0916C10AA96ACACBDAC06
:10170000CEACDFACAA97A81AB90ACA0ADB0AC6018E
:10171000B5010F9482AE20917D1030917E104091E2
:101720007F10509180100F94D1B421966CAF7DAF93
:101730008EAF9FAF219769837A838B839C83AE960C
:101740006CAD7DAD8EAD9FADAE9764197509860900
:1017500097090F9482AE20918110309182104091B0
:101760008310509184100F94D1B44B015C016D83B0
:101770007E838F8398876F966CAD7DAD8EAD9FAD68
:101780006F97C9A8DAA8EBA8FCA86C197D098E0987
:101790009F090F9482AE2091851030918610409160
:1017A0008710509188100F94D1B46B017C01698728
:1017B0007A878B879C8769966CAD7DAD8EAD9FAD2A
:1017C00069970DA91EA92FA938AD601B710B820B5B
:1017D000930B0F9482AE2091891030918A10409122
:1017E0008B1050918C100F94D1B46D877E878F87AA
:1017F000988B27E5229DF001239DF00D1124EA57D7
:10180000F84F208131814281538125962CAF3DAF25
:101810004EAF5FAF25972630310541055105D4F411
:101820000481158126813781063011052105310596
:101830008CF400851185228533850630110521053C
:10184000310544F4DC01CB01BF7786A797A7A0AB95
:10185000B1AB2EC021966CAD7DAD8EAD9FAD219705
:101860000F94E6A72B013C01C501B4010F94E6A734
:101870009B01AC01C301B2010F94E3B34B015C01C6
:10188000C701B6010F94E6A79B01AC01C501B401E5
:101890000F94E3B30F9467B727E5229DF001239DD2
:1018A000F00D1124EA57F84F66A777A780AB91ABEC
:1018B00087E5829DF001839DF00D1124EA57F84FD2
:1018C00046A457A460A871A8A301920160E070E04B
:1018D00080E89FE30F94D1B42BA539A54FA558A953
:1018E0000F94E9A76B017C01809100079091FF069E
:1018F000891B8F708DAF90E00297069708F042C069
:10190000A701960160E074E284E799E40F94D1B4F2
:101910000F94DBB64B015C018091BD109091BE101D
:10192000A091BF10B091C01088169906AA06BB06F8
:1019300048F588199909AA09BB09BC01CD01660FB0
:10194000771F881F991FCDAC0C2D10E020E030E0F0
:10195000A90198010F94A7B3CA01B9010F9480AEF1
:101960000F94DBB6680D791D8A1D9B1D0F9480AE08
:101970009B01AC0160E074E284E799E40F94D1B478
:101980006B017C01A3019201C701B6010F94E9A785
:1019900029966CAF7DAF8EAF9FAF299787E5829D6B
:1019A0008001839D100D11240A57184F29968CAC85
:1019B0009DACAEACBFAC2997D80192968D929D920A
:1019C000AD92BC92959750966D917D918D919C9121
:1019D00053970F9480AE6BA77CA78DA79EA79B0102
:1019E000AC01C701B6010F94E9A70F94BAB40F94E4
:1019F00048B52D966CAF7DAF8EAF9FAF2D97F80198
:101A000067AB70AF81AF92AF8090220D8DAA8E012F
:101A10000F5F1F4F63961FAF0EAF6397005F1F4F9F
:101A2000A1961FAF0EAFA19780902B0290902C0231
:101A30006B969FAE8EAE6B9765961FAF0EAF659798
:101A400000E010E019A61FA620E828AB3FE339AB61
:101A50006396AEADBFAD63972D913D914D915D9174
:101A60006396BFAFAEAF6397C701B6010F94E9A706
:101A70006596EEADFFAD65976193719381939193F8
:101A80006596FFAFEEAF65974B015C01E894B7F840
:101A90006B96AEADBFAD6B972D913D914D915D9124
:101AA0006B96BFAFAEAF6B9761962CAF3DAF4EAFAD
:101AB0005FAF6197C501B4010F942EB6181614F5E7
:101AC000A501940161966CAD7DAD8EAD9FAD619722
:101AD0000F94D1B45B014C0129A53FA548A959A990
:101AE0000F942EB6181624F0A9A6BFA688AA99AA04
:101AF00081E090E0002E01C0880F0A94EAF78DA8DB
:101B0000882A8DAA0F5F1F4F0430110509F0A0CF5E
:101B10009DA89092220D20E030E040E85FE369A5A7
:101B20007FA588A999A90F947CAE87FF4CC07E0140
:101B300001E2E00EF11CA1960EAD1FADA19729A503
:101B40003FA548A959A9D8016D917D918D919C918E
:101B50000F94E9A7F80161937193819391938F0199
:101B6000EE15FF0561F787E5829D8001839D100DCD
:101B700011240A57184F29962CAD3DAD4EAD5FADDF
:101B8000299769A57FA588A999A90F94E9A7D801E4
:101B900092966D937D938D939C9395972D966CADB6
:101BA0007DAD8EAD9FAD2D970F9480AE29A53FA53D
:101BB00048A959A90F94E9A70F9448B5F80167AB54
:101BC00070AF81AF92AFA30192016BA57CA58DA5EB
:101BD0009EA50F94D1B42B013C0125968CAC9DACF5
:101BE000AEACBFAC259789288A288B2891F587E56C
:101BF000829D8001839D100D11240A57184FF80112
:101C000084819581A681B781892B8A2B8B2B09F53D
